:020000040800F2
:10000000A837001081020008936600080357000813
:100010009166000841170008758E00080000000076
:10002000000000000000000000000000A101000826
:100030002D21000800000000FD010008F5770008F0
:100040009B0200089B0200089B0200089B0200081C
:100050009B0200089B0200089B0200089B0200080C
:100060009B0200089B0200089B0200089B020008FC
:100070009B0200089B020008E91D0008F51D00080E
:10008000011E00080D1E00089B0200089B020008CC
:100090009B0200089B0200089B0200089B020008CC
:1000A0009B0200089B0200089B0200089B020008BC
:1000B0009B02000800000000000000009B020008F6
:1000C0009B0200089B0200089B0200089B0200089C
:1000D0009B020008058D0008518D00089B02000856
:1000E0009B0200089B0200080000000000000000C6
:1000F0000000000000000000000000000000000000
:10010000000000009B020008000000009B020008A5
:100110000000000000000000818100089B02000830
:100120009B0200089B0200089B0200089B0200083B
:100130009B0200080000000000000000000000001A
:100140009B0200089B0200089B02000800000000C0
:100150009B0200089B0200089B0200089B0200080B
:100160009B0200089B0200089B02000800000000A0
:100170009B0200089B020008000000000000000035
:100180009B0200089B0200089B020008DFF80CD0CD
:1001900000F068FE0048004765AC0008A837001072
:1001A0002C4B1968086800F05AB880F30988BFF32F
:1001B0006F8F4FF0000080F311887047000000003F
:1001C00008480068006880F308884FF0000080F35A
:1001D000148862B661B6BFF34F8FBFF36F8F00DF35
:1001E00000BF00BF08ED00E0DFF80C00016841F43B
:1001F00070010160704700BF88ED00E0EFF30980F7
:10020000BFF36F8F134B1A681EF0100F08BF20ED5D
:10021000108A20E9F04F106009B44FF0500080F3CD
:100220001188BFF34F8FBFF36F8F0CF00DFE4FF0AF
:10023000000080F3118809BC1968086800F014B840
:100240001EF0100F08BF00F014B880F30988BFF348
:100250006F8F7047D4000020EFF30580704730C8DF
:10026000B0E8C04FFFF7A1BF30C8B0E8C04FFFF7FC
:10027000E7BFB0EC088AB0EC08CAFFF7E6BF0000A1
:100280000648804706480047FEE7FEE7FEE7FEE730
:10029000FEE7FEE7FEE7FEE7FEE7FEE7717800080F
:1002A0008D0100082DE9F05F0546002092469B462F
:1002B00088460646814640241BE02846414647467C
:1002C000224600F0F9FB53465A46C01A914110D31A
:1002D00011461846224600F0E0FB2D1A67EB010894
:1002E0004F4622460120002100F0D7FB17EB000902
:1002F0004E41201EA4F10104DFDC484631462A4667
:10030000434600F000B830BCBDE8C09F40EA01039E
:100310009B0703D009E008C9121F08C0042AFAD2BB
:1003200003E011F8013B00F8013B521EF9D270477F
:10033000D2B201E000F8012B491EFBD27047002227
:10034000F6E710B513460A4604461946FFF7F0FFD4
:10035000204610BD421E12F8013F002BFBD111F8C0
:10036000013B02F8013B002BF9D1704730B505463F
:100370002A460B4612F8010B13F8014B08B1A042B4
:10038000F8D01CB1002802D06D1CF1E7284630BD22
:1003900010B5044604E00B7800F8013B03B1491C9A
:1003A000521EF8D2204610BDCAB2401E10F8011FDE
:1003B0008A4202D00029F9D100207047421C10F86F
:1003C000011B0029FBD1801A704710B5002200E004
:1003D000521C835C8C5CA34201D1002BF8D1D8B2B3
:1003E000E1B2401A10BDCBB203E00178994203D0CC
:1003F000401C521EF9D20020704730B50446002040
:10040000034600E05B1C934203D2E05CCD5C401BE2
:10041000F8D030BD034611F8012B00F8012B002A5B
:10042000F9D11846704730B505460020034600E074
:100430005B1C934205D2EC5CC85C201A01D1002CF5
:10044000F6D130BD0FB400B58DB010A909900B9056
:1004500000914FF0FF300A9000200C900548069064
:10046000054807906A4609A80F9900F069FB0DB08E
:100470005DF814FB5D0B00087B0B00082DE9FF5FA6
:100480001D464FF0FF3BD5E9014691465F464FF0D0
:100490000008A9697F1C01988847296A8246884715
:1004A0000028F6D1BAF1FF3F0CD024F4C064002E2E
:1004B00019DD600614D5BAF12B0F09D0BAF12D0F52
:1004C0000ED103E0584604B000F07EB844F48064D6
:1004D000A9697F1C01988847761E8246002E02DD9E
:1004E000BAF1300F03D0B9F1000F26D032E0A9697C
:1004F000761E44F400747F1C019888478246002EC3
:1005000005DDBAF1780F06D0BAF1580F03D0B9F172
:10051000000F10D01EE0B9F1000F02D0B9F1100F9A
:1005200018D1A969761E24F400747F1C01988847AD
:100530008246102002E0082000E00A20814609E0FF
:1005400008FB0908A969761E44F400747F1C019811
:1005500088478246002E05DD4946504600F0DBFA0A
:100560000028EDDAE96901988847A00502D46FF008
:100570000100A8E7E00725D1600613D5600502D584
:10058000C8F1000000E0404629680A1D2A60096899
:10059000220501D5087015E0220701D5088011E079
:1005A00008600FE02868011D29600068210502D558
:1005B00080F8008006E0210702D5A0F8008001E065
:1005C000C0F8008038467EE730BCBDE8C09F2DE90A
:1005D000F04791460F4680460446002614F8015B1A
:1005E0002DB100F08BFA0068405DC007F6D12B2DCD
:1005F00002D02D2D18D0641E4A463946204600F000
:10060000CDFA27B13968A14201D1C7F80080710540
:100610004FF002040BD54042002803DD08F0AAFC8D
:100620000460A007BDE8F08746F48066E4E7002890
:10063000F8DA08F09FFC04606FF00040F2E72DE963
:10064000F05F93460F4680460446002608F092FC71
:10065000D0F80090824614F8015B2DB100F04EFAFC
:100660000068405DC007F6D12B2D02D02D2D1AD089
:10067000641E0021CAF800105A463946204600F090
:100680008DFA014627B13868A04201D1C7F8008031
:10069000DAF80000022809D0CAF80090700505D5E4
:1006A000484200F005B846F48066E2E70846F8E7FD
:1006B00030BCBDE8C09F70B5064608F05BFC04681E
:1006C00005460A2200213046FFF781FF2C6070BDED
:1006D0002DE9FE4F804681EA0300C00F0C460090D2
:1006E00021F0004123F00045B8EB0200A94105D2FA
:1006F0004046214690461C460B46024623F00040E9
:10070000104347D0270DC7F30A00C3F30A510290E4
:10071000401A019040286BDAC3F3130040F4801BA9
:100720000098924620B10023D2EB030A63EB0B0B37
:1007300001985946C0F14002504600F0AEF9064615
:100740000D4650465946019A00F0C6F910EB0800D4
:100750006141002487EA115284EAE7731A4340D0CA
:10076000009A62B3019A012A4FEA075215DC001B76
:1007700061EB02014FF0004202EA0752CDE900426C
:10078000001C41F5801132462B4600F0EDFA03B013
:1007900000F045B840462146F9E7001B61EB020135
:1007A000001C41F5801300185B412018A2F50017CA
:1007B00047EB030140EAD570B6196D4111E06D08B1
:1007C0004FEA360645EAC0754FEA0752001B61EB57
:1007D0000201001C41F5801149084FEA3000001960
:1007E000514132462B4603B000F01CB800F0ADBAC0
:1007F0000098012240000023D0EB020263EBE0737B
:10080000009821464FEAE074B8EB000061EB040168
:10081000E9E783F000435BE781F0004158E730BC33
:10082000BDE8C08F30BCBDE8C04FFFF7DFBF2DE98A
:10083000FE4F81EA030404F0004421F000410094DB
:100840004FF0000B23F0004350EA01045ED052EA5F
:1008500003045BD0C3F30A54C1F30A552C44A4F239
:10086000F3340194A0FB0254C1F3130141F480114D
:10087000C3F3130343F4801301FB024400FB034E54
:10088000840A970A44EA815447EA8357A4FB07681D
:1008900002958D0A05FB07854FEA932C04FB0C5447
:1008A0002705029D4FEA065847EA1637B5EB0805BB
:1008B0006EEB070C870E920E47EA811742EA83120D
:1008C000A7FB0201B6EB0B0164EB00042B0D43EA1E
:1008D0000C335E1844EB1C50DA465146E7FB02012C
:1008E000C5F313044FEA0B3343EA14534FEA0432BF
:1008F000019C43EA0603A4F10C040294009CCDE998
:1009000000B400F031FA03B000F003B80020014653
:10091000F9E730BCBDE8C08F2DE9F04D81EA030452
:1009200004F0004B21F0004514464FF0000A23F07C
:10093000004150EA050220D054EA01021DD0C5F35F
:100940000A570246C5F31303C1F31300C1F30A5655
:1009500040F4801543F48013A7EB0608101BD6461D
:1009600008F2FD3873EB050002D308F1010801E03D
:1009700092185B41B8F1000F03DA00200146BDE890
:10098000F08D00204FF48011064684460EE0171BC0
:1009900073EB050705D3121B63EB050306434CEA13
:1009A000010C49084FEA300092185B4150EA0107F8
:1009B000EDD152EA030012D082EA040083EA050175
:1009C000084305D0101BAB4106D20122002306E0EC
:1009D00000224FF0004302E06FF0010253101AEBC7
:1009E00006004CEB085110EB0A0041EB0B01BDE88F
:1009F000F04D00F0AAB90EB540F23341029100214A
:100A0000CDE900110A460B4600F0AEF903B000BD77
:100A100000F0004230F000400AD0C10D01F56071D5
:100A2000C0F3160042EA0151C20840071143704763
:100A300000200146704701F0004330B421F000412E
:100A400050EA010206D00A0DA2F56072C1F313014B
:100A5000002A02DC30BC00207047440F44EAC10485
:100A6000C100E01830BC00EBC25000F037B930B51F
:100A70000B46014600202022012409E021FA02F55C
:100A80009D4205D303FA02F5491B04FA02F52844F6
:100A9000151EA2F10102F1DC30BD202A04DB203A50
:100AA00000FA02F1002070479140C2F1200320FAC1
:100AB00003F3194390407047202A04DB203A21FABF
:100AC00002F00021704721FA02F3D040C2F1200267
:100AD0009140084319467047202A06DBCB17203A7D
:100AE00041FA02F043EAE07306E041FA02F3D04033
:100AF000C2F12002914008431946704700487047F0
:100B000058E5000810B50446FFF7F8FF0068005DDF
:100B100000F0010010BD3A2800D2303820F0200249
:100B2000412A01D3A2F13700884201D34FF0FF30B0
:100B3000704700000268114413780160184670473E
:100B4000D1600449516104491162002111611146CB
:100B500000F09AB9350B0008050B0008426842B155
:100B6000016811F8013B23B1521EC0E9001218467A
:100B700070470121C160881E704742685AB1C3683E
:100B8000016843B983688B4205D0491E521CC0E9F5
:100B90000012002070474FF0FF3070472DE9F05FE2
:100BA00082460078002715468B460AF10104B946B3
:100BB000302801D09DB113E014F8010B01277828EB
:100BC00003D0582801D045B10AE00DB1102D07D14E
:100BD0000027102514F8010B02E0082500E00A2583
:100BE0000026B0460EE005FB080005FB06F10127D4
:100BF00001EB10461FFA80F8B6F5803F00D3B946E6
:100C000014F8010B2946FFF786FF0028EBDABBF149
:100C1000000F05D00FB1641E00E05446CBF8004031
:100C2000B9F1000F06D008F0A5F902210160C81E35
:100C300000F003B848EA0640FAE730BCBDE8C09FC0
:100C40000FB4002300B589B00CA900910B996FF087
:100C50000042CB601E4B06931E4B07930423CDE945
:100C600001321D4A089202466B46002000F026FB26
:100C700009B05DF814FB70B586B006464FF0FF3042
:100C80000091CDE90101002015460C460490324642
:100C9000694604A8FFF7D4FF03460498211825B13C
:100CA00008B10A4600E022462A6000280DD0002B39
:100CB00002DD0098884208D0081B0094CDE90104A9
:100CC0003246694604A8FFF7BBFF06B070BD0000BE
:100CD0005D0B00087B0B0008050B00080029A8BF6E
:100CE0007047401C490008BF20F00100704710B455
:100CF000B0FA80FC00FA0CF050EA010404BF10BC0A
:100D0000704749B1CCF1200421FA04F411FA0CF136
:100D100018BF012121430843A3EB0C01CB1D4FEA6F
:100D200000614FEA102042BF002010BC704700EB6A
:100D3000C35010440029A4BF10BC7047401C490098
:100D400008BF20F0010010BC704710B5141E73F1ED
:100D5000000408DA401C41F1000192185B411A437B
:100D600001D120F0010010BD2DE9F04D92469B46C7
:100D700011B1B1FA81F202E0B0FA80F2203290466D
:100D8000FFF78BFE04460F4640EA0A0041EA0B01DA
:100D900053465A46084313D0114653EA010019D06E
:100DA000C8F140025046FFF787FE05460E46504602
:100DB00059464246FFF771FE084305D0012004E082
:100DC00020463946BDE8F08D0020054346EAE0762E
:100DD0002C4337430A986305E40AA0EB080000227D
:100DE000FD0A44EA47540A3002D500200146E9E7EB
:100DF000010510196941DDE9084500196941BDE89F
:100E0000F04DA2E7C1F30A52C1F3130140F2FF33E0
:100E100041F480119A4202DA00200146704740F204
:100E200033439A42A2F2334202DC5242FFF744BEFD
:100E3000FFF733BE30B5041E71F1000404DB4FF040
:100E40000044404264EB0101141E73F1000405DB11
:100E50001C464FF00043524263EB0403994208BF23
:100E6000904230BD064C074D06E0E06840F00103BB
:100E700094E8070098471034AC42F6D3FFF78AF99C
:100E800020EF000860EF00082DE9F34F8BB04FF022
:100E9000000801F10C000C464FF0010B46460DF125
:100EA000080A01906269012101989047051E2DD022
:100EB000252D2CD0216A8847C0B162690121019893
:100EC0009047216A88470028F7D1411E626901983E
:100ED000904700E0761CA1690B988847216A8847F3
:100EE0000028F7D1E1690B988847DBE7A1690B98E7
:100EF00088470746A84201D1761CD3E7E1690B98E1
:100F000088477F1C02D1B8F1000F6FD046E100275F
:100F100062693D463946019890472A2804D16269A2
:100F20000121019890470125DFF88492626901212F
:100F300001989047A0F130010A290AD24F45E5DC1B
:100F400007EB870100EB4107303FDFD445F0100588
:100F5000ECE7E90601D46FF000476C280AD04C2872
:100F600014D0682815D06A280DD074281CD07A288F
:100F70001AD01DE062690121019890476C2802D0C7
:100F800045F0040514E045F002050DE045F02005AC
:100F90000AE06269012101989047682802D045F073
:100FA000080505E045F40065626901210198904754
:100FB000C4E9015765283DD019DC58287AD00CDCEB
:100FC000452837D004DC252826D0412831D131E00E
:100FD00046282FD047282CD12CE05B2877D06128D9
:100FE00028D063287CD0642823D15AE0D0E06F2831
:100FF00048D008DC66281DD067281BD0692821D07E
:101000006E2816D127E0702845D0732868D075283F
:1010100047D078280DD14DE0A1690B988847054647
:1010200025283FF469AFE1690B9888476D1C3FF4B0
:101030006AAFB3E023466A466FF001000B9900F0F7
:101040003DF99EE045F040006060A80723464FF060
:10105000000236D43EE0E8077FF447AF2068011D68
:1010600021600068290501D506701BE7290701D515
:10107000068017E7A90703D5F117C0E9006111E75A
:1010800006600FE745F040006060A80723464FF078
:10109000080216D41EE040F60E0125EA0100606049
:1010A00016E045F040006060A80723464FF00A02B2
:1010B00007D40FE045F040006060A80708D523463C
:1010C00010226FF001000B99AFF3008059E007E0A8
:1010D000234610226FF001000B99FFF7CFF950E083
:1010E0004FF000094F464B46632802D05B2806D0DC
:1010F00040E0E80601D40120A06001273AE06269DF
:101100000121019890475E2805D14FF001096269DD
:10111000494601989047216939B900210A4653464A
:1011200043F82120491C0829FADBB0B3216969B9C9
:10113000C11700EBD16253110AEB830122F01F02A9
:10114000821A01200B68904003430B606269012101
:10115000019890475D28E8D1B9F1000F09D000202F
:10116000514651F82020D24341F82020401C082845
:10117000F7DB02AB224600976FF001000B99AFF34B
:10118000008000280CDA401C08D1BBF1000F05D00C
:101190004FF0FF300DB000F00DB8FFE74046F9E723
:1011A000E90701D108F1010806444FF0000B79E688
:1011B000CCCCCC0C30BCBDE8C08F00002DE9FF4F7B
:1011C000087881B09946FF2805D0491C2D2804D005
:1011D0000024002308E000230BE00124F9E703EBDF
:1011E000830300EB4303491C0878FF28F7D104B1BF
:1011F0005B4200200090147801462D2C01D02B2C4E
:1012000004D1521C2D2C12D00024009400251678F5
:10121000FF2E0ED00A24A0FB04C801FB0481002786
:1012200000FB0711521C16EB0C006941EFE701248B
:10123000EBE7994450EA01020ED00024AA4D26465D
:10124000DFF8A88200F059F982468B46B9F1000018
:1012500009DAC9F100071BE001980021C0E900117B
:1012600005B000F047B9074612E0F80707D022465C
:101270002B4630464146FFF7DAFA064688462246B4
:101280002B4610461946FFF7D2FA04460D467F104A
:10129000002FEAD1B9F1000F324643465046594675
:1012A00002DAFFF739FB01E0FFF7C1FA009A0AB151
:1012B00081F00041019AC2E90001D1E72DE9FF4F19
:1012C0001F468DB0D7E901464FF0FF382E20454626
:1012D0004FF000090B90B9696D1C0E988847396A68
:1012E000824688470028F6D1BAF1FF3F0AD024F49D
:1012F000D064002E11DDBAF12B0F08D0BAF12D0FFA
:101300000BD102E0404611B0ABE744F48064B96908
:101310006D1C0E9888478246761E6946600501D589
:101320002D2000E02B208DF8000001F1010B0DF1C4
:10133000200809E0B9696D1C0E98884782460F980D
:1013400044F40074761E0560002E02DDBAF1300F01
:10135000F0D00B998A453ED144F0800406E00F9905
:10136000681CA9F1010944F400740860B9696D1C96
:10137000761E0E98884782463028F0D02BE00B99D5
:101380008A4505D1200603D444F08004761E18E077
:10139000504607F0D6FE08B30DF11301761E44F453
:1013A00000748B4508D2AAF130000BF8010B20061F
:1013B00007D5A9F1010003E0200602D409F10100DC
:1013C0008146A00502D50F99681C0860B9696D1C9B
:1013D0000E9888478246002ED1DC53E0002E51DD66
:1013E000BAF1650F02D0BAF1450F4BD1A00549D52E
:1013F000B9696D1C24F44074761E0E9888478246A5
:10140000002E0CDD2B2804D0BAF12D0F07D144F4A7
:101410008074B9696D1C0E9888478246761EE00577
:1014200001D52D2100E02B2108F8011BCDF82C80DF
:1014300021E00DF12901761E44F4007488450CD298
:10144000AAF1300010F0FF0088F8000002D10B99DB
:10145000884509D908F1010806E0E00501D52448CE
:1014600001E042F20F708146B9696D1C0E98884701
:1014700082460F980560002E04DD504607F061FE9D
:101480000028D6D1F9690E988847FF208BF8000014
:1014900088F800000020069007904B466A4608A98D
:1014A00006A8FFF78BFEA00502D46FF001002AE723
:1014B00014F0240F0AD0E00714D1DDE906123868D1
:1014C000031D3B600068C0E900120BE0DDE9060186
:1014D000FFF7B1FA0146E00704D13868021D3A600F
:1014E0000068016028460EE7000024400000F03F3D
:1014F000F1D8FFFF30BCBDE8C08F0EB540F23342DB
:1015000002920022CDE900221346FFF72DFC03B022
:1015100000BD70B58D1810F8014B14F0030201D115
:1015200010F8012B231106D110F8013B03E010F84D
:10153000016B01F8016B521EF9D1ABB110F8012B10
:1015400004F00C048A1A0C2C03D0A2EB84129B1C0E
:1015500008E010F8014BA2EB0422F8E712F8014B67
:1015600001F8014B5B1EF9D5A942D4D3002070BD10
:1015700000EE900A9FED071AF8EEE00A60EE810A8D
:1015800060EE800A00EE101AB8EE401A80EE810A72
:101590007047000000008034144910B50860012233
:1015A00010214FF0904002F047F8052009F0E8FBC9
:1015B000FE2000F05BF8052009F0E2FB0F2000F0B0
:1015C00055F80621002000F087F80021022000F0E5
:1015D00083F8A121032000F07FF8F02000F046F806
:1015E000BDE810400A2009F0CBBB000050010020EC
:1015F0007CB50007000E00F057F84FF09045012130
:10160000284602F014F80128F9D0002210212846BB
:1016100002F012F80120144C8DF8040002460A234F
:1016200001A9206803F079F80A2000F079F80A206F
:1016300000F076F80A2303226946206802F0A6FF2C
:1016400001221021284601F0F7FF9DF800009DF8C7
:101650000110000440EA01209DF802100843010235
:1016600001D540F07F407CBD5001002031B54FF0E6
:10167000904400221021204601F0DEFF09480A2391
:1016800001226946006803F048F8052000F048F898
:1016900001221021204601F0CFFF022000F040F887
:1016A00038BD00005001002070B504464FF0904551
:1016B0000121284601F0BBFF0128F9D044F00801C0
:1016C000012000F009F8FC20FFF7D0FFBDE87040D2
:1016D0000020FFF7CBBF000038B5002200F00F005C
:1016E00040F0500000928DF800008DF802104FF08D
:1016F00090441021204601F09FFF08480A2303224E
:101700006946006803F009F8052000F009F8012295
:101710001021204601F090FF38BD0000500100204C
:101720000549064A0968B1FBF2F1414300E000BFF8
:10173000491EFCD270470000D0000020404B4C00F6
:10174000FEE70000F8B50C46074616467F212A2022
:1017500001F010F805461848A5F54051553920D03C
:101760000021317021709FED150A04468DED000AAD
:1017700080ED0E0A80ED0A0A80ED0B0A00F180066A
:1017800000231A466946F06909F04CFB0028F7D09F
:101790006078002804D02A46394609A007F06CFB7F
:1017A000F8BD407820B12A4639460EA007F064FB08
:1017B00001203070F8BD0000000000200000000093
:1017C0005B54464443323231342D25645D206572CA
:1017D000726F723A2049443D3078253034580D0AF2
:1017E000000000005B54464443323231342D2564FE
:1017F0005D206F6B3A2049443D3078253034580DD8
:101800000A000000C4B0184C4FF487770126A4F1F9
:101810008005E06840B100231A46694609F002FBE2
:1018200038B1001D0AD015E010A007F025FB0120FB
:1018300016E0694615A007F01FFB0BE014A007F0A7
:101840001BFBE06809F0D8FA00223946202009F095
:101850001BFBE060287810B900F0DEF82E700F2036
:1018600009F08EFAD5E70000800000204661696C1F
:10187000656420746F20637265617465207072699D
:101880006E74207175657565210A0000257300006E
:101890005B435249544943414C5D20517565756520
:1018A00020636F7272757074696F6E206465746501
:1018B0006374656421205265696E69742E2E2E0A48
:1018C000000000000FB400B5C5B047AB4FF48771FE
:1018D0006846469A07F008FB074800231A466946FF
:1018E000006809F0FDFA010002D004A007F0C4FA74
:1018F00045B05DF814FB00008C0000205B5741529E
:101900004E5D204661696C656420746F2073656E5E
:1019100064206C6F6720746F207175657565202871
:101920007374617475733D2564290A0070B513469C
:101930000A46032804D3014613A007F09DFA09E0E4
:1019400052B14FF40064A3420AD22246194616A0AF
:1019500007F092FA002070BD22A007F08DFAF9E797
:10196000284951F8201000205B1E08E00D5C15543A
:101970000D5CFF2D05D0401C80B2A04201D29842E0
:10198000F4DB0021115470BD5B44425F44756D70FF
:101990005D20496E76616C69642044422049443A76
:1019A0002025640A000000005B44425F44756D70AE
:1019B0005D2042756666657220746F6F20736D617D
:1019C0006C6C3A206275665F6C656E203D20256404
:1019D0002C207265717569726564203D2025640A4A
:1019E000000000005B44425F44756D705D204E5501
:1019F0004C4C2062756666657220706F696E746506
:101A0000720A000008DE000810B500F077F8BDE8A3
:101A1000104000F055B900002DE9F0413D27234D5D
:101A20009AB0002405EBC400242146686846FEF7FE
:101A300086FC3D213046FEF7B7FCC8B1821B9046BC
:101A400031466846FEF7A4FC00200DF8080040214E
:101A500009A8FEF774FC15F83400402309AA69466A
:101A600009F098FE20B915F83400314605F0AEFCB7
:101A70000F4801F020FE012009F082F9641CBC42ED
:101A8000D0D30D480B4A0DA14261002000F004F9AB
:101A90000CA007F0F1F9642009F072F9FFF7B4FF28
:101AA0001AB010A0BDE8F04107F0E6B914DE000856
:101AB00030270010ECC007004032001076657273CA
:101AC000696F6E0044425F496E6974416C6C436F8C
:101AD0006E6669677320636F6D706C6574652E0A3E
:101AE0000000000044425F44756D705F746F5F4A90
:101AF00073526F6F74206F6B200D0A002DE9F04157
:101B0000094D0A4E00244FF4006700BF05EBC421C5
:101B10003A462046FFF70AFF26F81400641CE4B298
:101B2000032CF3D3BDE8F081149D0020A402001023
:101B30002DE9FC47164688460746032805D2B8F12A
:101B4000000F02D0B6F5006F03D923A007F094F977
:101B50002FE0264850F82750284608F041F828B1D1
:101B600001F0C4FB0024DFF8889026E0294621A07C
:101B700007F082F91DE000BF4FF0FF30CDE9000013
:101B8000321B082A00D3082208EB04016846FEF73E
:101B9000BDFBDDE900232919002001F051FB58B1FC
:101BA00099F8000018B129191BA007F065F901F098
:101BB0003DFB002000F058B80834B442DCD301F0FB
:101BC00035FB99F8000020B1324639461BA007F0DA
:101BD00053F90120EEE7000044425F53617665202F
:101BE000706172206572726F720A000008DE000870
:101BF0000100001044425F536176653A20666C61D3
:101C000073685F6572617365206661696C20307806
:101C1000253038580A00000044425F536176653A27
:101C200020666C6173685F777269746520666169AC
:101C30006C203078253038580A00000044425F5349
:101C40006176653A20666C6173685F777269746566
:101C500020737563632069643D25642C206C656E78
:101C60003D25640A000000000CBCBDE8F0870000C0
:101C700010B5A2B004460B46009205A2802101A82F
:101C800007F00AF901A9204605F0A0FB22B010BD1B
:101C900025733D257300000010B592B004460B4635
:101CA000009205A2402101A807F0F6F801A92046FC
:101CB00005F08CFB12B010BD25733D2575000000AA
:101CC0002DE9F04F2E48B9B0016D09B92D490165D4
:101CD000DFF8B490DFF8B4A0002600BF3AF8160091
:101CE00009EBC624071941E0391B022328A220462C
:101CF00009F010F8E0B3851C791B022324A22846C2
:101D000009F008F8040000D13C46621B3D2128463A
:101D1000FEF769FB5FEA000828D0A8EB05002690D3
:101D2000A4EB0800A0F1010B2698402801D33F2026
:101D30002690BBF1800F01D34FF07F0B294627A8D7
:101D4000269AFEF725FB269827A900250D545A460A
:101D500008F1010104A8FEF71BFB04A927A801F85C
:101D60000B500AF09DFD0B4801F0A5FCBC42BBD313
:101D7000761CF6B2032EB1D339B000F00DB80000D6
:101D800040320010A8320010149D0020A402001060
:101D9000232300003027001030BCBDE8C08F0000B6
:101DA00008B5002000906A4605A1022009F0D3FC86
:101DB00007480099016307A007F05EF808BD00001E
:101DC0006961704C6F6164537461747573000000D5
:101DD000403200106961704C6F61645374617475B6
:101DE000732025640D0A0000014801F0A1B800002D
:101DF000F4280010014801F09BB80000AC28001046
:101E0000014801F095B800003C290010014801F09C
:101E10008FB800008429001030B590F8444004F0D9
:101E20001C050124AC40056C6C6004686360836829
:101E3000102B036803D099600068C26030BD9A60BF
:101E40000068C16030BD00009CB0DFF8A881DFF8F9
:101E5000A891DFF8A8A16A4D4FF4967B002600BF39
:101E600004F036FD04F04EFD0A2008F089FF98F8D2
:101E70000000444628B14FF4A041624800F04AFFF8
:101E8000267099F800004C4628B14FF4A0415E48F6
:101E900000F040FF26709AF80000544670B15B488D
:101EA0005BA10288AA860220FFF7F6FE5A485BA1D2
:101EB000026802202A62FFF7EFFE2670286B584561
:101EC00075D158480078002871D04E4C4FF4A0418D
:101ED000204600F01FFF642008F052FF4FF420520C
:101EE0004949204600F06AFF642008F049FF4EA0EF
:101EF00006F0C2FF00241AAF05EB44003A1952A1C4
:101F00002430FEF79FFA641C042CF5DB50A006F089
:101F1000B3FF684603F006FEA88E3A49B0F5007F8D
:101F20002A6A684600D0103A04F07EF9694616A87D
:101F300003F0D0FD4DA006F09FFF53A006F09CFFDC
:101F4000002456A0395D06F097FF641C042CF8DBD2
:101F500054A006F091FF54A006F08EFF002416AFA7
:101F60004EA0395D06F088FF641C042CF8DB4DA000
:101F700006F082FF04221AA916A8FEF73EFAC8B19D
:101F80004DA006F079FF40F291122E6354A1022079
:101F9000AA63FFF781FE55A102202A6BFFF77CFEA2
:101FA000002305224AF6BB2142200AF011FC07F06B
:101FB000E1FC55E751A006F05FFF0220AE63324618
:101FC00047A12863FFF768FE48A102202A6BFFF7AC
:101FD00063FE584608F0D4FEBFF34F8F51480168A6
:101FE000514A01F4E06111430160BFF34F8F00BF1C
:101FF000FDE70000380000101D0000101E0000105A
:10200000403200100040010800800208200000104B
:10201000737562636F6465002800001069617073F6
:10202000697A6500000000200D0A20436F70792056
:102030004941504461746142756666657220746FEF
:1020400020415050320000002532686878000000BE
:102050000D0A205265616420466C6173684D6435D9
:1020600020436F6D706C6574650000000D0A20439D
:10207000616C63756C617465204D643520436F6DD0
:10208000706C657465000000415050325F6D6435BE
:102090005F6279746573203A200000002530325861
:1020A000200000000A00000063616C5F6170703204
:1020B0005F6D6435203A20000D0A436F7079204926
:1020C00041504461746142756666657220746F2088
:1020D00041505032204661696C6564212121200005
:1020E00075626F6F746261636B0000006961704CB0
:1020F0006F61645374617475730000000D0A2043AE
:102100006F7079204941504461746142756666651B
:102110007220746F20415050322073756363657371
:10212000732000000CED00E00400FA05704770B564
:1021300000231C4611E011F82350055531F82350B7
:102140002E0A05196E7051F82360360CAE7051F8E6
:1021500023605B1C360EEE70241D9442EBD370BDE1
:1021600072B6FEE72749F0EE400ADFED281A91ED3E
:102170000A0A254AB4EEE00AF1EE10FA3BDA91EDD4
:10218000000AB4EEE00AF1EE10FA02D89FED200A40
:1021900070479FED202A002001EB800393ED000A99
:1021A00093ED011AF4EEC00AF1EE10FA26D8F4EE1F
:1021B000C10AF1EE10FA21DB02EB800070EEC10AD9
:1021C00090ED003AD0ED012A30EE411A124933EE7B
:1021D000623A60EE830A80EE810A30EE220AB5EEA2
:1021E000C00AF1EE10FA02D2B0EE420A704710EEC9
:1021F000100A8842FADDB0EE610A7047401C0A28D6
:10220000CADBF1E74884002094DB00080000C842E4
:102210000000B442000000000000C84210B511EEFA
:10222000900A2DED068BB0EE41AAB0EE408AF0EE9A
:10223000608AFEF7EDFB9FED150B41EC190B53EC9B
:10224000102B51EC180BFEF7F2FA41EC180B1AEEBA
:10225000100AFEF7DDFB53EC182BFEF7E8FA53ECFF
:10226000182BFEF7E4FA41EC100B53EC102B9FED0A
:10227000090B51EC100BFEF74FFB53EC192BFEF73B
:10228000C8FABDEC068B41EC100B10BD4AD8124DBC
:10229000FB21194000C84E676DC1AB4310B5044621
:1022A0002DED028B0846FEF7A6FB41EC180B1048FB
:1022B000005DFEF7A0FB41EC100B0E4800EBC400E4
:1022C00090ED001B51EC100B53EC112BFEF7AFFA05
:1022D00053EC182BFEF7ABFA9FED071B53EC112BB9
:1022E000FEF7A5FABDEC028B41EC100B10BD00000F
:1022F000AC02001018B50020000000000000303EC5
:102300002DE9F0418846642430B1012808D0022824
:102310000AD003280FD10BE00027012608250AE088
:1023200002270326042506E004270526022502E0ED
:1023300006270726012518212A2000F01BFA06E0AF
:1023400018212A2000F016FA641E24B28CB128420B
:10235000F6D074B139462A2000F00CFA0404314654
:102360002A2000F007FA2043C8F800000120BDE849
:10237000F0810020FBE7000070B5134D4FF480643E
:1023800000222146284601F057F9022007F018FBE9
:1023900000F032FA00226100284601F04DF90220D7
:1023A00007F00EFB01222146284601F045F90220E4
:1023B00007F006FB00222146284601F03DF9BDE862
:1023C0007040022007F0FCBA0004004870B5134DBD
:1023D0004FF4806400222146284601F02DF90220A6
:1023E00007F0EEFA00F008FA0122D102284601F0C7
:1023F00023F9022007F0E4FA01222146284601F0E1
:102400001BF9022007F0DCFA00222146284601F0E1
:1024100013F9BDE87040022007F0D2BA000400486A
:102420002DE9F04701221E4F8046D6020024314696
:10243000384601F001F900F0C9F9B1463E460025E1
:102440004FF480676006040E00223946304601F0E2
:10245000F3F8022007F0B4FA01223946304601F0C1
:10246000EBF8022007F0ACFA4946304601F0DFF8FD
:1024700008B1641CE4B26D1CEDB2082DE2D3002259
:102480003946304601F0D8F8B8F1000F04D0FFF714
:1024900073FF2046BDE8F087FFF798FFF9E70000DB
:1024A000000400482DE9F041054600F0A5F9174F5A
:1024B0004FF4806600223146384601F0BDF8002412
:1024C0004FF40068022007F07BFA280601D50122AC
:1024D00000E000224146384601F0AEF86806050EDD
:1024E00001223146384601F0A7F8022007F068FAC9
:1024F00000223146384601F09FF8022007F060FACA
:10250000641CE4B2082CDDD3BDE8F081000400486F
:1025100070B500F071F90122104DD4022146284611
:1025200001F08AF8012296023146284601F084F82B
:10253000022007F045FA00222146284601F07CF8E7
:10254000022007F03DFA00223146284601F074F8D7
:10255000BDE87040022007F033BA000000040048D4
:1025600070B500F049F9134D4FF480640022214604
:10257000284601F061F8022007F022FA66000022E6
:102580003146284601F058F8022007F019FA0122D6
:102590002146284601F050F8022007F011FA0122E6
:1025A0003146284601F048F8BDE87040022007F0A7
:1025B00007BA0000000400482DE9F041002400F0B3
:1025C00005F90122144DD6023146284601F034F8AF
:1025D000022007F0F5F9012297023946284601F05A
:1025E0002BF8022007F0ECF908E0641CE4B2FA2CA6
:1025F00004D9FFF7B5FF0120BDE8F0813146284638
:1026000001F015F80028F0D100223946284601F0E3
:1026100013F80020F0E70000000400482DE9F04125
:102620002F4C207810B12FA006F026FC7F212A2005
:1026300000F0A0F80546207818B1294631A006F030
:102640001BFCA5F5405044F620674FF47A665538D8
:102650000CD0207810B133A006F00EFC207810B119
:1026600037A006F009FC0120BDE8F08100F0A8F8D1
:102670003946002000F0B4F93146002000F0C8F9D6
:1026800001220221002000F0E1F8002000F07BF997
:10269000012000F040F9012000F02CF9002000F0AA
:1026A00061F904220021012000F08BF9002000F0E4
:1026B000B9F81521002000F03FF9002000F0BEF924
:1026C000207810B126A006F0D7FB207810B11CA00E
:1026D00006F0D2FB642008F053FB0020C4E70000A2
:1026E000010000200D0A3D3D3D2046444332323179
:1026F000345F6465766963654944203D3D3D0D0A5C
:1027000000000000464443323231345F646576692C
:102710006365494420203A20307825303278200DF6
:102720000A0000004644433232313420496E697455
:10273000204661696C65642121200D0A00000000BB
:102740003D3D3D3D3D3D3D3D3D3D3D3D3D3D3D3DB9
:102750003D3D3D3D3D3D3D3D3D3D3D3D0D0A000086
:102760004644433232313420496E6974204F4B2144
:102770000D0A000070B50D460446FFF7C9FE60065D
:10278000000EFFF78FFEFFF717FF2846FFF78AFEC0
:10279000FFF712FFFFF7BCFE012000EB4400C0B2C0
:1027A000FFF780FEFFF708FF0120FFF739FE040264
:1027B0000020FFF735FE0443FFF7D2FE204670BD30
:1027C0001C214FF400422A2000F049B900B585B021
:1027D00014216846FDF7B3FD4FF40060009000201F
:1027E0000190012002906946024800F035FE05B0D4
:1027F00000BD00000004004800B585B01421684603
:10280000FDF79DFD4FF40060009011200190012024
:1028100002906946024800F01FFE05B000BD0000AE
:102820000004004810B504461A212A20FFF7A2FF31
:102830004FF6FF7101EA8432C0F30D0002431A2102
:10284000BDE810402A2000F00AB9000070B5044627
:102850004FF6FF7000EA0136C2F30900064319483B
:10286000154601551848007810B118A006F004FB71
:102870002846FEF7C0F841EC100B53EC102B9FEDEF
:102880001A0B51EC100BFEF747F8194A02EBC40281
:10289000C2E9000164B1012C0DD0022C0ED0032C32
:1028A0000FD132461721BDE870402A2000F0D7B87A
:1028B00032461421F7E732461521F4E73246162155
:1028C000F1E770BDAC020010010000204672657196
:1028D00075656E63795F73656C65637420203A205B
:1028E0002564200D0A00000000000000D012834182
:1028F00018B5002010B504461A212A20FFF73AFF28
:1029000020F400720CB142F400721A21BDE81040AC
:102910002A2000F0A4B810B504461A212A20FFF797
:1029200029FF20F400620CB142F400621A21BDE8D4
:1029300010402A2000F093B84FF6FF7202EAC1223D
:1029400048B1012809D0022809D0032809D1212142
:102950002A2000F084B81E21FAE71F21F8E7202181
:10296000F6E7704710B504461A212A20FFF702FF48
:1029700020F040020CB142F040021A21BDE81040A4
:102980002A2000F06CB810B504461A212A20FFF75F
:10299000F1FE20F080020CB142F080021A212A20C0
:1029A00000F05DF819212A20FFF7E4FE20F0010273
:1029B0000CB142F001021921BDE810402A2000F0BC
:1029C0004EB838B1C00340EA4130104380B240F401
:1029D000027201E042F402721B212A2000F03FB88B
:1029E000FF2914D950B101280BD002280CD003289C
:1029F0000DD10A460B212A2000F031B80A460821E1
:102A0000F9E70A460921F6E70A460A21F3E7704783
:102A100050B101280BD002280CD003280DD10A4652
:102A200013212A2000F01BB80A461021F9E70A46B4
:102A30001121F6E70A461221F3E7704710B5044664
:102A40001A212A20FFF796FE20F400520CB142F41E
:102A500000521A21BDE810402A20AFF3008070B563
:102A600014460E460546FFF753FD6806000EFFF7B5
:102A700019FDFFF7A1FD3046FFF714FDFFF79CFDA0
:102A8000200AFFF70FFDFFF797FDE0B2FFF70AFD01
:102A9000FFF792FDBDE87040FFF762BD144A117F59
:102AA0001448012901D003290FD1036823F40073CE
:102AB0000360036843F400630360036823F4006366
:102AC0000360036843F400730360022901D0032903
:102AD0000BD1016841F480510160016821F48051FB
:102AE0000160016841F48061016000201077704747
:102AF000B000002000200240C107054803D0416912
:102B000041F004014161416941F480314161704704
:102B10000020024008494A69C0B222F47E7242EAAB
:102B2000C0004861486940F002004861486940F4CB
:102B3000803048617047000000200240054910B510
:102B40004C6944F001044C610260BFF36F8F436035
:102B500010BD000000200240094A10B5546940230E
:102B600044F480245461EFF3108272B610C910C08F
:102B70005B1E13F0FF03F9D182F3108810BD000033
:102B80000020024070B5054600F05CFD0646134C7F
:102B900008E0681C06D000F055FD801BA84201D358
:102BA000032070BD2069C003F3D420690C4908409C
:102BB0000CD00C494A6802434A60810F01D0A169D8
:102BC000A161810000D02061012070BD2069C00793
:102BD00001D001202061002070BD000000200240D3
:102BE000FAC30200B00000202DED048BBCB0684693
:102BF00004F0A2FD0BA804F09FFD16A804F09CFDB4
:102C000021A804F099FD2CA804F096FD3E4DB0EEED
:102C1000048AF6EE008AB1EE0C9AA5F18004E86908
:102C200090B100231A4637A908F0FCF860B99DED71
:102C3000370A684604F08AFD84ED0A0A94ED0A0A10
:102C4000FFF790FA84ED0B0AA86960B100231A46D9
:102C500038A908F0E7F830B99DED380A0BA804F060
:102C600075FD84ED100A6869B0B100231A4639A9D0
:102C700008F0D8F880B99DED390A16A804F066FD71
:102C800084ED040A94ED040A30EE480A20EE280A86
:102C900020EE090A84ED050A286AB0B100231A461D
:102CA0003AA908F0BFF880B99DED3A0A21A804F0CE
:102CB0004DFD84ED130A94ED130A30EE480A20EE20
:102CC000280A20EE090A84ED140A686AC0B10023BC
:102CD0001A463BA908F0A6F890B99DED3B0A2CA82E
:102CE00004F034FD84ED170A9FED081ADFED080AA1
:102CF00094ED170A03F0CEFC03F0E2FC84ED180A11
:102D0000052008F03DF88AE7800000209A994742A4
:102D10003333534070B586B00D00044629D01648B1
:102D2000844226D80026049600F0E0FA1348816910
:102D300041F0404181614CF2FA3101612046009638
:102D400000F01EF80190A4F10060C00A029004EBAC
:102D50008500401E0299A0F10060C1EBD020401C0C
:102D6000039004A9684600F0F1F9002801D000F0B2
:102D70005DFA06B070BD00000000040800200240AB
:102D80000449096804494FF001000968CA43120464
:102D9000120C704700000140E075FF1F064B10B594
:102DA000984207D8002303E010F8014BCC545B1C79
:102DB0009342F9D310BD0000000004082DE9F04152
:102DC00017460E46044600F091FA0A4884420DD296
:102DD000002509E0D6E900232146002000F030FA62
:102DE00020B908346D1C0836BD42F3D3BDE8F0416C
:102DF00000F01CBA0000040810B590F8251000225D
:102E0000022905D00421C16380F82420012010BDCF
:102E100001680B6823F00E030B6001680B6823F058
:102E200001030B6090F84410046C01F01C030121B5
:102E300001FA03F3636080F8251080F8242010461F
:102E400010BD10B590F825100024022903D00421EC
:102E5000C16301241AE001680A6822F00E020A60C8
:102E600001680A6822F001020A6090F84410036CBD
:102E700001F01C02012101FA02F25A6080F82510CB
:102E8000002180F82410816B01B18847204610BDD5
:102E900030B590B101680A6822F001020A60204C46
:102EA000036814211F4AA34209D21F4C1C44B4FBDF
:102EB000F1F18900C0E910210BE0012030BD184C70
:102EC00064421C44B4FBF1F189004164144908399F
:102ED00001640021196090F8443003F01C040123C0
:102EE000A340046C6360046C0F23944202D152F837
:102EF000A84F02E00A4AA032146890F8445005F046
:102F00001C05AB409C431460C16201634163816353
:102F1000C16380F8251080F82410002030BD000027
:102F20000804024000000240F8FFFDBFC06B70477C
:102F3000F0B4016C0C6801680D6890F8442002F050
:102F40001C06042202FA06F3234211D06B070FD5A8
:102F50000B689B0603D40B6823F004030B6090F806
:102F6000441001F01C018A40016C4A60016B1DE0B5
:102F7000022303FA06F727424FF0000C4FF001023C
:102F800018D0AF0716D50C68A40605D40C6824F039
:102F90000A040C6080F8252090F8441001F01C0110
:102FA0008B40016C4B6080F824C0C16A00291AD0A4
:102FB000F0BC08470823B340234214D02B0712D596
:102FC0000B6823F00E030B6090F84410036C01F0C3
:102FD0001C0102FA01F15960C26380F8252080F8D3
:102FE00024C0416BE2E7F0BC7047000070B568B1E7
:102FF0002B4C036814212B4AA34209D22A4C1C44AF
:10300000B4FBF1F18900C0E910210BE0012070BD93
:10301000234C64421C44B4FBF1F189004164204913
:1030200008390164022180F825101C6847F6F07108
:103030008C43D0E902152943D0E90456354329438E
:1030400085692943C5692943056A294321431960D4
:103050008168B1F5804F19D0036C0F21934202D1E2
:1030600052F8A83F02E00E4AA032136890F844409C
:1030700004F01C04A1408B43136090F84430416875
:1030800003F01C0399401368194311600021C163C8
:10309000012280F8252080F82410084670BD000029
:1030A0000804024000000240F8FFFDBF70B504466E
:1030B00090F82400002501280CD0012084F8240079
:1030C00094F825600020012E06D084F82400022503
:1030D000284670BD022070BD022684F82560E0639A
:1030E0002068066826F0010606602046FEF794FE7A
:1030F000206B00282068016802D041F00E0106E034
:1031000021F0040101602068016841F00A010160BA
:103110002068016841F001010160D9E70A4810B553
:103120004FF0FF318163C16300228263C263016497
:10313000026481628262C162C2620163026300F062
:1031400025FB002010BD0000001002402DE9F05FBB
:10315000054632488946017801290CD0012680466F
:1031600006704CF2503B5846FFF70CFD07004FF03D
:10317000000A03D04EE0022000F054B85146404609
:10318000C8F804A0264C226892050AD52168490592
:1031900005D5216821F480612160032109E00677CB
:1031A00008E02268520504D5216821F4806121607D
:1031B000022101772868012807D04FF0FF31C9F8B4
:1031C000001040F2FA3BAE681DE06868FFF794FC1F
:1031D0005846FFF7D7FC0746606920F0040060619D
:1031E00016E030466968FFF795FC4CF25030FFF767
:1031F000C9FC0700606920EA0B00606102D0C9F8D1
:10320000006005E0761CD5E902010844B042E8D828
:10321000FFF744FC88F800A03846ADE7B000002076
:103220000020024030BCBDE8C09F00000348416957
:1032300041F0004141610020704700000020024041
:103240002DE9FF5F254C0646904620789A460128D6
:103250000BD0012020704CF2503B5846FFF792FCF7
:1032600007004FF0000904D02AE0022004B000F06B
:1032700039B84846C4F80490194D2968490504D561
:10328000286820F4806028600220207726B1012E73
:1032900009D0022E07D00CE0424653460198FFF7B2
:1032A0004DFC012612E041460198FFF755FC022E25
:1032B0000AD05846FFF766FC4FEA0007FFF7EEFB1F
:1032C00084F800903846D1E74FF480265846FFF73F
:1032D00059FC07466869B0436861EFE7B000002019
:1032E0000020024030BCBDE8C09F0000064900201D
:1032F0004A69002A07DA054A8A60054A8A604969EC
:10330000002900DA012070470020024023016745B0
:10331000AB89EFCD2DE9F84F00230126DFF818C166
:103320000F2782E006FA03F414EA01027CD023F0AE
:1033300003056544AA46D5F808909D074FEA157E17
:1033400007FA0EF505EA090B0095B0F1904F05D08C
:103350003A4DA84205D14FF0010816E04FF00008A1
:1033600013E0374DA84202D14FF002080DE0354D71
:10337000A84202D14FF0030807E0334DA84202D122
:103380004FF0040801E04FF0070808FA0EF8D8459E
:1033900026D1DFF8B880D8F8009029EA0209C8F8E9
:1033A000009008F10408D8F8009029EA0209C8F84A
:1033B0000090DFF8988008F10C08D8F8009029EA0E
:1033C0000209C8F80090A8F10408D8F80050954305
:1033D000C8F80050009DDAF80820AA43CAF808206F
:1033E000D0F800804FEA4309032202FA09F248EAC2
:1033F0000208C0F80080DD0800EB8505AA46D5F874
:1034000020804FEA43794FEAD96907FA09F528EA9B
:103410000508CAF820808568954385604568A543FE
:103420004560C4689443C4605B1C31FA03F27FF4C6
:1034300079AF00F00DB80000000001400004004822
:1034400000080048000C004800100048000401403B
:1034500018BCBDE8E08F00002DE9F04FDFF8AC911B
:1034600000230325A9F1040B85B04FF0010C0F27B1
:1034700009F1040AABF1040EBFE000BF0CFA03F639
:10348000324075D00C7904F00304012C01D0022CD9
:103490001BD1846800945C0005FA04F80494009C35
:1034A00024EA08040094D1F80C80049C08FA04F87B
:1034B000009C48EA0408C0F808804468B4430E79C8
:1034C000C6F300169E40264346600C79E443A407E9
:1034D0000AD0C4684FEA430805FA08F6B4438E6878
:1034E00006FA08F62643C6600C7904F00304022CA1
:1034F00010D1DC0800EB84040294246A5E074FEAD2
:10350000D66807FA08F6B4430E6906FA08F62643A9
:10351000029C266204684FEA430805FA08F6B443A1
:103520000E7906F0030606FA08F6264306604C6894
:1035300014F4403F60D0364C266E46F001062666F5
:10354000246E23F0030604F001040094314C34444B
:103550000294A4689E074FEA167807FA08F6B44367
:10356000B0F1904F05D02C4EB04204D1012612E0AC
:1035700042E000260FE0294EB04201D102260AE0C7
:10358000274EB04201D1032605E0264EB04201D1BC
:10359000042600E0072606FA08F62643029CA660E9
:1035A000D9F800604C46D1F8048096435FEAC828F9
:1035B00000D516432660DAF800405646D1F804805C
:1035C00094435FEA882800D514433460DBF8004058
:1035D0005E46D1F8048094435FEA883800D51443EE
:1035E0003460DEF800407646D1F8048094435FEA08
:1035F000C83800D5144334605B1C0A6832FA03F4FF
:103600007FF43CAF05B000F00FB8000008040140A3
:10361000001002400000014000040048000800487B
:10362000000C00480010004830BCBDE8C08F0069A5
:10363000084000D0012070470AB181617047816263
:103640007047000001488068704700000C000010BF
:1036500070B5040011D021684CF6CC400860216898
:1036600045F255500860D4E9000141602168A06826
:103670008860FFF7E7FF05460DE0012070BD00BF41
:10368000FFF7E0FF401B312805D92068C0684007DC
:1036900001D0032070BD2068C0684007F0D12068C9
:1036A0000269E1688A4201D0016102E04AF6AA217A
:1036B0000160002070BD00684AF6AA210160002068
:1036C00070470000024881680278114481607047A9
:1036D0000C00001010B50024032000F0B1F80F20FA
:1036E00000F008F808B1012401E000F051F820468C
:1036F00010BD000030B505461F4887B0816D41F010
:1037000010018165806D06A900F01000009001A8ED
:1037100000F054FB0498B0B100F070FB4000174972
:10372000174AB0FBF1F11748491E0260416040F2B0
:10373000E7320021C0E903218160816101F022FAB2
:10374000040003D015E000F059FBE8E70D4801F054
:1037500087FA04000DD1362000F045F8102D07D26D
:1037600000222946362000F04BF80748056000E0AB
:10377000012407B0204630BD0010024040420F0037
:1037800000100040DC2A00101000001070470000FC
:103790000B4882B0016E41F001010166016E01F03B
:1037A00001010091816D41F080518165806D0022A1
:1037B00000F0805000900F21901E02B000F020B861
:1037C0000010024000280DDB00F01F020121914093
:1037D0004009800000F1E020C0F88011BFF34F8F56
:1037E000BFF36F8F7047002809DB00F01F02012133
:1037F00091404009800000F1E020C0F800117047BE
:10380000F0B40E4B1B680C46C3F30223C3F107054B
:10381000042D00D90425191D072901D2002300E039
:10382000DB1E012606FA05F1491E214099409E4003
:10383000761E16403143F0BC05F068BB0CED00E08D
:10384000064900F0070208684FF6FF03184040EAF7
:103850000220034A10430860704700000CED00E0AE
:103860000000FA051649B0F5007F0868C0F3412052
:1038700009D0022805D0086820F4C06040F48060B8
:103880000860002070470128FBD0086820F4C06061
:1038900040F4007008600B483222006850430A4A26
:1038A000B0FBF2F0401C00E0401E4A69520501D511
:1038B0000028F9D148694005E3D50320704700008E
:1038C00000700040D000002040420F000248006815
:1038D00000F4C06070470000007000402DE9F84F10
:1038E000044600270088A84D3E46000515D5606CAB
:1038F00060B1B0F5000F04D0B0F5400F2BD0012718
:103900000AE0E86840F48030E86024E00021201DEF
:1039100003F0D8F807001ED03E46206880033AD551
:10392000A86D4FF00008C00009D4A86D40F0805089
:10393000A865A86D4FF0010800F080500090DFF8F6
:103940004CA2DAF8001041F48071CAF80010FFF7B9
:1039500079FE814610E0D5F88800616C20F44000C3
:103960000843C5F88800D8E7FFF76CFEA0EB090014
:10397000022801D9032705E0DAF80000C005F3D5D5
:10398000002F7DD04FEA0706B8F1000F03D0A86DD5
:1039900020F08050A8652078C00707D0D5F88800AF
:1039A000216A20F003000843C5F8880020788007CA
:1039B00007D5D5F88800616A20F00C000843C5F8E7
:1039C00088002078400707D5D5F88800A16A20F044
:1039D00030000843C5F888002078800607D5D5F860
:1039E0008800E16A20F440600843C5F88800208818
:1039F000800507D5D5F88800E16B20F44020084306
:103A0000C5F888002088400507D5D5F88800216CC6
:103A100020F440100843C5F888002078400607D5F8
:103A2000D5F88800216B20F440500843C5F8880081
:103A30002078000607D5D5F88800616B20F4404057
:103A40000843C5F888002088C00507D5D5F8880048
:103A5000A16B20F440300843C5F8880020684FF07F
:103A6000006700034FF0806850D5D5F88800A16C3E
:103A700020F040600843C5F88800A06CB84200E020
:103A800005E03BD1E86840F48010E8603EE0D5F8FE
:103A9000900010F4407014D0A16D814211D0D5F87F
:103AA0009000D5F8901020F4407041F48031C5F8B2
:103AB0009010D5F8901021F48031C5F89010C5F819
:103AC0009000C00711D0FFF7BDFD074641F28839CD
:103AD00007E000BFFFF7B6FDC11B494501D903262A
:103AE00052E7D5F890008007F4D5D5F89000A16D85
:103AF00020F440700843C5F8900045E7404505D1E3
:103B00000121201D02F0DEFF00B1064620684003BF
:103B100017D5D5F88800E16C20F040600843C5F85F
:103B20008800E06CB84204D1E86840F48010E86096
:103B300007E0404505D10121201D02F0C3FF00B17F
:103B400006462088400411D5D5F88800216D20F064
:103B500040500843C5F88800206DB0F1805F05D162
:103B60000221201D02F0AEFF00B1064620880004AD
:103B700006D555F8880F616D20F080400843286015
:103B8000304600F005B80000001002400070004010
:103B900018BCBDE8E08F00002DE9F0470F46050096
:103BA0006BD0494E306800F00700B84209D2306847
:103BB00020F0070038433060306800F00700B8425A
:103BC0005BD12878414C80070AD5A868A16801F02C
:103BD000F001884204D9A16821F0F0010143A160FD
:103BE0002878C0072CD06868032811D0022812D08A
:103BF000216898B1490500293FDAA16821F0030145
:103C00000143A160FFF71EFD804641F2883910E0B4
:103C100021688901EFE721688903ECE78907EAE772
:103C2000FFF710FDA0EB0801494502D90320BDE8CC
:103C3000F087A068696800F00C00B0EB810FEFD14D
:103C4000287880070AD5A868A16801F0F0018842A9
:103C500004D2A16821F0F0010143A160306800F0B6
:103C60000700B8420BD9306820F0070038433060B5
:103C7000306800F00700B84201D00120D7E728786B
:103C8000400705D5A068E96820F4E0600843A0601B
:103C90002878000706D5A068296920F4605040EA1A
:103CA000C100A06000F0CEF8A168094AC1F3031179
:103CB000515C01F01F01C8400649086006480068D1
:103CC000BDE8F047FFF716BD00200240001002409B
:103CD00020DB0008D0000020100000102DE9F0418A
:103CE000314C206840F001002060FFF7ABFC054636
:103CF00005E000BFFFF7A6FC401B022833D8206870
:103D00008007F7D5206820F0F00040F060002060C8
:103D10000025A56026492548086026480068FFF769
:103D2000E9FC10B10120BDE8F081FFF78BFC0646ED
:103D300041F2883705E000BFFFF784FC801BB842E2
:103D400011D8A06810F00C0FF6D120681A4908406D
:103D50002060FFF777FC064607E000BFFFF772FC24
:103D6000801B022801D90320DDE7206810F0206FB6
:103D7000F4D1E560E06840F48050E060256120699E
:103D800040F480502061206820F480202060A561EC
:103D90004FF0FF302062D4F8940040F40000C4F8E3
:103DA00094000020BFE70000001002400024F4004F
:103DB000D000002010000010FFF4FEFA0F22026075
:103DC0000C4A936803F003034360936803F0F00325
:103DD0008360936803F4E063C36092684FF4E06328
:103DE00003EAD20202610448006800F0070008609C
:103DF00070470000001002400020024005480649BC
:103E000000688968054AC1F30221515C01F01F0175
:103E1000C8407047D00000200010024060DB00085E
:103E20000548064900688968054AC1F3C221515C0A
:103E300001F01F01C8407047D00000200010024070
:103E400060DB000870B52549002318468A68CC68F5
:103E500012F00C0204F00306214C4FEA640509D06D
:103E60000C2A05D0042A32D0082A00D1284670BD79
:103E7000012E10D10B681B0704D4D1F89430C3F382
:103E8000032302E00B68C3F30313164E56F82330E6
:103E9000DAB10C2AEBD1C86800F00300022818D070
:103EA000032818D01846CA68CB68C2F30212C3F3BD
:103EB00006234343521CB3FBF2F2C868C0F34160CF
:103EC000401C4000B2FBF0F070BD184670BD2046AB
:103ED00070BD2046E7E72846E5E7000000100240F5
:103EE0000024F40030DB00082DE9F84304006FD013
:103EF000FA4DA86800F00C06E86800F00307207887
:103F0000C00664D576B10C2E01D1012F0AD0A0696C
:103F1000002828687AD040F001002860FFF792FB63
:103F200080465DE02868800702D5A0690028DED0C1
:103F3000216A2868000703D5286800F0F00004E033
:103F4000D5F89400F02202EA1010814216D90846F2
:103F500002F04EFE00283BD1286840F0080028609F
:103F60002868216A20F0F000084328606868E16949
:103F700020F47F4040EA0120686016E0286840F0A5
:103F8000080028602868216A20F0F00008432860B3
:103F90006868E16920F47F4040EA0120686026B942
:103FA000206A02F025FE0028D5D1FFF74BFFA96853
:103FB000CB4AC1F30311515C01F01F01C840C9494C
:103FC0000860C9480068FFF795FB00287ED12EE005
:103FD000CAE000BFFFF736FBA0EB0800022876D846
:103FE00028688007F6D5286840F00800286028680F
:103FF000216A20F0F000084328606868E16920F435
:104000007F4040EA0120686011E0FFE720F00100F6
:104010002860FFF717FB804606E000BFFFF712FBA2
:10402000A0EB08000228DAD828688007F6D42078A8
:10403000C00740D0082E18D00C2E01D1032F14D069
:104040006068B0F5803F17D0B0F5A02F286817D072
:1040500020F480302860286820F480202860606880
:10406000E0B1FFF7EFFA804614E02868800322D51C
:104070006068002878D01EE0286840F48030EDE7C2
:1040800040F480202860F7E7FFF7DCFAA0EB080097
:104090006428A4D828688003F6D50CE0FFF7D2FA8C
:1040A000804605E0FFF7CEFAA0EB0800642896D81A
:1040B00028688003F6D4207880073BD5042E11D0E1
:1040C0000C2E01D1022F0DD0E06801E0AAE1FFE043
:1040D000002828681ED040F480702860FFF7B2FAEC
:1040E00007460CE0286840050CD5E0680028C1D0E0
:1040F00008E000BFFFF7A6FAC01B022893D8286883
:104100004005F7D56868217C20F0F85040EA01604E
:1041100068600FE020F480702860FFF793FA07468C
:1041200005E000BFFFF78EFAC01B0228B1D828684F
:104130004005F7D42078000729D560690028D5F814
:10414000940012D040F00100C5F89400FFF77AFA0D
:10415000074604E0FFF776FAC01B022899D8D5F885
:1041600094008007F6D512E02BE120F00100C5F89D
:104170009400FFF767FA074605E000BFFFF762FA11
:10418000C01B022885D8D5F894008007F6D4207883
:10419000400766D5A86D0027C00008D4A86D40F080
:1041A0008050A865A86D012700F0805000904F480E
:1041B0000168C90512D40168814641F4807101602B
:1041C000FFF740FA804605E0FFF73CFAA0EB080055
:1041D00002287DD8D9F80000C005F5D5A0680128CF
:1041E00016D00528D5F8900017D020F00100C5F8AA
:1041F0009000D5F8900020F0040000BFC5F89000B2
:10420000A06841F28839C0B1FFF71CFA80460FE080
:10421000D5F8900040F00100F0E740F00400C5F848
:104220009000F5E7FFF70EFAA0EB080149454FD8DB
:10423000D5F890008007F5D50EE0FFF703FA804629
:1042400006E000BFFFF7FEF9A0EB080149453FD8A3
:10425000D5F890008007F5D41FB1A86D20F08050EC
:10426000A8652078800628D5606A0028D5F89800CF
:1042700012D040F00100C5F89800FFF7E3F90746B7
:1042800005E000BFFFF7DEF9C01B022820D8D5F8F3
:1042900098008007F6D510E020F00100C5F89800DE
:1042A000FFF7D0F9074604E0FFF7CCF9C01B02285E
:1042B0000ED8D5F898008007F6D4A06AF0B302288B
:1042C00016D00C2E7DD0286820F08070286000E089
:1042D000A7E0FFF7B7F90446A6E00000001002408F
:1042E00020DB0008D000002010000010007000400B
:1042F000E868E26A00F00301914228D1216B00F0E6
:10430000700209011039914221D1626B00F4FE4123
:10431000B1EB022F1BD194F8382000F07841B1EBBB
:10432000C26F14D1A18F00F4C00249084905A1F55C
:10433000001191420BD194F8401000E06AE0490866
:10434000490600F0C060A1F1007181424BD00C2EF3
:1043500073D02868400170D4286820F080702860ED
:10436000FFF770F9064604E0FFF76CF9801B02289E
:1043700057D828688001F7D4F4E90B016FF00F02D9
:1043800002EB01110843218A5204490802EB415112
:10439000A26841EA02210843217D4FF07E4249088C
:1043A00002EB41610843217B40EAC160E968244A8D
:1043B00011400843E860286840F080702860E86891
:1043C00000E03AE040F08070E860FFF73BF9044617
:1043D00005E000BFFFF736F9001B022821D8286846
:1043E0008001F7D527E02868800124D4286840F0B0
:1043F00080702860E86840F08070E860FFF722F97C
:10440000044604E0FFF71EF9001B022809D82868BB
:104410008001F7D50FE000BFFFF714F9001B022859
:1044200002D90320BDE8F88328688001F4D4E86845
:1044300004490840E8600020F4E70120F2E70000AA
:104440008C809D01FCFFEEFE70B5040009D0606A0F
:10445000002540B125616561A56294F85D0040B119
:104460000CE0012070BD6068B0F5827FF4D0E5619A
:10447000F2E784F85C50204600F056F8022084F8F9
:104480005D002068016821F040010160E1684FF49F
:10449000E062914201D9002001E04FF48050B1F573
:1044A000706F02D0914200D0A562A188228901F4E8
:1044B000827102F404421143227C02F00202114391
:1044C000227D02F001021143228B02F4007211439B
:1044D000227F02F03802114394F8202002F080027B
:1044E0001143228D02F40052114322681160A16928
:1044F000042202EA114194F8242000F4805002F0D2
:104500001002114394F8342002F008021143A289EA
:1045100002F4706211430143206841602566012066
:1045200084F85D00002070BD10B586B004461421EB
:104530006846FBF704FF1349206888421FD11248E0
:10454000016E41F480510166016E01F480510591C4
:10455000C16C41F00101C164C06C694600F001000A
:104560000590E0200090022001900020029003209E
:104570000390052004904FF09040FEF76DFF06B0C9
:1045800010BD000000300140001002402DE9F84F3E
:10459000044640680025984616460F464FF0040B27
:1045A000B0F5827F01D1A06888B194F85C00012841
:1045B00018D0012084F85C00FFF744F8814694F895
:1045C0005D004FF0000A01280ED0022599E084F822
:1045D0005DB013460A462046CDF8008000F064F92D
:1045E00000F098B80220FBE7002F77D0002E75D09E
:1045F00084F85DB0C4F860A02764A4F84460A4F80F
:104600004660C4F838A0A4F83CA0A4F83EA0C4F8C2
:104610004CA0C4F850A0E0684FF4E06188422068E4
:10462000426802D922F4805201E042F48052426092
:10463000A068B0F5004F09D12068026822F040025E
:1046400002602068026822F48042026020680268EA
:10465000520603D4026842F040020260E0688842D9
:104660001DD93FE020688168C9070BD0017B206C11
:104670000170206C401C2064B4F84600401EA4F871
:1046800046000CE0FEF7DEFFA0EB0901414503D335
:10469000B8F1FF3F03D03BE0B8F1000F38D0B4F8D9
:1046A00046000028DED121E020688168C9070BD0D0
:1046B000C068216C0880206C801C2064B4F846001F
:1046C000401EA4F846000DE0FEF7BCFFA0EB090178
:1046D000414504D3B8F1FF3F04D019E010E0B8F130
:1046E000000F15D0B4F846000028DDD14A464146F7
:1046F000204602F03DFD08B120202066206E00B16A
:104700000125012084F85D0084F85CA0284667E755
:104710000325F6E718BCBDE8E08F2DE9F84F044605
:1047200090F85C0000271D461646894601280DD0EA
:104730004FF0010B84F85CB0FEF784FF804694F8DC
:104740005D00BA46012804D00227A4E0022000F050
:10475000A8B8B9F1000F74D0002E72D0032084F8ED
:104760005D00C4F860A0C4F83890A687E687C4F856
:1047700040A0A4F844A0A4F846A0C4F850A0C4F8EF
:104780004CA0A068B0F5004F09D12068016821F065
:10479000400101602068016841F4804101602068A7
:1047A0000168490603D4016841F040010160E068F6
:1047B000B0F5E06F606823D908B1012E1CD1A06B61
:1047C00021680088C86006E020688168890709D5EB
:1047D000A16B0988C160A06B801CA063E08F401EA4
:1047E000E08709E0FEF72EFFA0EB0800A84202D305
:1047F000681C01D046E0ADB3E08F0028E4D136E07C
:1048000008B1012E30D1E08F0128A06B03D92168B7
:104810000088C8600FE021680078087314E0E08722
:1048200022E020688168890714D5E18F0129A16BF6
:1048300008D90988C160A06B801CA063E08F801E2E
:10484000EDE727E009780173A06B401CA063E08FBF
:10485000401EE4E7FEF7F6FEA0EB0800A84202D3F4
:10486000681C01D00EE06DB1E08F0028D9D142461E
:104870002946204602F0B6FC08B120202066A06838
:1048800010B105E0032706E02068C1688068009049
:10489000206E00B1012784F85DB084F85CA0384632
:1048A00055E718BCBDE8E08F2DE9F05F044690F8AD
:1048B0005C0000270A9E1D4692468B464FF0010978
:1048C00001280ED0012084F85C00FEF7BBFE804674
:1048D00094F85D00616801280CD0B1F5827F07D1A2
:1048E00002E0022000F011B9A16809B9042801D042
:1048F000022700E1BBF1000F24D0BAF1000F21D054
:1049000005B394F85D00042802D0052084F85D000A
:1049100000202066C4F840A0A4F84650A4F84450F3
:10492000C4F838B0E587A587E0642065E0684FF4F7
:10493000E061884201D8012D06D92068426822F43E
:10494000805205E00127D6E02068426842F4805298
:10495000426020680268520603D4026842F04002B6
:104960000260E0688842606845D908B1012D3AD1FB
:10497000A06B21680088C860A06B801CA063E08FDA
:10498000401EE0872FE02068816889070FD5E18FFE
:1049900069B1B9F1010F0AD1A16B0988C160A06B9F
:1049A000801CA063E08F401EE0874FF00009206864
:1049B0008168C9070FD0B4F8461061B1C068216C96
:1049C0000880206C801C2064B4F84600401EA4F8C7
:1049D00046004FF00109FEF735FEA0EB0800B0429B
:1049E00001D3701C75D1E08F0028CCD1B4F84600FB
:1049F0000028C8D176E008B1012D6CD1E08F0128E4
:104A0000A06B08D921680088C860A06B801CA063D7
:104A1000E08F801E07E0216800780873A06B401CBF
:104A2000A063E08F401EE08755E020688168890719
:104A30001AD5E18FC1B1B9F1010F15D1E18F01296B
:104A4000A16B07D90988C160A06B801CA063E08FAF
:104A5000801E06E009780173A06B401CA063E08F04
:104A6000401EE0874FF0000920688168C90728D000
:104A7000B4F8461029B3B4F84610012914D9C06817
:104A8000216C0880206C801C2064B4F84600801ED5
:104A9000A4F84600B4F84600012810D82068416800
:104AA00041F4805141600AE0007B216C0870206C69
:104AB000401C2064B4F84600401EA4F846004FF0A5
:104AC0000109FEF7BFFDA0EB0800B04202D3701C45
:104AD00001D018E0BEB1E08F0028A6D1B4F846009E
:104AE0000028A2D142463146204602F07BFB10B19D
:104AF000012720202066012084F85D00002084F832
:104B00005C003846EEE60327F5E730BCBDE8C09F01
:104B10007047704770470000F0B590F83C20012ABC
:104B200029D0012480F83C40022280F83D2003680F
:104B30005A689D68114EB34203D122F470074A6847
:104B40003A4322F070070A683A435A600268B24258
:104B500005D0B2F1804F02D0094B9A4204D1896846
:104B600025F080031943916080F83D40002180F8D2
:104B70003C100846F0BD0220F0BD0000002C0140B2
:104B80000040014010B5040003D094F83D0010B17E
:104B900007E0012010BD002084F83C00204600F012
:104BA00023F8022084F83D00211D206803F0EEFA6E
:104BB000012084F8480084F83E0084F83F0084F81F
:104BC000400084F8410084F8420084F8430084F8EF
:104BD000440084F8450084F8460084F8470084F8CF
:104BE0003D00002010BD000008B50068064988425D
:104BF00008D10648016E41F480310166006E00F470
:104C00008030009008BD00000040014000100240CC
:104C100090F83D10012901D001207047022180F851
:104C20003D1000680B49884205D0B0F1804F02D09A
:104C30000949884207D18168084A1140062906D0EF
:104C4000B1F5803F03D0016841F00101016000200F
:104C500070470000002C01400040014007000100A7
:104C600090F83D10012901D001207047022180F801
:104C70003D100168CA6842F00102CA6000680B4931
:104C8000884205D0B0F1804F02D00949884207D14F
:104C90008168084A1140062906D0B1F5803F03D04B
:104CA000016841F00101016000207047002C0140C3
:104CB000004001400700010070B5044690F83C0038
:104CC0000025012817D0012684F83C60022084F8D2
:104CD0003D00226890682F4B184020F47F40906080
:104CE0000868502838D00DDC20284FD005DC90B360
:104CF000102811D14AE0022070BD302846D040284B
:104D00000AD13BE060282FD070280DD0B0F5805F2D
:104D100003D0B0F5005F12D0012584F83D6000207B
:104D200084F83C00284670BDCB68D1E90121206899
:104D300003F062FA2068816841F0770109E0CB68EE
:104D4000D1E90121206803F057FA2068816841F415
:104D500080418160E1E719E0CA684968206803F092
:104D60005DFA5021206806E0CA684968206803F0AF
:104D700066FA6021206803F049FACEE7CA684968FC
:104D8000206803F04BFA40212068F4E722680146CE
:104D90001046F0E788FFFEFF704770B504460068D4
:104DA00001694FF00005C943890715D4C168C9439B
:104DB000890711D4E91E01610120207720688069EC
:104DC0008007204602D0FFF7E7FF04E000F0A7F8D5
:104DD000204600F0A5F8257720680169C9434907F6
:104DE00017D4C168C943490713D46FF004010161A6
:104DF000022020772068806910F4407F204602D08E
:104E0000FFF7CAFF04E000F08AF8204600F088F8B7
:104E1000257720680169C943090716D4C168C943C9
:104E2000090712D46FF0080101610420207720687F
:104E3000C0698007204602D0FFF7AEFF04E000F013
:104E40006EF8204600F06CF8257720680169C943A8
:104E5000C90617D4C168C943C90613D46FF010013D
:104E60000161082020772068C06910F4407F204647
:104E700002D0FFF791FF04E000F051F8204600F067
:104E80004FF8257720680169C943C90708D1C1686F
:104E9000C943C90704D1891E0161204600F042F8C8
:104EA00020680169C943090609D4C168C9430906D4
:104EB00005D46FF0800101612046FFF72AFE2068CB
:104EC0000169C943C90509D4C168C943090605D4A4
:104ED0006FF4807101612046FFF71AFE20680169B6
:104EE000C943490609D4C168C943490605D46FF0CE
:104EF00040010161204600F01FF820680169C943A4
:104F000089060BD4C168C943890607D46FF0200114
:104F100001612046BDE87040FFF7FCBD70BD7047E1
:104F20007047000000680349884201D1FEF7CABB00
:104F3000704700000010004070477047704770B520
:104F40000446806FE66F216889684FF010050906F6
:104F500018D5212816D12068083050E8001F21F00C
:104F6000800140E80012002AF5D1E06E38B1FDF76B
:104F700043FF20B1E06EFDF7D9FF202821D0204665
:104F800003F0FDFC20688068400618D5222E16D15B
:104F90002068083050E8001F21F0400140E800126E
:104FA000002AF5D1206F38B1FDF726FF20B1206F20
:104FB000FDF7BCFF202804D0204603F0BBFC0020F6
:104FC00070BDC4F88050032070BD70B5040019D0C6
:104FD0002420A0672068016821F001010160206899
:104FE000002505602068456020688560204600F047
:104FF0008BF9C4F88050A567E56744F8605F00202E
:10500000257570BD012070BD704700002DE9F0418D
:1050100002680446D0691168936840F60F0528427B
:105020004FF0000505D186067ED58E067CD5616ED3
:105030001BE1994F03F001060F40374374D0C707B7
:1050400009D0CF0507D501271762D4F8802042F098
:105050000102C4F8802082070AD5DA0708D0276841
:1050600002223A62D4F8802042F00402C4F8802080
:1050700042070AD5DA0708D0236804221A62D4F856
:10508000802042F00202C4F8802002070CD501F013
:105090002002324308D0236808221A62D4F8802004
:1050A00042F00802C4F8802002050BD54A0109D558
:1050B00023684FF400621A62D4F8802042F0200284
:1050C000C4F88020D4F88020002A35D0800605D589
:1050D000880603D5616E09B120468847D4F8800060
:1050E00021688968490602D410F0280F26D020468E
:1050F00003F020FC2068806840061AD5206808303C
:1051000050E8001F21F0400140E80012002AF5D1CC
:10511000206F70B161498163206FFDF792FE002816
:105120000AD0206F816B01E00EE02046BDE8F0411F
:1051300008472046FFF768FFBDE8F0812046FFF7EB
:1051400063FFC4F88050F7E7276E2026012F7BD13C
:10515000C70679D5CF0677D5102010622068806801
:10516000400641D5216F086840680004000CE3D078
:10517000B4F858208242DFD9A4F85A0008680068C1
:1051800080062AD4206850E8001F21F4807140E88E
:105190000012002AF6D12068083050E8001F21F0E4
:1051A000010140E80012002AF5D12068083050E8DB
:1051B000001F21F0400140E80012002AF5D1E66707
:1051C0002566216851E8000F20F0100041E8000238
:1051D000002AF6D1206FFDF70FFEB4F85800B4F89E
:1051E0005A10401A81B22AE0B4F85800B4F85A10A4
:1051F000401A81B2B4F85A0000289DD000299BD0F3
:10520000226852E8000F20F4907042E80003002B5F
:10521000F6D12068083050E8002F22F0010240E863
:105220000023002BF5D1E66725666566226852E803
:10523000000F20F0100042E80003002BF6D12046BA
:10524000FFF77BFE78E7FFE7C70209D55B0207D5CA
:105250004FF4801010622046BDE8F041FFF76EBEAB
:10526000020606D50A0604D5A16E00297FF45DAFBB
:1052700062E74006E6D54806E4D52046026852E8D3
:10528000001F21F0400142E80013002BF6D1866791
:10529000856600F027FA4FE720010004ED8700083B
:1052A00010B5040002D0A06F10B107E0012010BDBE
:1052B000002084F87400204600F05EF82420A067E7
:1052C0002068016821F001010160204603F064FBC1
:1052D0000128ECD0606A10B1204603F0F5F920688F
:1052E000416821F4904141602068816821F02A01E1
:1052F00081602068016841F0010101602046BDE83D
:10530000104003F045BA000010B50446174B016881
:1053100017484FF09042994210D1016E21F480411C
:1053200001664FF4C0611046FDF7F4FF206FFDF7F2
:10533000AFFDE06EFDF7ACFD252011E00D4B99426D
:1053400012D1816D21F4003181650C211046FDF7E9
:10535000E1FF206FFDF79CFDE06EFDF799FD262033
:10536000BDE81040FEF72EBA10BD00000038014025
:1053700000100240004400402DE9F04F9DB004466B
:10538000142117A8FAF7DBFF5C216846FAF7D7FF6C
:1053900061492068614F002502264FF003094FF054
:1053A000070A4FF0800B884256D1012000900895E3
:1053B0006846FEF793FA08B1FCF7D2FE386E40F467
:1053C00080403866386E00F480401C90F86C40F0E5
:1053D0000100F864F86C19AA00F001001C904FF469
:1053E000C060CDE9170682E8200617A94FF090406B
:1053F000FEF732F84B4F4A48D8463860C7E9016596
:10540000C7E9035B7D61BD61FD6138463D62FDF723
:10541000EDFD08B1FCF7A4FE2767BC62414F404890
:1054200048371438E7E802061020A7E821013D4874
:1054300047F814594830BD61FD613D62FDF7D6FD66
:1054400008B1FCF78DFEE766002205212520BC622D
:10545000FEF7D6F9252059E03349884258D16846ED
:1054600000960995FEF73AFA08B1FCF779FEB86D97
:1054700040F40030B865B86D00F400301C90F86C52
:1054800040F00100F864F86C19AA00F001001C90CB
:105490000C20CDE9170682E82006B046374617A94A
:1054A0004FF09040FDF7D8FF1E4E1D489036143047
:1054B0003060C6E90175C6E9035B7561B561F561E8
:1054C0005F4630463562FDF791FD08B1FCF748FEB6
:1054D0002667B462134E1248D8362830E6E8020830
:1054E0001020A1C60F4846F81459D830B561F561AF
:1054F0003562FDF77BFD08B1FCF732FEE66600225F
:1055000005212620B462FEF77BF92620FEF76BF911
:105510001DB000F00BB80000003801400010024040
:1055200058000240AC2800100044004030BCBDE8E8
:10553000C08F000030B4C36F202B20D1E1B1DAB1AD
:1055400090F87430012B1AD0012380F874300023B6
:1055500003660C4C0368A3420BD05B681B0208D5A2
:10556000046854E8003F43F0806344E80035002DB0
:10557000F6D130BC03F010BB012030BC70470220D4
:10558000FBE7000000800040704770472DE9F843BA
:105590000446806F1F4616460D4620284FD1CDB1D8
:1055A000C6B194F87400012849D0012084F8740031
:1055B0004FF00008C4F880802120A067FEF742F871
:1055C000A4F850608146A4F85260A068B0F5805FEE
:1055D00003D004E00120BDE8F883206928B12E46FD
:1055E0005FF0000584F8748010E00026FAE780215F
:1055F000204603F023FBB8B9C6B116F8010B2168A9
:105600000885B4F85200401EA4F85200B4F85200C5
:105610004B464FF0000200970028E8D14FF04001C0
:10562000204603F00BFB30B10320D4E735F8020B22
:10563000C0F30800E3E72020A0670020CBE70220AA
:10564000C9E7000070B50446806F202841D169B3D6
:1056500062B394F8740001283BD0012084F87400F0
:10566000E164A4F85020A4F852200025C4F880502A
:105670002120A067E06ED8B11749C162E16E1748DA
:1056800013460863E16E16484863E06E856326683A
:10569000E16C06F12802E06EFDF708FD40B1102034
:1056A000C4F8800004F8745F20206060012070BDA1
:1056B00021684020086284F874502068083050E85F
:1056C000001F41F0800140E80012002AF5D10020BF
:1056D00070BD022070BD0000E98800082B89000819
:1056E0000188000800680549884205D10022C114DC
:1056F0004FF09040FDF7A0BF704700000038014018
:105700007047FEE700261A4FDFF8688035464FF4F1
:105710008039B2461848FDF7CEFF387920B102280B
:1057200004D0012804D004E0032402E0052400E0B2
:105730000924B44203D02646304603F02FFB0F491C
:105740000F4800F087F90E490C4800F083F9642DEA
:1057500009D9D8F818000025401CC8F81800484599
:1057600001DBC8F818A002206D1C05F009FBD1E789
:1057700000000020403200103027001050000010C0
:105780003C0000102DE9F0410568064644681548C4
:1057900085421CD11448844219D1144F387820B165
:1057A0002246294612A003F067FB387810B11CA0EE
:1057B00003F062FBFEF792FAFDF7B0FC20480660AA
:1057C00085F3088872B6A0470120BDE8F081224623
:1057D000294607A003F050FB1AA003F04DFB002060
:1057E000F3E70000A8370010814201080000001014
:1057F0000D0A204A756D70696E67206170705F6177
:105800006464726573732E2053503D3078253038B0
:10581000582C2050433D307825303858200D0A0050
:105820000D0A204A756D70696E67206170705F6146
:1058300064647265737320737563636573730000CA
:1058400008ED00E00D0A204A756D70696E672061F1
:1058500070705F61646472657373206661696C0067
:1058600030B59BB00C460546032815D2A4B164217F
:1058700001A8FAF764FD00201A901AA800902346A8
:1058800009A2622101A803F007FB01A9284601F043
:105890009DFD18B106A002E007A000E00EA003F0F5
:1058A000EBFA1BB030BD000025733D2573000000EE
:1058B0006F6B0D0A000000006572726F723D696EB9
:1058C00076616C696420706172616D732C20726CFA
:1058D000743D3435330D0A006572726F723D646534
:1058E0006C657465206661696C2C20726C743D3443
:1058F00035340D0A0000000070B5AAB014460D46FC
:10590000064603280ED26DB164B140211AA8FAF7F9
:1059100016FD40231AAA2946304605F03BFF18B170
:105920000DA014E012A012E0642101A8FAF707FD0F
:105930002B4617A2622101A8009403F0ADFA01A939
:10594000304601F043FD08B113A000E014A003F0BD
:1059500093FA2AB070BD00006572726F723D65786F
:10596000697374732C20726C743D3435360D0A00E3
:105970006572726F723D696E76616C6964207061E8
:1059800072616D732C20726C743D3435350D0A00D4
:1059900025733D25730000006F6B0D0A00000000A9
:1059A0006572726F723D696E7365727420666169AB
:1059B0006C2C20726C743D3435370D0A00000000E9
:1059C00070B59AB014460D460646032813D295B119
:1059D0008CB1642101A8FAF7B2FC2B4609A262211E
:1059E00001A8009403F058FA01A9304601F0EEFC3A
:1059F00018B106A002E007A000E00EA003F03CFAF8
:105A00001AB070BD25733D25730000006F6B0D0A41
:105A1000000000006572726F723D696E76616C699C
:105A20006420706172616D732C20726C743D34352A
:105A3000310D0A006572726F723D75706461746534
:105A4000206661696C2C20726C743D3435320D0A0D
:105A50000000000070B50446807A002839D0E38841
:105A6000002B36D020890A3082B22281A57C00200A
:105A700055B1E1898A422CD320812073A074E0744F
:105A8000A1880022206810E09A4222D32081E07C85
:105A900078B10020E07470B18B8808680022194644
:105AA000FDF7CAFDA18820680122BDE87040FDF71E
:105AB000C3BD0120EEE7A18800222068FDF7BCFDF0
:105AC000207B401CC0B22073E17A884201D30120C0
:105AD000A07470BD7CB50C4605460822103168469E
:105AE000FCF725FB208AC0F3C500382802D2C0F19C
:105AF000380201E0C0F178020949204600F094FB29
:105B000008226946204600F08FFB102221462846D5
:105B1000FCF70DFB58220021204600F0C6FB7CBD9F
:105B200064020010002141610161054901600549DD
:105B300041600349C94381600249C943C16070475C
:105B40000123456789ABCDEF2DE9F04750F804AB51
:105B5000002690E8340090B0E9464FF0400C334600
:105B6000001FCF181B1D97F803803F6868F31F675D
:105B700049F82670761CC8466345F2D302EA040150
:105B800025EA02031943FE4B009E0B4406EB0A0173
:105B9000194402EB716303EA020124EA030631436C
:105BA000F84E3144019E3544294403EB315101EA5A
:105BB000030522EA01063543F34E3544029E344480
:105BC0002C4401EBF43404EA010523EA04063543CE
:105BD000EE4E3544039E32442A4404EBB22202EADC
:105BE000040521EA02063543E94E3544049E334458
:105BF0002B4402EB736303EA020524EA03063543F0
:105C0000E44E3544059E3144294403EB315101EA09
:105C1000030522EA01063543DF4E3544069E34442F
:105C20002C4401EBF43404EA010523EA040635436D
:105C3000DA4E3544079E32442A4404EBB22202EA8B
:105C4000040521EA02063543D54E3544089E334407
:105C50002B4402EB736303EA020524EA030635438F
:105C6000D04E3544099E3144294403EB315101EAB9
:105C7000030522EA010635430A9EA5F5244534446E
:105C80004F3D2C4401EBF43404EA010523EA0406F9
:105C90003543C54E35440B9E32442A4404EBB222B0
:105CA00002EA040521EA02063543C04E35440C9E43
:105CB00033442B4402EB736303EA020524EA030630
:105CC0003543BB4E35440D9E3144294403EB3155D9
:105CD00005EA030122EA05063143B64E31440E9E21
:105CE0003444214405EBF13101EA050423EA0106BD
:105CF0003443B14E34440F9E3244224401EBB2226D
:105D000002EA050421EA05063443AC4E3444019E00
:105D10003344234402EBF36303EA010422EA01065D
:105D20003443A74E3444069E35442C4403EBF454CC
:105D300004EA020523EA02063543A24E35440B9ECF
:105D40003144294404EBB14101EA030524EA030686
:105D500035439D4E3544009E32442A4401EB323295
:105D600002EA040521EA04063543984E3544059EAF
:105D700033442B4402EBF36303EA010522EA0106F4
:105D80003543934E35440A9E34442C4403EBF4547B
:105D900004EA020523EA020635438E4E35440F9E7F
:105DA0003144294404EBB14101EA030524EA030626
:105DB0003543894E3544049E32442A4401EB323245
:105DC00002EA040521EA04063543844E3544099E5F
:105DD00033442B4402EBF36303EA010522EA010694
:105DE00035437F4E35440E9E34442C4403EBF4542B
:105DF00004EA020523EA020635437A4E3544039E3F
:105E00003144294404EBB14101EA030524EA0306C5
:105E10003543754E3544089E32442A4401EB3232F4
:105E200002EA040521EA04063543704E35440D9E0E
:105E300033442B4402EBF36303EA010522EA010633
:105E400035436B4E3544029E34442C4403EBF454EA
:105E500004EA020523EA02063543664E3544079EEE
:105E60003144294404EBB14101EA030524EA030665
:105E70003543614E35440C9E32442A44059D01EB66
:105E800032321D4482EA01035C4E634033442B44AA
:105E9000089D02EB3373254483EA02044C40584EBC
:105EA00034442C440B9D03EB74540D4484EA0301E9
:105EB000544E5140314429440E9D04EB3141154468
:105EC00081EA0402504E5A4032442A44019D01EBBB
:105ED00072221D4482EA01034C4E634033442B443A
:105EE000049D02EB3373254483EA0204484E4C4080
:105EF00034442C44079D03EB74540D4484EA03019D
:105F0000444E51403144294404EB31450A99424EF4
:105F10000A4485EA040159403144114405EB7126D5
:105F20000D99CA1886EA05013C4B61401944114499
:105F300006EB317300990A1983EA0601384C69406F
:105F400021441144039A03EB7151541981EA03026D
:105F5000344D72402A442244069C01EB3242A5197A
:105F600082EA0104304E5C4034442C44099D02EB2B
:105F700074241D4484EA02032C4E4B40334457E002
:105F800078A46AD756B7C7E8DB702024EECEBDC12F
:105F9000AF0F7CF52AC68747134630A8019546FD0A
:105FA000D8988069AFF7448BBED75C892211906B7B
:105FB000937198FD8E4379A62108B44962251EF697
:105FC00040B340C0515A5E26AAC7B6E95D102FD62D
:105FD0005314440281E6A1D8C8FBD3E7E6CDE12102
:105FE000D60737C3870DD5F4ED145A4505E9E3A963
:105FF000F8A3EFFCD9026F678A4C2A8D4239FAFF69
:1060000081F6718722619D6D0C38E5FD44EABEA4DE
:10601000A9CFDE4B604BBBF670BCBFBEC67E9B28D3
:10602000FA27A1EA8530EFD4051D880439D0D4D9E8
:106030002B440C9D04EB33730D4483EA0401674E3B
:1060400051403144294403EB71550F99644E0A4481
:1060500085EA030161403144114405EB3146029960
:106060000A1986EA05015F4C594021441144009AFF
:1060700006EB7121134461EA05025B4C7240224435
:106080001A44079B01EBB2625C1962EA0603574DA2
:106090004B402B44234402EBB3540E9B9D1964EAFE
:1060A0000103534E534033442B4404EB7345059B8B
:1060B000504E0B4465EA020161403144194405EB3E
:1060C000F1230C994C4E0A4463EA040169403144BF
:1060D000114403EBB1620399484E0C4462EA050196
:1060E00059403144214402EBB1540A99444E0D44C5
:1060F00064EA0301514031442944019D04EB71419C
:106100001D4461EA02033F4E634033442B44089D23
:1061100001EBF323154463EA04023B4E4A40324448
:106120002A440F9D03EBB262254462EA0104374E14
:106130005C4034442C44069D02EBB4540D4464EAA4
:106140000301334E5140314429440D9D04EB71410C
:106150001D4461EA02032F4E634033442B44049DE7
:1061600001EBF323154463EA04022B4E4A40324408
:106170002A440B9D03EBB262254462EA0104274ED8
:106180005C4034442C44029D02EBB4540D4464EA58
:106190000301234E514031442944099D04EB7141D0
:1061A0001D4461EA020363401E4E33442B440568DC
:1061B00001EBF3232A44026042681A444260826879
:1061C00011448160C16840222144C16000214046E1
:1061D00000F06BF810B0BDE8F0870000E599DBE651
:1061E000F87CA21F6556ACC4442229F497FF2A43C9
:1061F000A72394AB39A093FCC3595B6592CC0C8F59
:106200007DF4EFFFD15D84854F7EA86FE0E62CFE24
:10621000144301A3A111084E827E53F735F23ABD13
:10622000BBD2D72A91D386EB2DE9F0410F46016905
:1062300005461646C1F3C50001EBC6012961B1EB65
:10624000C60F696901D2491C696101EB5671C0F141
:1062500040046961A64216D32844224639461830C4
:1062600000F01AF805F118012846FFF76DFC04E06C
:1062700039192846FFF768FC403404F13F00B0426A
:10628000F6D3002000E00024321B39192844BDE871
:10629000F0411830AFF3008010B5002302E0CC5C71
:1062A000C4545B1C9342FAD310BD0023C9B201E071
:1062B000C1545B1C9342FBD370470000154808B5DE
:1062C000816C41F001018164806C002200F00100CA
:1062D000009005210E20FDF793FA0E20FDF783FABA
:1062E000002205210F20FDF78BFA0F20FDF77BFA26
:1062F000002205211020FDF783FA1020FDF773FA24
:10630000002205211120FDF77BFABDE8084011208D
:10631000FDF769BA0010024070B53C4D3C4C0220BC
:106320002871B4F8440080B201F0C4F900F0D6FE40
:1063300000F0F6FE3748206537A002F09DFD4FF4CF
:1063400088763D4A3146142004F09EFD05F1800414
:10635000394AA0601832B11E202004F095FD364A5B
:10636000E06030323146202004F08EFD324A206158
:10637000483204211E2004F087FD2F4A60616032FC
:1063800004211E2004F080FD2B4AA06178320421F4
:106390001E2004F079FD284AE061903204211E207D
:1063A00004F072FD244A2062A83204211E2004F069
:1063B0006BFD214A6062D83A0021204804F0C4FDF8
:1063C0001D4A2867B43A00211D4804F0BDFD1A4A51
:1063D0006867903A00211B4804F0B6FD164AA8678A
:1063E0006C3A0021184804F0AFFD134AE867483AB8
:1063F0000021164804F0A8FD0F4A2060243A00212D
:10640000134804F0A1FD606070BD00000000002092
:1064100040320010A83200100D0A204150495F4D53
:10642000554C206170703120323032355F30385F2A
:106430003230200D0A00000060DA0008055700081D
:10644000AD6D0008491E0008051800081970000805
:10645000E92B00082DE9F04186B014216846F9F7D0
:106460006EFF3048C16C41F00101C164C16C01F0A4
:1064700001010591C16C41F00201C164C06C4FF093
:10648000904600F002000590012210213046FDF7F1
:10649000D3F8DFF89480012240F6C3414046FDF76F
:1064A000CBF843F22407002239464046FDF7C4F8F2
:1064B00000224FF408413046FDF7BEF800240125C4
:1064C000CDE90054694630460294FCF7C5FF48F612
:1064D00010000090CDE90154694630460394FCF762
:1064E000BBFF03200226CDE90005CDE9024669463F
:1064F0004046FCF7B1FF0097CDE90154694640469C
:106500000394FCF7A9FF4FF44C60009001AA1120FE
:1065100082E8610069464046FCF79EFF06B0BDE890
:10652000F081000000100240000400480A4810B545
:10653000084901600321416040F6FF71C16081603C
:10654000FDF786F8002803D0BDE81040FBF708BE31
:1065500010BD00000030004030270010124810B578
:10656000104901604FF48271416000214FF4E062F4
:10657000C0E902120122C0E90412520282613822EB
:10658000C0E9072107224162C0E90A1201634163A1
:10659000FDF75AFF002803D0BDE81040FBF7E0BD2F
:1065A00010BD0000003001404027001010B588B039
:1065B00000241848009401940294039404940594D0
:1065C0001349069401600F21C0E901144FF6FF71D1
:1065D000C0E9031444618461FEF7D4FA08B1FBF703
:1065E000BFFD4FF48050009069460A48FEF764FBF7
:1065F00008B1FBF7B5FD049404A906480694FEF71C
:106600008BFA002801D0FBF7ABFD08B010BD0000ED
:1066100000400140D03C00200D4810B50B490160FE
:106620004FF416514160002181600C22C160C0E925
:1066300004128161C16101624162FEF731FE0028EE
:1066400003D0BDE81040FBF78BBD10BD0038014002
:10665000A42700100D4810B50B4901604FF4E1313B
:106660004160002181600C22C160C0E90412816197
:10667000C16101624162FEF713FE002803D0BDE84C
:106680001040FBF76DBD10BD0044004028280010ED
:10669000FEE7FEE7B5EEC00AF1EE10FA04D9B4EE5B
:1066A000E00AF1EE10FA02DBBFEE000A7047C0EE1E
:1066B000801AB7EE000A31EEC00A20EE010A7047D8
:1066C0001A49002001EB8002D2ED010AF4EEC00A63
:1066D000F1EE10FA24D8D2ED000AF4EEC00AF1EE81
:1066E00010FA1DDB01EB8001D2ED011AD1ED000A99
:1066F000A0F11401133801EE101A02EE100A30EE68
:10670000600AB8EEC11AB8EEC22A71EEE01A32EE93
:10671000412A20EE020AC0EE210A30EE810A7047BB
:10672000401C9128CEDB9FED020A7047C0DB0008B9
:106730009AF979C42DE9F04F2DED048B83B006460C
:10674000DDE910BA0078B0EE408A984691460D46D1
:10675000DFED408A404F0028A7F180045BD0087825
:10676000002853D018EE100AFAF752F941EC180B32
:106770005846FAF740F941EC190B4046FAF73BF955
:1067800041EC100BB0EE491AF0EE691A484603F0DE
:1067900093FA53EC182B51EC100BFAF73AF8FAF77E
:1067A0004AF908EE100A84ED088A8DED028A6078B5
:1067B000B0B194ED080A10EE100AFAF729F905466F
:1067C000B0EE480A0E4610EE100AFAF721F941EC35
:1067D000100BCDE9005653EC102B20A002F04CFB1F
:1067E00000231A4602A9F86900F0E4F800280DD049
:1067F000607800280AD018EE100AFAF709F941EC7F
:10680000100B1FA053EC102B02F036FB03B0BDECB5
:10681000048B00F059B8FBF701FF28B1002030705D
:1068200020B1012028709DE70120F8E7607818B1B9
:1068300051461BA002F020FBCDED028A00231A4630
:1068400002A9F86900F0B6F84FF4FA6004F098FA7B
:10685000DCE7000000000000800000206D7367315D
:106860002E64617461205B252E35665D206F696C36
:106870005F636170205B252E35665D0D0A000000A8
:106880000D0A51756575652066756C6C2C20636109
:10689000703D252E3366206E6F742073656E740014
:1068A0000D0A5265747279696E672025642054461A
:1068B00044433232313420696E69742020696E207D
:1068C0003273202E2E2E000030BCBDE8C08F000099
:1068D00000B50B48C5B000231A466946006804F0AD
:1068E000A1FA00280AD1BDF80E0128B19DF80000D8
:1068F00010B1684604F06CFB00F012FC45B000BD1E
:106900009000002070B52248C4B000231A466946A2
:10691000006804F087FA00281FD11E4D287810B1B6
:106920001DA002F0A9FA00246E4605E018B1315D01
:106930001DA002F0A1FA641CBDF80E01A042287847
:10694000F4DC10B11AA002F097FA684604F008F9D6
:106950000028684603D005F0E7F844B070BD04F0A5
:106960001FF90028684602D005F018F9F5E704F091
:1069700037F90028684602D005F052F9EDE704F037
:106980004DF90028E9D0684605F0AAF9E5E70000CE
:106990008800002000000010343835727842756697
:1069A0006665723A20000000253032582000000051
:1069B0000A0000002DE9F041C4B01D4616460F46FE
:1069C000804604F08DFA040008D0E01C08D00CA02A
:1069D00002F052FA204644B0BDE8F0810020FAE708
:1069E00000231A466946404604F01CFA0CA002F047
:1069F00043FA2B4632463946404604F071FAEAE73C
:106A00005B51756575655075744F766572777269FF
:106A100074655D206572726F72200D0A00000000BF
:106A20005B51756575655075744F766572777269DF
:106A300074655D2066756C6C200D0A00F0B5174614
:106A40000646B9423DDA06EB81000C4690ED000A9D
:106A5000154626E06D1EAC4208DA06EB8500D0ED47
:106A6000000AF4EEC00AF1EE10FAF3DA06EB850044
:106A700006EB8402D0ED000AC2ED000A00E0641CBF
:106A8000AC4208DA06EB8402D2ED000AF4EEC00A4A
:106A9000F1EE10FAF3D906EB8402D2ED000AC0ED54
:106AA000000AAC42D7DB06EB8400621E80ED000AD0
:106AB0003046FFF7C3FF3A46611C3046BDE8F04060
:106AC000BCE7F0BD2DE9F041444C05468846E0683E
:106AD0000026810728680DD0E16801F0030181429A
:106AE00016D1A8B1E0686968C0F30210401C884262
:106AF0000ED120E0012804D0022805D0032807D1B8
:106B000008E02168890701E021684905002907DBC1
:106B100001265FE02168890302D421684903F5E773
:106B2000E1686A686FF00F0321F0730103EB021252
:106B300011430143E160206820F080602060FCF791
:106B400081FD074605E000BFFCF77CFDC01B022865
:106B500037D820680001F7D4B8F1000F18D0B8F189
:106B6000010F1DD0287D4FF07E41400801EB4060B1
:106B7000A96840EA01202169194A114008432061AF
:106B8000206840F080602060FCF75CFD07461AE05A
:106B9000A868297B000240EAC1602169114AECE73C
:106BA000288A1149400801EB4050A96840EA0120B9
:106BB00021690E4AE1E700BFFCF744FDC01B022833
:106BC00001D9032606E020680001F5D52069A969EE
:106BD000084320613046BDE8F0810000001002400B
:106BE000FF80FFF9FF80FF070000E0FFFF809FFFAD
:106BF000F8B51C4D06460024A86DC00002D5FCF770
:106C000065FE0DE0A86D40F08050A865A86D00F00D
:106C100080500090FCF75AFEA96D21F08051A965C3
:106C2000B0F5007F04D0802E07D94FF003040AE0AE
:106C3000802E08D9A02E01D804E001D1022402E060
:106C4000702E00D101240848016821F0070121437A
:106C50000160006800F00700A04201D00120F8BDEB
:106C60000020F8BD001002400020024010B5184876
:106C7000006828B105F0E0FE014616A002F0FCF81D
:106C80001E48006828B105F0D7FE01461CA002F09E
:106C9000F3F82548006828B105F0CEFE014623A090
:106CA00002F0EAF82B48006828B105F0C5FE01465D
:106CB00029A002F0E1F832480068002807D005F06A
:106CC000BBFE0146BDE810402EA002F0D5B810BDB5
:106CD00070000020486967686573745461736B487D
:106CE000616E646C6520737461636B2072656D61A5
:106CF000696E696E673A20256C750A007400002081
:106D0000526561645461736B48616E646C65207395
:106D10007461636B2072656D61696E696E673A209C
:106D2000256C750A00000000780000204465616C45
:106D30005461736B48616E646C6520737461636B3E
:106D40002072656D61696E696E673A20256C750AFF
:106D5000000000007C000020436F6D6D6F6E546179
:106D6000736B48616E646C6520737461636B207231
:106D7000656D61696E696E673A20256C750A000061
:106D800080000020526561645461736B3032486149
:106D90006E646C6520737461636B2072656D6169EC
:106DA0006E696E673A20256C750A00002DED028B26
:106DB00084B06648FAF7F0FB4FF090479FED648A85
:106DC000644DA5F1800401213846FCF730FC002811
:106DD00078D1E078FAF70CFC0121B0EE040AFAF75A
:106DE000C7FBE07820B1012838D002286BD16EE0D3
:106DF000C0EE080A94ED030A30EE800A84ED020A20
:106E000094ED020A8DED010AA07860B194ED020ABA
:106E100010EE100AF9F7FCFD41EC100B4EA053ECFC
:106E2000102B02F029F800231A4601A96869FFF720
:106E3000C1FD00287ED0666E761C6666A0780028AC
:106E400078D094ED050A10EE100AF9F7E1FD41EC57
:106E5000100B45A053EC102B009669E0C0EE080A19
:106E600094ED120A30EEC00A84ED110A94ED110A75
:106E70008DED020AA07860B194ED110A10EE100AAF
:106E8000F9F7C6FD41EC100B43A053EC102B01F0B9
:106E9000F3FF00231A4602A9286AFFF78BFD00289A
:106EA00048D0A66E761CA666A078002842D094ED45
:106EB000140A10EE100AF9F7ABFD41EC100B53EC7D
:106EC000102B01E03EE035E037A0009630E0D4ED35
:106ED000160A30EE600A84ED150A94ED150A8DED60
:106EE000030AA07860B194ED150A10EE100AF9F7C4
:106EF0008FFD41EC100B38A053EC102B01F0BCFFC0
:106F000000231A4603A9686AFFF754FD90B1E66EA4
:106F1000761CE666A07868B194ED150A10EE100AAA
:106F2000F9F776FD41EC100B2FA053EC102B0096D7
:106F300001F0A2FFE078401CC0B2E070022801D945
:106F40000020E0700A2003F01BFF3CE74027001000
:106F5000CDCCCC3E800000204144535F76302025CC
:106F60002E3566200D0A00000D0A517565756520E5
:106F700066756C6C2C204D5058565F50303D252E58
:106F80003366206E6F742073656E742E2044726FAA
:106F9000707065643D2564004144535F763120255F
:106FA0002E3566200D0A00000D0A517565756520A5
:106FB00066756C6C2C204D5058565F50313D252E17
:106FC0003366206E6F742073656E742E2044726F6A
:106FD000707065643D2564004144535F763220251E
:106FE0002E3566200D0A00000D0A51756575652065
:106FF00066756C6C2C204144535F76323D252E33F0
:1070000066206E6F742073656E742E2044726F70EC
:107010007065643D2564000086B00020DFF8B8800C
:107020008DF80C008DF80800054641F2883600BF47
:10703000FCF708FB0446C01BB04205D3274604AA50
:1070400005A90120FAF77EFB9DF81000C8B198ED64
:10705000070A012205A8BCEEC00A10EE101AC9B238
:10706000CDE9001298ED070A98ED060A0022BCEE61
:10707000C00A10EE101A98ED090ACBB204A9FFF766
:1070800059FB601BB04205D3254602AA03A9022082
:1070900000F0F6FB9DF80800C8B198ED0D0A022239
:1070A00003A8BCEEC00A10EE101AC9B2CDE9001256
:1070B00098ED0D0A98ED0C0A0022BCEEC00A10EE05
:1070C000101A98ED0F0ACBB202A901F0CBF80A20F2
:1070D00003F056FEACE700000000002070B50E483B
:1070E000FDF72DFF0C4C1020216808622068016814
:1070F00021F0100101604FF4877529460748F9F720
:107100001EF92A4605492046FEF714FA2068016850
:1071100041F01001016070BDA4270010CC290010BF
:1071200070B51048FDF70BFF4FF4877529460E48E0
:10713000F9F705F90B4C2068016821F01001016096
:107140000A49002008602168102008622A46064982
:107150002046FEF7EFF92068016841F01001016058
:1071600070BD0000282800101C3D00200800001001
:107170002DE9F843044640684FF482761546894667
:107180004FF400474FF48068B04209D1A068B8427C
:1071900001D0404504D12068016821F04001016020
:1071A0004B46002280212046009500F0B3F880B9BC
:1071B0006068B04214D1A068B84201D040450FD1F8
:1071C0004B4600224FF4C0612046009500F02EF897
:1071D00030B1206E40F0200020660320BDE8F88327
:1071E0000020FBE7F8B515460E460B460092044614
:1071F00000224FF4C05100F019F888B9334600223C
:1072000080212046009500F085F848B933460022D9
:107210004FF4C0612046009500F008F8002804D023
:10722000206E40F0200020660320F8BD2DE9FE4FBF
:107230004FF0000A984617460E4604460C9D8DF8FE
:1072400004A0FCF7FFF9411BA8EB0105FCF7FAF9D4
:10725000814620684FF4C06B0C3002902A480068C9
:10726000C0EBC00000EB8000000D6843009043E0DD
:107270005E4506D12FB9029800788DF804009DF87C
:107280000400B8F1FF3F37D0FCF7DCF9A0EB0900B0
:10729000A84203D215B1009858B32BE0206841688A
:1072A00021F0E00141606068B0F5827F0BD1A068F9
:1072B000B0F5004F02D0B0F5806F04D120680168AE
:1072C00021F040010160A06AB0F5005F09D120689B
:1072D000016821F4005101602068016841F4005107
:1072E0000160012084F85D0084F85CA0032000F0B8
:1072F0000DB80025401E0090206880683040B842DC
:10730000B6D10020F3E70000D00000201EBCBDE88D
:10731000E08F00002DE9F8431E469146884604465A
:10732000089DFCF78FF9401B351AFCF78BF90746CF
:1073300025480068C0F3CB30684338E0701C37D074
:10734000FCF780F9C01BA84203D215B1009860B3C6
:107350002CE02068416821F0E00141606068B0F5F0
:10736000827F0BD1A068B0F5004F02D0B0F5806FDE
:1073700004D12068016821F040010160A06AB0F5E5
:10738000005F09D12068016821F400510160206884
:10739000016841F400510160012084F85D00002083
:1073A00084F85C000320BDE8F8830025401E0090AF
:1073B0002068816838EA010004D000214945BDD128
:1073C0000020F0E70121F9E7D00000202DE9F34F7C
:1073D000ABB000252B988946032807D20846B9F19F
:1073E000000F03D0F8F7EAFF622803D366A001F08C
:1073F00043FD12E0242119A8F8F7A1FF3D214846DA
:10740000F8F7D2FF060004D0A6EB09044846202C6A
:1074100007DD494667A001F02FFD00202DB000F0E8
:1074200045B90146224619A8F8F7B2FF19A9AA469C
:107430000D556B4D287810B16AA001F01DFD4FF479
:10744000006421466E48F8F77AFF22466C492B9873
:10745000FAF76CFA0146287810B16AA001F00CFD29
:1074600021467148F8F76BFF4FF0000864483CE094
:10747000801C83466DA1F8F779FF040002D0A4EBCD
:107480000B0002E05846F8F799FF0746642168466A
:10749000F8F755FF3A4659466846F8F779FFEB4644
:1074A0000DF807A03D215846F8F77EFF07001AD0D7
:1074B000242122A8F8F743FFA7EB0B073A466946B9
:1074C00022A8F8F765FF22A922A801F807A019A9A8
:1074D000F8F77BFF90B155A15348F8F73BFF694699
:1074E0005148F8F737FF2CB1204650A1F8F73EFF7E
:1074F0000028BDD1B8F1000F1CD02DE04FF00108DD
:10750000701CF8F75BFF68B148A14748F8F722FF05
:1075100049464548F8F71EFF28780028E3D0494639
:1075200043A004E028780028DDD022A948A001F07B
:10753000A3FCD8E7701CF8F741FF68B13BA13A48BB
:10754000F8F708FF49463848F8F704FF287818B1DB
:10755000494645A001F090FC34A13348F8F7FAFE03
:10756000287838B13048F8F729FF01462E4A46A05E
:1075700001F082FC2C48F8F721FF82B22A492B98AF
:10758000FAF7D6FA4AE700005B4B565D20496E7663
:10759000616C6964204442204944206F72206B76FC
:1075A0005F73747220746F6F206C6F6E672F6E75CF
:1075B0006C6C0A005B4B565D20273D27206E6F7474
:1075C00020666F756E64206F72206B657920746F12
:1075D0006F206C6F6E6720696E20272573270A0065
:1075E000010000105B4B565D2050726F6365737332
:1075F000696E67206B65793D272573270A000000B7
:10760000148500205B4B565D204578697374696E64
:1076100067204442206C656E6774683A20257520A7
:1076200062797465730A0000148D00202323000022
:107630005B4B565D205570646174696E67206B65A5
:107640007920696E20706C6163653A2025730A00A9
:107650005B4B565D2044656C6574696E67206B6595
:10766000793A2025730A00005B4B565D2041646423
:10767000696E67206E6577206B7620617420656E79
:10768000643A2025730A00005B4B565D2046696E04
:10769000616C20444220636F6E74656E7420286CA8
:1076A000656E3D2575293A0A25730A0030BCBDE890
:1076B000C08F000010B54FF4165109281AD2DFE828
:1076C00000F0190519080B0E111417004FF496510C
:1076D00010E04FF461510DE04FF496410AE04FF491
:1076E000164107E04DF6C02104E04FF4614101E08E
:1076F0004FF4E1310F480E4AC0E9002100218160BA
:107700000C22C160C0E904128161C1610162416261
:10771000FDF75BFC08B1FAF723FD0648FDF7C0FD55
:10772000002803D0BDE81040FAF71ABD10BD0000D4
:1077300000380140A427001010B504462821F8F7AE
:10774000FEFD002004F8280F607010BD10B590F801
:1077500028108AB000EB81010A2281ED000A90F81E
:107760002810491CB1FBF2F302FB131480F82840E7
:10777000ACB190F8291001B10A240146A200684674
:10778000F8F7C4FD621E00216846FFF757F9DFEDE8
:10779000180A6946022C17D90120621E0CE001214B
:1077A00080F82910E8E700BF01EB8003401C93ED4F
:1077B000000AC0B270EE200A9042F5DBA41E00EE73
:1077C000104AB8EEC01A0FE0002007E001EB80027B
:1077D000401C92ED000AC0B270EE200AA042F5D320
:1077E00000EE104AB8EE401A0AB080EE810A10BDD1
:1077F0000000000010B54FF0E020006905F00EFF1A
:10780000012803D0BDE8104005F0CABB10BD10B57B
:1078100096B044216846F8F792FD142111A8F8F7B4
:107820008EFD4FF40070FCF71DF808B172B6FEE74C
:107830001820009001200024CDE906040590802046
:1078400008900A946846FCF74FFB08B172B6FEE751
:107850000F20CDE9110413941494002111A815945C
:10786000FCF79AF9002801D072B6FEE716B010BDF9
:107870000248016841F470010160704788ED00E042
:107880002DE9F8430F46804615467F212A2000F057
:10789000E7FA0446174EA0F54050553820D0002096
:1078A00028709FED150A387006F180058DED000AED
:1078B000034602466946A869FFF77CF800231A468A
:1078C0006946A86903F0AEFA0028F7D0707800285E
:1078D00004D02246414609A001F0CEFABDE8F88363
:1078E000707820B1224641460DA001F0C5FA012072
:1078F0002870F3E700000020000000005B544644BD
:1079000043323231342D25645D206572726F723AD4
:107910002049443D3078253034580D0A00000000DD
:107920005B54464443323231342D25645D206F6B05
:107930003A2049443D3078253034580D0A00000083
:1079400010B511EE900A2DED068BB0EE41AAB0EE07
:10795000408AF0EE608AF9F75BF89FED150B41EC79
:10796000190B53EC102B51EC180BF8F760FF41EC9E
:10797000180B1AEE100AF9F74BF853EC182BF8F71E
:1079800056FF53EC182BF8F752FF41EC100B53EC59
:10799000102B9FED090B51EC100BF8F7BDFF53ECCA
:1079A000192BF8F736FFBDEC068B41EC100B10BD20
:1079B0004AD8124DFB21194000C84E676DC1AB4338
:1079C00010B504462DED028B0846F9F714F841EC8A
:1079D000180B1048005DF9F70EF841EC100B0E483B
:1079E00000EBC40090ED001B51EC100B53EC112B7D
:1079F000F8F71DFF53EC182BF8F719FF9FED071B45
:107A000053EC112BF8F713FFBDEC028B41EC100B7C
:107A100010BD000044030020683300100000000087
:107A20000000303E2DE9F0418846642430B1012841
:107A300008D002280AD003280FD10BE00027012626
:107A400008250AE002270326042506E00427052668
:107A5000022502E006270726012518212A2000F02A
:107A6000FFF906E018212A2000F0FAF9641E24B27A
:107A70008CB12842F6D074B139462A2000F0F0F9D2
:107A8000040431462A2000F0EBF92043C8F8000036
:107A90000120BDE8F0810020FBE7000010B5124C8A
:107AA000002240212046FBF7C7FD022000F0AAFC7F
:107AB00000F016FA002280212046FBF7BDFD0220CF
:107AC00000F0A0FC012240212046FBF7B5FD02207A
:107AD00000F098FC002240212046FBF7ADFDBDE8F8
:107AE0001040022000F08EBC0004004810B5124C7B
:107AF000002240212046FBF79FFD022000F082FC7F
:107B000000F0EEF9012280212046FBF795FD0220CE
:107B100000F078FC012240212046FBF78DFD022079
:107B200000F070FC002240212046FBF785FDBDE8F7
:107B30001040022000F066BC000400482DE9F0412E
:107B40001A4E07460024012280213046FBF774FDBF
:107B500000F0B2F900256006040E002240213046F4
:107B6000FBF76AFD022000F04DFC01224021304667
:107B7000FBF762FD022000F045FC80213046FBF758
:107B800056FD08B1641CE4B26D1CEDB2082DE2D3C1
:107B9000002240213046FBF74FFD27B1FFF77EFF63
:107BA0002046BDE8F081FFF7A1FFF9E70004004897
:107BB00070B5054600F094F9144E0022402130467D
:107BC000FBF73AFD0024022000F01CFC280601D53A
:107BD000012200E0002280213046FBF72DFD6806DF
:107BE000050E012240213046FBF726FD022000F061
:107BF00009FC002240213046FBF71EFD022000F068
:107C000001FC641CE4B2082CDDD370BD0004004804
:107C100010B500F065F9104C012280212046FBF7D9
:107C20000BFD012240212046FBF706FD022000F05B
:107C3000E9FB002280212046FBF7FEFC022000F039
:107C4000E1FB002240212046FBF7F6FCBDE8104096
:107C5000022000F0D7BB00000004004810B500F07F
:107C60003FF9114C002240212046FBF7E5FC0220A1
:107C700000F0C8FB002280212046FBF7DDFC02203B
:107C800000F0C0FB012240212046FBF7D5FC02207A
:107C900000F0B8FB012280212046FBF7CDFCBDE8B7
:107CA0001040022000F0AEBB0004004870B5002474
:107CB00000F002F9134D012280212846FBF7BCFC9D
:107CC000022000F09FFB012240212846FBF7B4FC74
:107CD000022000F097FB07E0641CE4B2FA2C03D901
:107CE000FFF7BCFF012070BD80212846FBF79FFCF9
:107CF0000028F1D1002240212846FBF79DFC0020FE
:107D000070BD0000000400482DE9F0412F4C2078A0
:107D100010B12FA001F0B0F87F212A2000F0A0F8C8
:107D20000546207818B1294631A001F0A5F8A5F53F
:107D3000405044F620674FF47A6655380CD02078CE
:107D400010B133A001F098F8207810B137A001F0FD
:107D500093F80120BDE8F08100F0A8F83946002032
:107D600000F0B0F93146002000F0C4F901220221F0
:107D7000002000F0DDF8002000F077F9012000F08D
:107D80003CF9012000F028F9002000F05DF9042200
:107D90000021012000F087F9002000F0B5F815213E
:107DA000002000F03BF9002000F0BAF9207810B173
:107DB00026A001F061F8207810B11CA001F05CF859
:107DC000642002F0DDFF0020C4E700000100002075
:107DD0000D0A3D3D3D2054464443323231345F6408
:107DE00065766963654944203D3D3D0D0A0000000C
:107DF00054464443323231345F6465766963654981
:107E00004420203A20307825303278200D0A0000B6
:107E1000544644433232313420496E6974204661FD
:107E2000696C65642121200D0A0000003D3D3D3D47
:107E30003D3D3D3D3D3D3D3D3D3D3D3D3D3D3D3D72
:107E40003D3D3D3D3D3D3D3D0D0A00005446444312
:107E50003232313420496E6974204F4B210D0A00B3
:107E600070B50D460446FFF7D3FE6006000EFFF71F
:107E70009FFEFFF71BFF2846FFF79AFEFFF716FF4E
:107E8000FFF7C6FE012000EB4400C0B2FFF790FEF2
:107E9000FFF70CFF0120FFF751FE04020020FFF75F
:107EA0004DFE0443FFF7DAFE204670BD1C214FF45F
:107EB00000422A2000F045B900B585B0142168467B
:107EC000F8F73DFA802000900020019001200290F8
:107ED00069460248FBF7C0FA05B000BD000400483F
:107EE00000B585B014216846F8F729FA8020009083
:107EF000112001900120029069460248FBF7ACFA7C
:107F000005B000BD0004004810B504461A212A201F
:107F1000FFF7A6FF4FF6FF7101EA8432C0F30D00B0
:107F200002431A21BDE810402A2000F00AB90000DF
:107F300070B504464FF6FF7000EA0136C2F309003F
:107F400006431948154601551848007810B118A085
:107F500000F092FF2846F8F74EFD41EC100B53EC71
:107F6000102B9FED1A0B51EC100BF8F7D5FC194AAA
:107F700002EBC402C2E9000164B1012C0DD0022C55
:107F80000ED0032C0FD132461721BDE870402A20B5
:107F900000F0D7B832461421F7E732461521F4E74E
:107FA00032461621F1E770BD440300200100002095
:107FB0004672657175656E63795F73656C65637430
:107FC00020203A202564200D0A0000000000000057
:107FD000D01283416833001010B504461A212A20BC
:107FE000FFF73EFF20F400720CB142F400721A2138
:107FF000BDE810402A2000F0A4B810B504461A21AC
:108000002A20FFF72DFF20F400620CB142F4006239
:108010001A21BDE810402A2000F093B84FF6FF72F5
:1080200002EAC12248B1012809D0022809D0032858
:1080300009D121212A2000F084B81E21FAE71F214E
:10804000F8E72021F6E7704710B504461A212A20E8
:10805000FFF706FF20F040020CB142F040021A2167
:10806000BDE810402A2000F06CB810B504461A2173
:108070002A20FFF7F5FE20F080020CB142F08002CA
:108080001A212A2000F05DF819212A20FFF7E8FEC6
:1080900020F001020CB142F001021921BDE81040AC
:1080A0002A2000F04EB838B1C00340EA41301043F6
:1080B00080B240F4027201E042F402721B212A20D5
:1080C00000F03FB8FF2914D950B101280BD0022885
:1080D0000CD003280DD10A460B212A2000F031B81C
:1080E0000A460821F9E70A460921F6E70A460A2165
:1080F000F3E7704750B101280BD002280CD00328B9
:108100000DD10A4613212A2000F01BB80A4610217F
:10811000F9E70A461121F6E70A461221F3E770470C
:1081200010B504461A212A20FFF79AFE20F40052C7
:108130000CB142F400521A21BDE810402A20AFF3DE
:10814000008070B514460E460546FFF761FD6806CF
:10815000000EFFF72DFDFFF7A9FD3046FFF728FDC4
:10816000FFF7A4FD200AFFF723FDFFF79FFDE0B214
:10817000FFF71EFDFFF79AFDBDE87040FFF76EBDEB
:108180000148FCF70ABE0000DC2A001070B5026846
:10819000164B4FF08046984201D0B04203D122F0F6
:1081A00070044A682243124C124D984205D0B042E6
:1081B00003D0A04201D0A84203D122F44076CA687D
:1081C00032434E6922F08002324302608A68C26202
:1081D0000A688262984203D0A04201D0A84201D12D
:1081E000096901630121416170BD0000002C01405B
:1081F000004001400044014010B5846842EA032277
:1082000024F47F440A432243826010BD826822F036
:1082100070020A4342F007018160704710B5036A9B
:10822000046A24F001040462846924F0F00444EA3E
:10823000021423F00A020A438461026210BD10B5E1
:10824000036A23F0100303628369046A23F4704312
:1082500043EA023224F0A00343EA01118261016281
:1082600010BD00002DE9F04F2DED048B83B00646C4
:10827000DDE910BA0078B0EE408A984691460D4686
:10828000DFED408A404F0028A7F180045BD00878DA
:10829000002853D018EE100AF8F7BAFB41EC180B7F
:1082A0005846F8F7A8FB41EC190B4046F8F7A3FB3A
:1082B00041EC100BB0EE491AF0EE691A484600F096
:1082C00009F953EC182B51EC100BF8F7A2FAF8F758
:1082D000B2FB08EE100A84ED0E8A8DED028A6078FA
:1082E000B0B194ED0E0A10EE100AF8F791FB0546B6
:1082F000B0EE480A0E4610EE100AF8F789FB41EC82
:10830000100BCDE9005653EC102B20A000F0B4FD6B
:1083100000231A4602A9B869FEF74CFB00280DD0CD
:10832000607800280AD018EE100AF8F771FB41ECCB
:10833000100B20A053EC102B00F09EFD03B0BDEC01
:10834000048B00F05BB8FFF7DFFC28B10020307031
:1083500020B1012028709DE70120F8E7607818B16E
:1083600051461CA000F088FDCDED028A00231A467C
:1083700002A9B869FEF71EFB4FF4FA6002F000FD97
:10838000DCE7000000000000800000206D73673211
:108390002E64617461205B252E35665D20726573E5
:1083A0005F6F696C5F636170205B252E35665D0DC4
:1083B0000A0000000D0A51756575652066756C6CC4
:1083C0002C206361703D252E3366206E6F74207300
:1083D000656E74000D0A5265747279696E672025A6
:1083E0006420544644433232313420696E6974202B
:1083F00020696E203273202E2E2E000030BCBDE886
:10840000C08F000004490A68516A89B2536A5B1A36
:108410008342FBD370470000D03C00202DE9F0419F
:1084200094B000240F46804626466D46761CB6B2B0
:1084300039464046FFF7F6FA012804D1386845F876
:108440002400641CA4B26420FFF7DCFF142C0FD2BC
:10845000642EEBD3142C0BD21148007818B12146AE
:1084600010A000F009FD4FF0FF3014B0BDE8F0811E
:10847000009C012123461A4655F82100984200DD50
:108480000346904200DA0246491C89B2044414298A
:10849000F2D3E01A801A122190FBF1F0E5E7000018
:1084A000000000104644433232313420646174616C
:1084B00020726561642074696D656F757421204F49
:1084C0006E6C792025642073616D706C65732E0D60
:1084D0000A00000070B5354C354D2DED068BB0EE21
:1084E000408AF0EE608AB0EE419A9FED2E0BF0EEDE
:1084F000619A68B3012838D0022843D003284ED1AE
:1085000004F11001FFF78AFF014620610320FFF705
:1085100057FA85ED060B00BFB0EE40AAF0EE60AA58
:1085200051EC190BF8F787FA09EE100A51EC180B09
:10853000F8F781FAF0EE491AB0EE4A0AF0EE6A0A4C
:10854000BDEC068B01EE100ABDE87040FFF7F8B9EC
:1085500016490020091DFFF761FF014660600020F9
:10856000FFF72EFA85ED000BD6E710490120083100
:10857000FFF754FF0146A0600120FFF721FA85EDC7
:10858000020BC9E7094902200C31FFF747FF0146FA
:10859000E0600220FFF714FA85ED040BBCE7BDECA8
:1085A000068B70BD000000000000000044030020A6
:1085B0008833001010B5ADF50A7D1A48FCF7BFFCF2
:1085C000194800684068D0F587741848046024D0C2
:1085D000B4F5877F21D84FF488716846F7F7AFFE6E
:1085E000ADF80E41224612496846F7F78FFE00208B
:1085F000104C0346889088AA6946206804F02EFE35
:1086000001280AD088AA44A9206804F023FF002387
:1086100088AA6946206804F021FEFEF75FFD0DF58B
:108620000A7D10BDA4270010AC280010AC0000206B
:10863000CC2900108800002010B5ADF50A7D1D483A
:10864000FCF77DFC1C4800684068C0F587741B4837
:108650000460201FB0F5857F04D9FEF761FD0DF59C
:108660000A7D10BD4FF488716846F7F768FE002058
:108670008890ADF80E41224611496846F7F746FE4C
:108680004FF487710E48F7F75AFE0E4C002388AA64
:108690006946206804F0E2FD0128E0D088AA44A9D8
:1086A000206804F0D7FE002388AA6946206804F0F9
:1086B000D5FDD4E7282800103C2900100800001040
:1086C0001C3D00209000002090F82410C90706D01F
:1086D00001684A68836A22F400321A434A6090F8BB
:1086E0002410890706D501684A68C36A22F48032DB
:1086F0001A434A6090F82410490706D501684A6871
:10870000036B22F480221A434A6090F82410090770
:1087100006D501684A68436B22F400421A434A6056
:1087200090F82410C90606D501688A68836B22F484
:1087300080521A438A6090F82410890606D5016891
:108740008A68C36B22F400521A438A6090F824109E
:10875000490611D501684A68036C22F480121A4355
:108760004A60016CB1F5801F06D101684A68436C0C
:1087700022F4C0021A434A6090F82410090606D574
:1087800001684A68806C22F4002202434A60704704
:10879000F8B500260446C0F88060FAF753FF054696
:1087A000206800686FF07E47000708D52B4600223E
:1087B0004FF400112046009700F040FA60B920689D
:1087C000006840070AD52B4600224FF4800120465E
:1087D000009700F033FA08B10320F8BD2020A0670D
:1087E000E067266684F874600020F8BD10B5806AE2
:1087F0000021A0F85A10A0F85210FCF705FC10BD9B
:1088000070B5846AA06FE56F216889684FF0000633
:10881000090606D5212804D1A4F85260204600F0AC
:10882000AEF820688068400606D5222D04D1A4F851
:108830005A60204600F07EF8D4F8800040F0100026
:10884000C4F880002046FCF7DFFB70BD10B5014680
:10885000806A0968096889062DD40021A0F85A1099
:10886000016851E8002F22F4807241E80023002BB8
:10887000F6D10168083151E8002F22F0010241E8E9
:108880000023002BF5D10168083151E8002F22F0B8
:10889000400241E80023002BF5D12021C167016E81
:1088A000012908D1026852E8001F21F0100142E8B6
:1088B0000013002BF6D1016E012902D0FCF764FEF3
:1088C00010BDB0F85810FCF738FB10BD10B5806A29
:1088D000016E012902D0FCF758FE10BDB0F8581007
:1088E0004908FCF72AFB10BD10B50146806A0968EB
:1088F0000968890616D40021A0F8521001680831D1
:1089000051E8002F22F0800241E80023002BF5D12E
:10891000026852E8001F41F0400142E80013002BBA
:10892000F6D110BDFCF7DEFE10BD10B5806AFCF775
:10893000E7FE10BD016851E8002F22F4907241E873
:108940000023002BF6D10168083151E8002F22F0F6
:10895000010241E80023002BF5D1016E012908D165
:10896000026852E8001F21F0100142E80013002BBA
:10897000F6D12021C1670021016641667047026877
:1089800052E8001F21F0C00142E80013002BF6D18D
:1089900020218167704700002DE9F04104460168FD
:1089A00080682269E3691043626900251A43104315
:1089B000714F0A68714B1A4002430A60206841688F
:1089C000E26821F44051114341602168A069B94235
:1089D00001D0226A10438A6822F4306202438A601E
:1089E0006749236867488B420DD1D0F8880010F0A2
:1089F000030006D0012847D0022843D0032830D1F5
:108A000044E001212EE060498B420BD1D0F8880070
:108A100010F00C0034D0042836D0082832D00C28AE
:108A20001FD133E059498B420BD1D0F8880010F0A8
:108A3000300025D0102827D0202823D0302810D16E
:108A400024E0BB420DD1D0F8880010F4406017D06C
:108A5000B0F5806F18D0B0F5006F13D0B0F5406F4F
:108A600014D010214A4A00264FF40040BB422FD1B7
:108A700071B102290FD004290FD0082973D10FE05A
:108A80000021EFE70221EDE70421EBE70821E9E708
:108A9000FBF7B4F903E0104602E0FBF7D3F9E8B3C3
:108AA000626802EB420181425DD8B0EB023F5AD8C6
:108AB000010E03025008181871410023F7F7F2FB6A
:108AC000344AA0F5407191424DD82168C8604BE00E
:108AD000E3694FF6EF77834228D1092943D2DFE8D3
:108AE00001F005080B420D4242421000FBF786F9E7
:108AF00006E0FBF795F903E0104602E0FBF7A2F968
:108B000060B14100606801EB5001B1FBF0F0A0F1F1
:108B10001001B94227D84FF6F07100E024E001407F
:108B2000C0F3420001432068C1601DE009291AD248
:108B3000DFE801F005080B190D1919191000FBF7F2
:108B40005DF906E0FBF76CF903E0104602E0FBF785
:108B500079F948B1616800EB5100B0FBF1F0A0F188
:108B60001001B94205D9012566662846A666BDE80A
:108B7000F08180B2A9E7000000800040F369FFEFB8
:108B8000003801400010024000440040004800400E
:108B90000024F400FFFC0F0070B54165A0F85820D8
:108BA00000250446C0F880502220E067206FD8B12D
:108BB0001F49C162216F1F4813460863216F1E4879
:108BC0004863206F8563666D216832462431206FCB
:108BD000FAF76CFA40B11020C4F8800004F8745F12
:108BE0002020A060012070BD84F87450206940B13D
:108BF000216851E8000F40F4807041E80002002A2B
:108C0000F6D12068083050E8001F41F0010140E82B
:108C10000012002AF5D12068083050E8001F41F00A
:108C2000400140E80012002AF5D1002070BD00008C
:108C30004D880008CD880008018800082DE9F0471C
:108C40009A4617460E4604464FF000094FF020089A
:108C5000089D4AE0681C48D0FAF7F4FCA0EB0A0033
:108C6000A8422AD84DB32068016849073DD5C0699C
:108C7000C043000539D421684FF4006008622068C1
:108C800050E8001F21F4D07140E80012002AF6D10C
:108C90002068083050E8001F21F0010140E8001270
:108CA000002AF5D1C4F87880C4F87C80C4F88080AC
:108CB00084F874900320BDE8F087216851E8000F24
:108CC00020F4D07041E80002002AF6D12068083074
:108CD00050E8001F21F0010140E80012002AF5D100
:108CE000C4F87880C4F87C80E2E72068C06936EA7E
:108CF000000004D00020B842ACD00020DBE7012007
:108D0000F9E7000010B5114C2068C169C943C906D4
:108D100003D410210162FFF74DFC2068C1690907E7
:108D200005D4C169490702D4C169890709D5082159
:108D30000162216804200862216802200862FEF7AF
:108D4000CDF9BDE810400148FCF760B9A427001038
:108D500010B5114C2068C169C943C90603D410215C
:108D60000162FFF769FC2068C169090705D4C16980
:108D7000490702D4C169890709D508210162216820
:108D800004200862216802200862FEF7C9F9BDE8E4
:108D900010400148FCF73AB9282800102DE9F047A7
:108DA00084464FF4FA77324B012430486425BE00E4
:108DB00000224FF480594FF4005AA3F11401BCF182
:108DC0000A0F50D2DFE80CF005050E191E242C32D4
:108DD00039429A728A72012249460446FAF72CFCFB
:108DE000002207E09A728A72002249460446FAF786
:108DF00023FC01225146204624E09C72DF808A72C7
:108E0000BDE8F0879C72DF808C72CD80CC7205E06B
:108E10009C72DF808C72CD8002200CE0CE811FE03E
:108E20009C72DF808C72CD80032004E09C72DF8016
:108E30008C72CD800420C872F0E79C72DF808A7249
:108E400001225146BDE8F047FAF7F6BB9C72DD807F
:108E5000DC72DA811A739A748C72CD80CC72CA81FA
:108E60000A738A74CCE79A72C9E7000000040048CC
:108E700050000010FEE700000FB4054B10B503A929
:108E8000044A029800F064F910BC5DF814FB00007D
:108E9000319C0008C00200100FB41CB50A46521ED7
:108EA000CDE9000207A9054B6A46069800F050F983
:108EB000009A002111701CBC5DF814FB8598000815
:108EC0000FB4084B10B504A902AA039800F040F9AA
:108ED000044602A9002000F0E0FC204610BC5DF82A
:108EE00014FB00009B9800087CB5491E1C461546E3
:108EF000CDE90001044B6A462146284600F028F9D6
:108F0000009A002111707CBD859800080907090EA0
:108F1000002804DB00F1E02080F80014704700F026
:108F20000F0000F1E02080F8141D7047BFF34F8F51
:108F300005480168054A01F4E06111430160BFF38F
:108F40004F8F00BFFDE700000CED00E00400FA05C4
:108F5000BFF34F8F05480168054A01F4E0611143F2
:108F60000160BFF34F8F00BFFDE700000CED00E094
:108F70000400FA05004870475C0300200000000070
:108F800000B583B09FED0A0B0A4601468DED000B3C
:108F90006846F7F770FE9DED000B51EC100BF7F7EC
:108FA0004AFD03B000EE100A00BD00000000000002
:108FB000000000000000000002E008C8121F08C105
:108FC000002AFAD170477047002001E001C1121F4A
:108FD000002AFBD1704700002DE9FF5FDDE9022088
:108FE000010DDDF838B0024318D044F61050A1F25C
:108FF000FF3141430D140F98012820D0A5EB0B0041
:10900000401C5FEA000A4FF00004474EDFF81C9155
:10901000A046504616D5CAF1000728E00F98012453
:1090200043A2012808D0002100980F9BC0E900212D
:10903000C0E9024300F082B86FEA0B01F4E7CBF11C
:109040000000DEE7074612E0F80707D02246334665
:1090500040464946F7F7EBFB8046894622463346B1
:1090600010461946F7F7E3FB04460E467F10002F23
:10907000EAD1DDE90201BAF1000F42464B4602DABD
:10908000F7F7D5FB01E0F7F747FC04460E46002250
:10909000284BF7F7CFFE03D84FF0FF30014607E02B
:1090A0000022254B20463146F7F712FBF7F7AAFEC0
:1090B000102409E0002C0ADB0A220023F7F7F2F85B
:1090C000019B30321A55641E50EA0102F2D1641C31
:1090D000019AC4F1110314440F9A012A03D001220A
:1090E00008430DD10AE0084304D000204FF0110BD3
:1090F0000F9080E7A3EB0B056D1E0DE05B4504DDD3
:109100004FF0000205F1010504E003DA4FF0000220
:10911000A5F10105002AECD000980F99C0E90231B1
:10912000C0E9004586E70000000024400000F03F51
:10913000300000000000F0430000E03F3FBCBDE80D
:10914000C09F30380A2801D20120704700207047A4
:109150002DE9FF4F95B09B468946064600250FE254
:10916000252877D100242746F84A0121059400E0FC
:10917000044316F8013F203B01FA03F01042F7D1F7
:1091800030782A2811D06FF02F033078A0F1300208
:10919000092A16D8059A44F0020402EB820203EB76
:1091A00042021044761C0590EFE759F8042B059213
:1091B000002A03DA504244F40054059044F00204BB
:1091C000761C30782E2816D116F8010F44F00404CE
:1091D0002A280DD06FF02F023078A0F13003092B30
:1091E00009D807EB870302EB4303C718761CF3E7A4
:1091F00059F8047B761C30786C280FD006DC4C289C
:1092000017D068280DD06A2814D104E0742810D033
:109210007A280FD10DE044F400140AE044F48014DD
:1092200001E044F440147278824202D104F58014C3
:10923000761C761C307866280BD013DC582877D043
:1092400009DC002875D04528F6D04628F4D04728F8
:109250001AD19DE118E0632835D0642879D06528BB
:1092600012D195E1702873D008DC6728F1D0692805
:109270006FD06E280DD06F2806D1B5E073282CD0A2
:10928000752875D0782874D05A46179990476D1C68
:1092900075E1C4F30250022809D003280DD0D9F893
:1092A000001004280DD00D6009F1040967E1D9F818
:1092B0000010EA17C1E90052F6E7D9F800100D8056
:1092C000F2E70D70F0E719F8041B8DF8001000208C
:1092D0008DF80100EA46012003E059F804AB4FF095
:1092E000FF3061074FF0000102D40DE008F10101E9
:1092F0008846B9420FDA8045F8DB1AF808100029D1
:10930000F4D108E008F1010188468142FADB1AF83D
:1093100008100029F6D105985B46A0EB0807214606
:109320003846179A00F097FA284400EB080507E042
:109330004DE029E10DE01AF8010B5A4617999047C4
:10934000B8F10108F7D25B4621463846179A13E177
:1093500042E00A220092C4F302524FF0000A022AAD
:1093600008D059F804CB032A4FEAEC710AD00DE07B
:1093700029E02AE009F1070121F00702F2E802C121
:10938000914609E00FFA8CFC4FEAEC71042A03D1F4
:109390004FFA8CFC4FEAEC71002907DA0A460021EB
:1093A000DCF1000C61EB02012D2202E0220504D564
:1093B0002B228DF80420012203E0E20701D02022B5
:1093C000F7E7904659E00A2102E010220DE0102153
:1093D0004FF0000A00910BE010224FF0000A44F019
:1093E00004040827009203E008224FF0000A0092CC
:1093F000C4F30252022A05D059F804CB0021032AF3
:1094000008D009E009F1070121F00702F2E802C1E2
:10941000914605E01FFA8CFC042A01D10CF0FF0CE8
:109420004FF00008220728D5702806D0009B83F053
:10943000100353EA0A0305D00EE040228DF8042001
:10944000012208E05CEA010206D030228DF80420F7
:109450008DF8050002229046009B83F0080353EA32
:109460000A030AD15CEA010201D1620705D5302264
:109470008DF804204FF001087F1E582804D034A036
:1094800003900EA802900DE036A0F9E7534660461F
:10949000009AF6F707FF84460398825C0298401E04
:1094A000029002705CEA0100F0D1029806A9081A45
:1094B00000F1200A600702D524F4803400E001277F
:1094C000574502DDA7EB0A0000E0002000EB0A018F
:1094D000009005984144401A0590E00306D45B468D
:1094E0002146179A059800F0B6F90544002706E0D2
:1094F00001A85A46C05D179990476D1C7F1C4745CF
:10950000F6DBE0030CD55B462146179A059800F080
:10951000A2F9054404E030205A46179990476D1C83
:109520000099481E00900029F5DC08E00298029995
:109530005A460078491C0291179990476D1CBAF160
:109540000001AAF1010AF1DC65E10000092801002F
:1095500030313233343536373839616263646566A9
:10956000000000003031323334353637383941426B
:10957000434445460000000000F05BF90544761CBA
:10958000307800287FF4ECAD19B0284600F04EB9D1
:10959000620700D4062709F1070222F0070CFCE855
:1095A0000223E14603F000485FEA080C02D00FF204
:1095B000702C0DE05FEA045C02D50FF2682C07E026
:1095C0005FEAC47C02D00FF2602C01E0AFF2700CB5
:1095D0004FF0FF3823F00043CDF850C065280CD081
:1095E00006DC452809D046281DD047283DD13DE05E
:1095F000662818D067287ED138E00021112F01DBC2
:10960000112000E0781CCDE9000106A90EA8FFF7A3
:10961000E3FCDDE90F010E9A03910021009207F1AE
:10962000010A04914DE04FF000400097CDE9011090
:1096300006A90EA8FFF7D0FCDDE90F0203920E9BEE
:1096400011990022DDF80CA00093049211B9791C45
:1096500000EB010AB7EB0A0004D4C0F1FF3007F1B8
:10966000010A0490AAEB0700019044E0012F00DA00
:1096700001270021112F01DD112000E03846CDE93E
:10968000000106A90EA8FFF7A7FCDDE90F010E9A5D
:109690000391002104910092BA4621070CD403994A
:1096A000514500DA8A46BAF1010F05DD009AAAF1A8
:1096B0000101515C302908D0B84202DA10F1040FE0
:1096C00006DA0121CDE9011015E0AAF10101E9E76F
:1096D000002805DC049901440491AAEB000102E092
:1096E000411C514500DD8A460499401A401C0190F6
:1096F0004FF000400290200704D40198504501DB50
:10970000CDF8048000208DF84F0002980DF14F072E
:10971000B0F1004F25D02B200E9002984FF0020898
:1097200000280CDA404202902D200E9007E00A211A
:109730000298F7F79CF93031029007F8011DB8F153
:109740000001A8F10108F2DC02980028EFD1791E8F
:109750000E980870307800F0200040F0450007F8BF
:10976000020D12A8C01B00F107081498007800B180
:10977000012000EB0A01019801EBE07105984144DA
:10978000401A401E0590E00306D45B462146179A16
:10979000059800F060F805441498007818B15A460E
:1097A000179990476D1CE00324D55B462146179A14
:1097B000059800F050F805441CE00498002807DBE9
:1097C000DDE90301884203DD0098405C179901E060
:1097D000179930205A469047049805F10105401C1E
:1097E00004900198401E019004D12E205A461799EA
:1097F00090476D1CBAF10001AAF1010ADDDC05E019
:1098000017F8010B5A46179990476D1CB8F10001E3
:10981000A8F10108F4DC5B462146179A0598ABE6EF
:109820002D0000002B0000002000000030BCBDE82F
:10983000C08F2DE9F041044600251E4617468804D6
:1098400004D405E039462020B0476D1C641EF9D5CC
:109850002846BDE8F0812DE9F041044600251E466A
:109860009046C80301D5302700E02027880404D59E
:1098700005E041463846B0476D1C641EF9D52846C0
:10988000BDE8F0814A68002A06D00A68531C0B60C4
:1098900010704868401E486070470A68531C0B608F
:1098A00010707047104810B5D0F89400800001D5B2
:1098B0000EA000E012A0FFF7DFFA1648006B0228A6
:1098C00006D000280ED114A0BDE81040FFF7D4BA8E
:1098D00019A0FFF7D1FA1F48FBF754FF002801D168
:1098E0001DA0F1E710BD0000001002400D0A204944
:1098F0005744475F52535420666C61670000000074
:109900000D0A204E6F20495744475F52535420663A
:109910006C616700403200100D0A204E6F207661A6
:109920006C696420415050322E2052756E20415097
:1099300050310D0A000000000D0A2076616C696448
:1099400020415050322E2052756E20415050320D21
:109950000A000000004001080D0A204A756D7020C1
:109960006661696C65642E2052756E2041505031DD
:109970000000000010B50B4C2078002811D0F9F73A
:1099800061FE6169401A4EF66021884209D9064895
:10999000007810B105A0FFF76FFABDE8104002F0A3
:1099A000D1BE10BD1C000010000000105570677281
:1099B0006164652074696D656F75740D0A0000003F
:1099C00004490A68516A89B2536A5B1A8342FBD31D
:1099D00070470000D03C00202DE9FF4F8BB01E46A1
:1099E00093462DA1F6F7C2FC05464FF00009DFF8BB
:1099F000AC8035E0A81C82463D21F6F7D5FC044634
:109A000025A15046F6F7B2FC074698F8000020B1B1
:109A1000524623A00C99FFF72FFAE4B1DFB1BC4204
:109A200019D224216846F6F78AFCA4EB0A025146B3
:109A300068460992F6F7ACFC099A69460DF802905F
:109A400098F8000010B124A0FFF716FA68460C99A8
:109A5000F6F7BBFC50B110A1A81CF6F787FC054631
:109A6000002DC7D100200FB000F05AB83D1B6D1E6D
:109A7000B54200D3751E2A46611C5846F6F788FC8D
:109A80000BF8059098F80000594610B11AA0FFF79E
:109A9000F3F90120E7E70000232300000100001094
:109AA0005B657874726163745F6B765D205365618A
:109AB000726368696E67206B65792027257327209C
:109AC00066726F6D207365676D656E743A20252E22
:109AD0003332730A000000005B657874726163744E
:109AE0005F6B765D20466F756E64206B65793A20FA
:109AF000272573270A0000005B6578747261637420
:109B00005F6B765D204D617463686564206B657979
:109B1000212056616C75653A20272573270A0000BD
:109B200030BCBDE8C08F00002DE9F04194B00024A6
:109B30000F46804626466D46761CB6B239464046EC
:109B4000F8F7DEFB012804D1386845F82400641CCE
:109B5000A4B26420FFF734FF142C0FD2642EEBD391
:109B6000142C0BD21148007818B1214610A0FFF731
:109B700083F94FF0FF3014B0BDE8F081009C012163
:109B800023461A4655F82100984200DD03469042CC
:109B900000DA0246491C89B204441429F2D3E01ABF
:109BA000801A122190FBF1F0E5E7000000000010A0
:109BB00046444332323134206461746120726561FD
:109BC000642074696D656F757421204F6E6C792007
:109BD00025642073616D706C65732E0D0A000000A2
:109BE00010B586B0044672B61048F9F764FDF9F76F
:109BF0007DFB00200490A4F100640090E00A029034
:109C000001200390019004A96846F9F79FFA20B15A
:109C1000F9F70CFB002006B010BDF9F707FB03486D
:109C2000F9F749FD62B60120F5E700003027001082
:109C300013B54FF6FF73012269460248FBF7A6FCF5
:109C400000981CBD2828001010B5002821D0114B09
:109C50000022001F196803E0814203D80A464968C0
:109C60000029F9D152B11368841A9C4204D10068CA
:109C700018441060104602E0506000E0186039B1EE
:109C800002680B1A934203D10B681A4402604968B8
:109C9000416010BD58030020064951F8201040F2E1
:109CA000FF700A5CFF2A01D0401C7047401EF8D5A7
:109CB0000020704708DE000870B52DED068BB0EE71
:109CC000418AF0EE618AB0EE409AF0EE609A9FED24
:109CD0005F0B604C604DC8B3604E9FED61AB0128D7
:109CE00057D002287ED003287DD104F11001FFF760
:109CF0001BFF014620610320F8F7D0FA85ED060B23
:109D0000307868B153EC1A2B51EC100BF6F704FEC7
:109D100041EC100B54A053EC102B2169FFF7ACF869
:109D200051EC180BF6F787FE08EE100A51EC190BF0
:109D3000F6F781FE01EE100A95ED060BF0EE481ADB
:109D4000BDEC068BBDE87040F8F768BA41490020C9
:109D5000091DFFF7E9FE014660600020F8F79EFA52
:109D600085ED000BB0EE40AAF0EE60AA51EC180BA6
:109D7000F6F761FE08EE100A51EC190BF6F75BFEE0
:109D800001EE100AF0EE481AB0EE4A0AF0EE6A0A46
:109D9000D6E7304901200831FFF7C6FE0146A06032
:109DA0000120F8F77BFA85ED020B307868B153ECAF
:109DB0001A2B51EC100BF6F7AFFD41EC100B33A052
:109DC00053EC102BA168FFF757F851EC180BF6F77E
:109DD00032FE08EE100A51EC190BF6F72CFE01EEDC
:109DE000100A01E003E02DE095ED020BA6E719490A
:109DF00002200C31FFF798FE0146E0600220F8F7E0
:109E00004DFA85ED040B307868B153EC1A2B51EC08
:109E1000100BF6F781FD41EC100B25A053EC102B35
:109E2000E168FFF729F851EC180BF6F704FE08EE8D
:109E3000100A51EC190BF6F7FEFD01EE100A95ED34
:109E4000040B7BE7BDEC068B70BD0000000000003A
:109E500000000000AC02001038B500200000001027
:109E60000000000000408F404348332052415720FB
:109E70003D2025752C204672657175656E637920CD
:109E80003D20256C66204B487A0D0A00434831205E
:109E9000524157203D2025752C204672657175650D
:109EA0006E6379203D20256C66204B487A0D0A00B0
:109EB00043483220524157203D2025752C204672C0
:109EC000657175656E6379203D20256C66204B4871
:109ED0007A0D0A0010B5044608281AD80E48224602
:109EE0000EA144640220F7F7D7FE642000F048FF7B
:109EF0002046FDF7DFFB0CA42046F6F75FFA82B29E
:109F0000642321460E48FBF741FBFDF7E7F80120EB
:109F100010BD002010BD0000403200106261756469
:109F200072617465000000004E657720626175649F
:109F300072617465206170706C6965640D0A00005F
:109F40002828001070B5054618A6A0B03046F6F7D0
:109F500035FA04462DB1024631462846F6F763FA33
:109F600008B115A01FE025442846F6F727FA98B156
:109F700080216846F6F7E3F9002480236A462946E3
:109F8000204601F007FC48B16B462A46214614A042
:109F9000FEF772FF20B070BD18A004E0641CE4B2AC
:109FA000032CEAD31CA0FEF767FFF3E72D2D6366B1
:109FB000675F6765743D00006572726F723D696E20
:109FC00076616C6964206366675F67657420666F9D
:109FD000726D61742C20726C743D3432300D0A0045
:109FE00066696C6569643D25642C205B25733D259D
:109FF000735D2C206F6B0D0A000000006572726F9C
:10A00000723D656D707479206B65792C20726C746B
:10A010003D3432310D0A0000726C743D3430342C02
:10A02000206572726F723D6E6F742065786973740B
:10A030002E0D0A0000B5B3B000218DF8C8108022A3
:10A0400002A9CDE90012402322AA32A901F0E4FAC4
:10A0500020B108A0FEF710FF33B000BD02AA22A96C
:10A060009DF8C80000F01AF802A922A802F018FC16
:10A07000F2E700006572726F723D696E76616C691D
:10A0800064206366675F73657420666F726D6174C8
:10A090002C20726C743D3431300D0A0070B590B0D4
:10A0A0000E4604461546032804D311A0FEF7E4FE2D
:10A0B00010B070BD1046F6F781F988B140216846AE
:10A0C000F6F73DF940236A463146204601F062FB2F
:10A0D00000282A463146204607D0FBF771FCE7E707
:10A0E00031462046FBF7BCFBE2E7FBF705FCDFE768
:10A0F0006572726F723D696E76616C69642064622C
:10A100002069642C20726C743D3431310D0A0000DA
:10A1100000B5B3B0802202A9CDE90012402322AAE3
:10A1200032A901F0C1FA20B107A0FEF7A5FE33B0B5
:10A1300000BD02AA22A99DF8C800FFF7AFFF02A93F
:10A1400022A802F0ADFBF2E76572726F723D696E94
:10A1500076616C6964206366675F736574782066F6
:10A160006F726D61742C20726C743D3431300D0A45
:10A170000000000070B5054611A63046F6F71EF93E
:10A1800004462DB1024631462846F6F74CF908B18F
:10A190000FA010E02819F6F78EFAC0B2032801D3F9
:10A1A00017A008E01E4951F82000FFF719FD08B17B
:10A1B0001CA000E01DA0BDE87040FEF75DBE0000E1
:10A1C0002D2D636C6561725F66696C6569643D0025
:10A1D0006572726F723D696E76616C696420636C42
:10A1E0006561725F66696C65696420666F726D6136
:10A1F000742C20726C743D3434300D0A0000000061
:10A200006572726F723D696E76616C69642064621A
:10A210002069642C20726C743D3434310D0A0000C6
:10A2200008DE00086F6B0D0A000000006572726F97
:10A23000723D6572617365206661696C2C20726C79
:10A24000743D3434320D0A007CB5A0F5AA41AA3918
:10A2500001D000207CBD1B4C0025012225631AA1E2
:10A260000220A263F7F718FD1AA10220226BF7F76C
:10A2700013FD642000F084FD00950195607B8DF84E
:10A28000000006218DF8011040208DF802004220C8
:10A290008DF8030055208DF80400AA208DF80500E4
:10A2A000684600F054FD8DF80600000A8DF807009E
:10A2B0000821684602F09AFB642000F061FDFEF779
:10A2C00047FE00004032001075626F6F7462616378
:10A2D0006B0000006961704C6F6164537461747548
:10A2E000730000007CB5054625A63046F6F766F8F3
:10A2F00004462DB1024631462846F6F794F808B1D7
:10A3000022A039E000208DF800000190281901AB4F
:10A310006A4628A1F6F796F8022801D027A02BE07C
:10A320009DF80000032801D32EA025E0354951F8FF
:10A330002040FFF7B1FC064684B17EB102469DF88D
:10A34000001031A0FEF798FD214637A0019AFEF7D4
:10A3500093FD3CA0FEF790FD00250AE03AA00BE03B
:10A36000605DA0F120015E2902D83E4902F0B9F8F3
:10A370006D1CB542F4D33CA0FEF77EFD7CBD000011
:10A380002D2D66696C6569643D0000006572726F11
:10A39000723D696E76616C69642066696C6569649A
:10A3A00020666F726D61742C20726C743D34333092
:10A3B0000D0A0000256868752C2564006572726FAF
:10A3C000723D696E76616C69642066696C6569646A
:10A3D00020706172616D732C20726C743D34333166
:10A3E0000D0A00006572726F723D696E76616C696C
:10A3F000642064622069642C20726C743D343332B2
:10A400000D0A000008DE000844425F44554D502C00
:10A410002066696C6569643D25642C206C656E3D21
:10A4200025752C0D0A000000616464723D307825AA
:10A430003038582B25642C636F6E74656E743D0D37
:10A440000A0000005B0000006572726F723D656D6E
:10A450007074792064622C20726C743D3433330D37
:10A460000A000000C00200105D2C206F6B0D0A0076
:10A47000006808600120704770B506461BA5A0B0B3
:10A480002846F5F79BFF0446024629463046F5F775
:10A49000CAFF08B118A00EE0301904462221F5F7D2
:10A4A00083FF05000BD080216846F5F748FF2D1B80
:10A4B000802D06D316A0FEF7DFFC20B070BD1AA0D9
:10A4C000F9E721462A466846F5F762FF00240DF8B1
:10A4D00005406A461BA12046FFF7E0FD0C226946B5
:10A4E0001948F5F755FF18480473E6E77B226D61BC
:10A4F00063223A22000000006572726F723D696E3D
:10A5000076616C6964206D616320636D640D0A007F
:10A510006572726F723D6D616320746F6F206C6F36
:10A520006E670D0A000000006572726F723D696E01
:10A5300076616C6964206D616320666F726D617411
:10A540000D0A00006D616300403200101CB5012847
:10A550004FF0000023D1124900900190497B8DF803
:10A56000001006218DF8011040228DF8040001230F
:10A570008DF802208DF803208DF80530684600F034
:10A58000E6FB8DF80600000A8DF8070008216846F2
:10A5900002F02CFA322000F0F3FBFEF7D9FC1CBDD0
:10A5A00040320010C2B2044810B5427303A1022029
:10A5B000F7F772FB012010BD403200106164647235
:10A5C00000000000084940B1922805D0952807D026
:10A5D000982807D00020704701200870012070479C
:10A5E0000220FAE70320F8E75401002070B51C4C64
:10A5F00005464AF6BB262078B8B1A88844F2010186
:10A6000040BA88422BD1F9F71DF86061E8882169CA
:10A6100040BA88420CD0002304223146422002F086
:10A62000A3F8BDE8704002F08DB80023082210E0C6
:10A630000C4BA068202205F108011844F8F7BEFB76
:10A64000A06800F58070A0602069401C83B20022E1
:10A6500020613146BDE87040422002F085B870BDEF
:10A660001C000010008002082DE9F04700234AF684
:10A67000BB2A9AB01A465146422002F0A9F8704D02
:10A68000DFF8C091704CA88816AEB0F5807F03D07B
:10A69000B0F5007F58D096E06846FBF743FAEA68C9
:10A6A00049466846103AFBF7BFFD694616A8FBF716
:10A6B00011FA644BE868103B102264491844F8F71B
:10A6C0006DFB207810B162A0FEF7D6FB0025207844
:10A6D00018B1715D61A0FEF7CFFB2807B0F1704F94
:10A6E00004D1207810B15FA0FEF7C6FB6D1C102DC1
:10A6F000EDDB207810B15BA0FEF7BEFB2078A04612
:10A7000010B159A0FEF7B8FB504F002598F8000093
:10A7100018B1795D51A0FEF7AFFB2807B0F1704F7B
:10A7200005D198F8000010B14EA0FEF7A5FB6D1CF6
:10A73000ADB2102DEAD398F8000010B149A0FEF791
:10A740009BFB102241493AE06846FBF7EBF949468A
:10A750006846EA68FBF768FD694616A8FBF7BAF990
:10A76000207810B145A0FEF787FB354F002518373C
:10A77000207818B1795D39A0FEF77EFB6D1CADB273
:10A78000042DF5D3207810B136A0FEF775FB2078A4
:10A7900010B13FA0FEF770FB0025207818B1715D65
:10A7A0002EA0FEF769FB6D1CADB2042DF5D3207809
:10A7B00010B12CA0FEF760FB21490422183116A825
:10A7C000F5F71BFEA0B1207810B139A0FEF754FBBD
:10A7D0004FF4A0414846F8F79DFA00230522514660
:10A7E000422001F0F5FF01F0ADFF1AB0BDE8F0879F
:10A7F000207810B13BA0FEF73FFB144D4FF496724A
:10A80000583D3EA102202A63F7F746FA002405EBE3
:10A810004400325D3DA12430FEF752FB641C042C41
:10A82000F5DB0020094A85F82C00343A39A10220D2
:10A83000F7F71EFA4FF4FA7000F0A2FAFEF776FB73
:10A840001C00001000800208000000109832001068
:10A85000726573756C745F6D64353A002025303213
:10A86000580000000A000000657870656374656434
:10A870005F6D64355F303130303A00006578706567
:10A88000637465645F6D64355F303230303A200048
:10A89000726573756C745F6D6435202866697273B8
:10A8A000742034206279746573293A200000000016
:10A8B000204D443520636865636B206661696C7365
:10A8C0002C20457261736520494150446174614296
:10A8D00075666665725F4144445220466C617368D8
:10A8E000200D0A00204D443520636865636B20709D
:10A8F0006173736564200D0A000000006961704C8B
:10A900006F616453746174757300000025303258B0
:10A91000000000006961706D643500002DE9F047AA
:10A92000534C0746207810B152A0FEF7A5FA2078C4
:10A9300010B159A0FEF7A0FA207810B15CA0FEF784
:10A940009BFAF8885E4D40BAA880F8F77BFE6861F4
:10A95000A888DFF8708101264AF6BB29B0F5807F10
:10A960000AD0B0F5007F3BD0002306224946BDE85F
:10A97000F047422001F060BF207810B152A0FEF7EE
:10A980007BFAD7F8170000BA20F0FF01B87E014328
:10A99000E960207810B151A0FEF76EFAE868B0F5D2
:10A9A000A03F02D900230222E0E700206E70A860D9
:10A9B00028612E7003460246AE704946422001F0DF
:10A9C0003BFF88F80060207810B14CA0FEF754FAE5
:10A9D0002078002849D0BDE8F0474CA0FEF74CBADB
:10A9E000207810B151A0FEF747FAB86800BA20F0FD
:10A9F000FF01F87A0143E960F868A861AE70207839
:10AA000010B136A0FEF738FA207810B14CA0FEF74E
:10AA100033FA2B4F00251837207818B1795D4DA0F7
:10AA2000FEF72AFAA807B0F1404F04D1207810B100
:10AA300029A0FEF721FA6D1C042DEDDB207810B162
:10AA400025A0FEF719FA207810B130A0FEF714FA0D
:10AA500000231A464946422001F0EEFE4FF4A04181
:10AA60003E48F8F757F988F80060BDE8F087000025
:10AA7000000000100D0A3D3D3D3D3D3D3D3D3D3D4D
:10AA80003D3D3D3D3D3D3D3D3D3D3D3D3D3D3D3DF6
:10AA90003D3D0D0A000000003D3D3D2055706772B0
:10AAA000616465207374617274203D3D3D0D0A0040
:10AAB0003078343030302073746172740D0A0000C5
:10AAC0001C00001004000020737562636F64653A17
:10AAD000203078303130300D0A0000006578706524
:10AAE000637465645F66696C655F73697A655B3022
:10AAF00078253034785D0D0A00000000307834305D
:10AB0000303020656E640D0A000000003D3D3D3D83
:10AB10003D3D3D3D3D3D3D3D3D3D3D3D3D3D3D3D65
:10AB20003D3D3D3D3D3D3D3D0D0A00007375626379
:10AB30006F64653A203078303230300D0A00000002
:10AB400065787065637465645F6D64355F3032305D
:10AB5000303A000020253032580000000080020802
:10AB60001CB50E4A0178527B914201D0FF2910D1C9
:10AB7000417803290DD1C188ADF80010062100F0FD
:10AB8000E6F8ADF80400022201A96846F5F735FCA5
:10AB900008B100201CBD01201CBD00004032001087
:10ABA0001CB50E4A0178527B914201D0FF2910D189
:10ABB000417806290DD1C188ADF80010062100F0BA
:10ABC000C6F8ADF80400022201A96846F5F715FCA5
:10ABD00008B100201CBD01201CBD00004032001047
:10ABE00010B50C4A0178527B914201D0FF290DD15A
:10ABF000417810290AD1084909684218891E32F89B
:10AC0000024C89B200F0A3F8844201D0002010BDAC
:10AC1000012010BD40320010AC00002010B50F4ADA
:10AC20000178527B914215D1FF2913D141784229F5
:10AC300010D18178AA290DD1C178BB290AD1084940
:10AC400009684218891E32F8024C89B200F07FF878
:10AC5000844201D0002010BD012010BD4032001000
:10AC6000AC000020F8F736FDFCF7D1FDFBF7F2FB56
:10AC7000FBF724FBFBF7D0FCFBF798FCFBF756FC3B
:10AC8000FBF76CFCFBF7E6FC0648F9F7C1FFF7F7AA
:10AC900087F8FEF707FE00F081F8FBF73DFB00F0B8
:10ACA0008FF8FEE7D03C0020F0B50B30154D20F0BA
:10ACB00007010024144A0FE003688B420BD38B4238
:10ACC00005D95E1A43184768C3E9006700E0436886
:10ACD000136002C004E0021D10680028ECD1204679
:10ACE000002802D1286808B10020F0BD064A0748B4
:10ACF0001060074A121A22F00702C0E9002401205E
:10AD00002860D7E7C4020010580300205CB500207B
:10AD1000A8B700202DE9F0411D469046060011D04D
:10AD2000B8F1000F0ED06DB1A9420BD300244F1B18
:10AD300006E030192A464146F5F75FFB28B1641C4E
:10AD4000A742F6D20020BDE8F0813019FBE770B5CC
:10AD500004464FF6FF7000224AF201050DE0A35CA5
:10AD600058400023C60702D085EA500000E04008A2
:10AD70005B1C082BF6DB521C92B28A42EFD370BDEB
:10AD800010B5EFF3058111B16FF0050403E0002465
:10AD900008B101F0A5FF204610BD0000EFF30580CB
:10ADA00010B16FF0050070470448016811B14FF011
:10ADB000FF3070470121016000207047180000102B
:10ADC00010B5EFF3058010B16FF0050010BD084815
:10ADD0000168012902D04FF0FF3010BD054A002163
:10ADE00082F8141D0221016001F0E2FF002010BD75
:10ADF000180000100BE000E070B50546EFF3058089
:10AE000010B16FF0050407E045B1284601F032FFAC
:10AE10000024284601F016FF204670BD6FF00304A1
:10AE2000FAE70000F8B51D466FF003026FF0020666
:10AE30004FF00004EFF30583A3B1F0B1E9B1E5B938
:10AE4000002200926A4602F005FB012817D1009803
:10AE5000B0B10C494FF080500860BFF34F8FBFF383
:10AE60006F8F0DE048B141B12A4602F057FA012830
:10AE700006D025B16FF0010402E0144600E034462C
:10AE80002046F8BD04ED00E0F8B514464FF000058B
:10AE9000EFF3058212BB08B301B3A4B1D4E90232C7
:10AEA00063B1502A1AD32269C2B1676900FB01F667
:10AEB000B74213D3009502F0AAF807E072B92269ED
:10AEC00062B9626952B9002202F080F8050005D02B
:10AED0000CB1216800E0002101F0A0FE2846F8BD79
:10AEE000F8B51D466FF003026FF002064FF0000444
:10AEF000EFF30583ABB100B3F9B1F5B90022134606
:10AF000000926A4602F0AAF9012818D10098B8B157
:10AF10000C494FF080500860BFF34F8FBFF36F8F25
:10AF20000EE050B149B100232A4602F0E7F80128AB
:10AF300006D025B16FF0010402E0144600E034466B
:10AF40002046F8BD04ED00E02DE9FF410B464FF02F
:10AF50000005EFF30581039549BB40B38027182115
:10AF600000244AB3166806B1344696691EB13146CC
:10AF7000761E382E02D21679F60703D0002004B0D0
:10AF8000BDE8F081566906B1B708D2F808C0BCF137
:10AF9000000F0DD0D5685C2D18D312693AB136B1C7
:10AFA0008DE806103A46214602F00CFB03900DE0B6
:10AFB000D6685EB912694AB903AACDE90012BAB2DD
:10AFC000214602F0CFFA012800D003950398D6E776
:10AFD00070B504007ED0207800287BD02046F5F79D
:10AFE000EDF90546052805D30522AEA12046F5F763
:10AFF0001AFA08B1ADA07FE0601910F8021C0D2903
:10B0000003D110F8011C0A2901D0B0A074E000217E
:10B0100000F8021C641D0822B4A12046F5F703FACB
:10B0200000286DD0B4A12046F5F7CFF900287ED0D6
:10B030000822B2A12046F5F7F6F900287BD00B22B2
:10B04000B1A12046F5F7EFF9002879D00A22B1A185
:10B050002046F5F7E8F9002877D00B22B0A120466A
:10B06000F5F7E1F9002875D00A22B0A12046F5F7DE
:10B07000DAF9002873D0B0A12046F5F7A6F9002828
:10B0800072D00922AEA12046F5F7CDF900287FD075
:10B090000F22AEA12046F5F7C6F900287DD00A227E
:10B0A000AEA12046F5F7BFF900287BD00C22AEA157
:10B0B0002046F5F7B8F9002869D00F22AEA1204646
:10B0C000F5F7B1F900287BD00D22AFA12046F5F7A6
:10B0D000AAF900E073E0002873D00D22AEA120464B
:10B0E000F5F7A1F900286DD00422AFA12046F5F7AD
:10B0F0009AF9002867D0AEA0BDE87040FDF7BCBE4D
:10B1000004F10800F5F7D7FA0246B0F5B46F0CD891
:10B11000002A04DDAFA103E009E00CE010E0AFA1DC
:10B12000BDE87040B0A0FDF7A7BEB9A0E4E7BDE858
:10B13000704000F087BB2046BDE87040FFF79CB927
:10B14000B9A0D9E701E005E009E02046BDE870407C
:10B15000FEF770BF2046BDE87040FEF7D9BF20461D
:10B16000BDE87040FEF7EEBEB4A0FDF785FEBFF36C
:10B170004F8FB4480168B44A01F4E06111430160A3
:10B18000BFF34F8F00BFFDE702E006E00AE01DE0DD
:10B190002046BDE87040FFF7A5B82046BDE87040E6
:10B1A000FEF7E8BFA94CD4F8940080000CD5A8A005
:10B1B000FDF762FE54F8940F40F40000206070BD6B
:10B1C00008E01AE02CE041E0A6A095E7BDE8704059
:10B1D000FBF74CBDE17B302903D0312903D0A6A079
:10B1E00030E0002100E00121AB480170007808B197
:10B1F00078A100E079A1A9A024E0617B302903D0E7
:10B20000312903D0AAA01DE0002100E00121B048AF
:10B210000170007808B16FA100E070A1ADA011E04D
:10B22000617B302903D0312903D0AEA00AE0002190
:10B2300000E00121B3480170007808B165A100E089
:10B2400066A1B1A0BDE87040FDF716BEB2A0F6F74A
:10B2500039FBB4A0F6F736FBB4A0F6F733FBB7A082
:10B26000F6F730FBBCA0F6F72DFBC3A0F6F72AFBE0
:10B27000C6A0F6F727FBC8A0F6F724FBCAA0F6F78E
:10B2800021FBCEA0F6F71EFBD0A0F6F71BFBD3A048
:10B29000F6F718FBD6A0F6F715FBBDE87040D9A06D
:10B2A000F6F710BB2323233A3A0000006572726F51
:10B2B000723D696E76616C6964207072656669784A
:10B2C0002C20726C743D3430310D0A006572726F3F
:10B2D000723D696E76616C696420656E64696E6743
:10B2E0002C20726C743D3430320D0A002D2D6465B3
:10B2F0006275673D000000006C7300007B226D6189
:10B3000063223A22000000002D2D7365745F74697A
:10B310006D653D002D2D6366675F7365743D0000AC
:10B320002D2D6366675F736574783D002D2D636610
:10B33000675F6765743D00007265626F6F7400003F
:10B340002D2D66696C6569643D0000002D2D636CD0
:10B350006561725F66696C6569643D002D2D697772
:10B3600064675F67657400002D2D537461636B5FC4
:10B3700073697A65000000002D2D64656275675F52
:10B380007072696E74663D002D2D6664635F707225
:10B39000696E74663D0000002D2D6164735F7072EC
:10B3A000696E74663D00000068656C700000000006
:10B3B0006572726F723D756E6B6E6F776E20636F24
:10B3C0006D6D616E642C20726C743D3430390D0AE1
:10B3D00000000000656E61626C6564006469736101
:10B3E000626C656400000000446562756720636FED
:10B3F0006E736F6C652025732C2074696D656F7595
:10B40000743D2564206D696E0D0A2C204F4B0000A1
:10B41000496E76616C696420646562756720746941
:10B420006D650D0A000000006E6F20727463207459
:10B43000696D652C206F6B0D0A0000006F6B0D0AA3
:10B44000000000000CED00E00400FA0500100240CE
:10B450000D0A20495744475F52535420666C616778
:10B46000000000000D0A204E6F20495744475F52EC
:10B47000535420666C616700496E76616C69642084
:10B4800064656275677072696E74662076616C754A
:10B49000653A2025630D0A000000001044656275BE
:10B4A00067207072696E742025730D0A0000000019
:10B4B000496E76616C6964206664637072696E744B
:10B4C000662076616C75653A2025630D0A000000E0
:10B4D00001000020464443207072696E7420257379
:10B4E0000D0A0000496E76616C69642061647370B6
:10B4F00072696E74662076616C75653A2025630DFD
:10B500000A00000002000020414453207072696E5E
:10B51000742025730D0A00002D2D64656275673D4A
:10B52000580D0A006C730D0A000000007B226D614B
:10B5300063223A2258227D0D0A0000002D2D6366F9
:10B54000675F7365743D247B6B6579317D3D247B3A
:10B5500076616C317D0D0A002D2D6366675F736522
:10B5600074783D582C247B6B65797D3D247B766116
:10B570006C7D0D0A000000002D2D6366675F676516
:10B58000743D247B6B65797D0D0A00007265626FE6
:10B590006F740D0A000000002D2D66696C656964EA
:10B5A0003D582C300D0A00002D2D636C6561725FD3
:10B5B00066696C6569643D580D0A00002D2D697738
:10B5C00064675F6765740D0A000000002D2D5374D9
:10B5D00061636B5F73697A650D0A00002D2D6465E8
:10B5E0006275675F7072696E74663D580D0A00007F
:10B5F0002D2D6664635F7072696E74663D580D0A26
:10B60000000000002D2D6164735F7072696E7466B6
:10B610003D580D0A000000002DE9F05F9B461746DB
:10B620000D4606004FF0FF392AD04DB347B30A98B4
:10B6300030B318A42046F4F7C1FE824602462146E4
:10B640003046F4F7F0FED8B94FF00008564485F8BC
:10B6500000803D213046F4F7A7FE040010D0A51B62
:10B660005D450DD22A4631463846F4F791FE641CFA
:10B6700007F805802046F4F7A1FE0B99884202D313
:10B68000484600F00DB821460A98F4F7C3FE0020A2
:10B69000F7E700002D2D6366675F7365743D00005A
:10B6A00030BCBDE8C09F00002DE9F05F9A46DDF890
:10B6B00028B016460D4607004FF0FF3939D0C5B304
:10B6C000BEB35FEA0B0034D01EA42046F4F776FE2A
:10B6D0008046024621463846F4F7A5FE48BB47445B
:10B6E0002C213846F4F760FE040022D04FF0000809
:10B6F00084F800803846F4F7DEFF28702C2004F828
:10B70000010B25463D212046F4F74EFE040010D0E3
:10B71000671B57450DD23A4629463046F4F738FEA6
:10B72000641C06F807802046F4F748FE0B9988420F
:10B7300002D3484600F00CB821465846F4F76AFE9A
:10B740000020F7E72D2D6366675F736574783D0011
:10B7500030BCBDE8C09F70B590B014460D4606469B
:10B76000032814D29DB194B140216846F4F7E7FD57
:10B7700040236A462946304600F00CF8002804D0E1
:10B780006846F4F798FF2060012010B070BD0020DB
:10B79000FBE700002DE9F041984614460D460646A9
:10B7A00003281CD2DDB1D4B14FF4006739460E48EE
:10B7B000F4F7C5FD3A460C493046F6F7B7F80146AE
:10B7C0000A48007810B10AA0FDF756FB434622460E
:10B7D00029460548FEF700F9C0B2BDE8F0810FA088
:10B7E000FDF74AFB0020F8E7149500200100001047
:10B7F0005B7069636B75705F737472696E675F66A7
:10B80000726F6D5F6B65795D2044756D7065642046
:10B810006C656E3A2025750A000000005B70696354
:10B820006B75705F737472696E675F66726F6D5F60
:10B830006B65795D20496E76616C696420696E7014
:10B8400075740A002DE9F0477F488EB000F1400181
:10B8500009AD1EC985E81E00D0E90E3405AD016BA7
:10B86000828E85E81E0000F1180200F124011CCA36
:10B87000CDE90341CDE9012341690091427B0146B5
:10B8800003697248F6F71EF871A0F6F71BF8764CBC
:10B89000002500BF54F82500F5F7BAF841EC100B6D
:10B8A000062D01DA71A000E071A0009053EC102B7E
:10B8B00070A0F6F707F86D1C072DEBDB6FA0F6F70D
:10B8C00001F8002504EB8500C069F5F7A1F841EC0B
:10B8D000100B0A2D01DA65A000E065A0009053EC82
:10B8E000102B64A0F5F7EEFF6D1C0B2DEADB6BA0AF
:10B8F000F5F7E8FF5FF0000504EB8500806CF5F7D5
:10B9000087F841EC100B052D01DA58A000E058A093
:10B91000009053EC102B57A0F5F7D4FF6D1C062DAB
:10B92000EADB67A0F5F7CEFF5FF0000504EB8500CA
:10B93000006EF5F76DF841EC100B052D01DA4BA008
:10B9400000E04BA0009053EC102B4AA0F5F7BAFF93
:10B950006D1C062DEADBD4F890007834F5F758F822
:10B96000074688466069F5F753F805460E46206994
:10B97000F5F74EF8CDE90201E068F5F749F88146A0
:10B980008A466068F5F744F8CDE900012068F5F7CC
:10B990003FF841EC100B208953EC102BCDE90980C6
:10B9A00006A880E8E000DDE90201CDE9029ACDE9D0
:10B9B00004014C48F5F786FF606BF5F729F8074658
:10B9C0008846206BF5F724F8CDE90201E06AF5F727
:10B9D0001FF881468A46A06AF5F71AF805460E4612
:10B9E000606AF5F715F8CDE90001206AF5F710F85F
:10B9F00041EC100B608F218FCDE90A10CDE908785A
:10BA0000DDE90201CDE9060102A953EC102B81E822
:10BA100060063548F5F756FF206CF4F7F9FF054648
:10BA20000E46E06BF4F7F4FF41EC100BB4F8440061
:10BA30000095CDE9016053EC102B2CA0F5F742FFE7
:10BA40000EB0BDE8F08700004032001050E700085B
:10BA50005B63616C69625F726F642E766F6C5F7698
:10BA6000616C7565735D3D00A83200102C0000000C
:10BA70000A000000252E3366257300005B63616CAD
:10BA800069625F6F696C5F77617465722E63617064
:10BA90005F76616C7565735D3D0000005B63616C92
:10BAA00069625F726573696475616C5F6F696C2E42
:10BAB0006361705F76616C7565735D3D00000000C9
:10BAC0005B63616C69625F726573696475616C5F09
:10BAD0006F696C2E766F6C5F76616C7565735D3D1A
:10BAE0000000000020E60008A4E6000874656D7000
:10BAF0005F766F6C5F6F66667365743D252E336687
:10BB00002C2074656D705F6469616C6F673D252ED4
:10BB100033662C2074656D705F636F6C74696D653E
:10BB20003D25640A0000000038B50546A0211948EB
:10BB3000F4F705FC68886979164C6A7840BA0029E0
:10BB400027D07D2925D8144B5B7B237062704A0077
:10BB5000A2700022ADF800206B46E21C00F048FD08
:10BB6000002816D0BDF80000C01C81B22046FFF7A7
:10BB7000EEF8BDF800102144C870BDF80010000AAE
:10BB800021440871BDF80000401D81B2204600F03C
:10BB90002DFF38BD74840020403200102DE9F041A3
:10BBA0000646A0211A48F4F7CAFB70881A4A45BA1B
:10BBB000B088777846BA164C00201649126822E001
:10BBC00031F83030AB421DD101EBC0004168304646
:10BBD0008847002819D011480621407B20706770E3
:10BBE000280AA070E570300A207166712046FFF7C0
:10BBF000AEF8A071000AE0712046BDE8F0410821CE
:10BC000000F0F4BE401C9042DAD3BDE8F0810000A1
:10BC100074840020640000108C000010403200107A
:10BC20002DE9F0470746A0212948F4F788FB7888DA
:10BC3000274C46BAB88897F8019045BA6800FFF7D4
:10BC400033F88046002008E007EB4001B1F8071008
:10BC500049BA28F81010401C80B2A842F4D31E4AFA
:10BC600000201C4912682BE000EB400331F82370E0
:10BC7000B74224D101EB83035B88AB421FD100EBB9
:10BC8000400001EB8000D0E9012140469047C8B157
:10BC900012480621407B207084F80190300AA07081
:10BCA000E670280A207165712046FFF750F8A071F0
:10BCB000000AE0710821204600F098FE02E0401CD6
:10BCC0009042D1D34046BDE8F047FDF7BDBF00002C
:10BCD00074840020900000104003002040320010C7
:10BCE00010B50446A0211248F4F729FBA08841BAF8
:10BCF000B1F5804F0ED06FF4804008180FD00128A6
:10BD000012D000230722BDE810404AF6BB21422092
:10BD100000F05EBD2046BDE81040FEF7FFBD2046A6
:10BD2000BDE81040FEF762BCBDE81040FEF79CBCC9
:10BD3000748400202DE9F041134C0F460546E66857
:10BD40002068001D00F064FE681C07D137B121682F
:10BD5000BDE8F0410D48091D00F0B2BE2068354431
:10BD6000B5424560216805D2A06BBDE8F041091DD0
:10BD700000F08EBE606B091D00F08AFEA06A85424D
:10BD800000D2A562BDE8F081D40000201C43002051
:10BD90002DE9F041054600F09FFE2D4CA068401CA7
:10BDA000A06020682B4F10B1606930B32BE0256094
:10BDB000A068012827D1002606EB860007EB80004B
:10BDC00000F058FE761C382EF6D3234800F052FEC1
:10BDD0002148143000F04EFE1F48283000F04AFE83
:10BDE0001D483C3000F046FE1B48503000F042FE3B
:10BDF000194860631430A06305E02068E96AC06AEE
:10BE0000884200D82560606A401C60626864E86A05
:10BE10002169884200D9206100EB800007EB800097
:10BE2000291D00F04DFE00F077FE606900280CD05F
:10BE30002068E96AC06A884207D208494FF08050FA
:10BE40000860BFF34F8FBFF36F8FBDE8F081000034
:10BE5000D40000206C3E0020CC42002004ED00E025
:10BE600038B500F039FE104C2068C8B90F4800F012
:10BE700001FE0E48143000F0FDFD0C48E060143067
:10BE800020610A4B0020F03B009003F1500210218A
:10BE90000A2001F0BCF8206010B105A100F0BEFE40
:10BEA000BDE8384000F038BE1001002020440020DA
:10BEB000546D72510000000030B4026C0B46002A31
:10BEC0000BD0C1681144C1608468A14201D30168EC
:10BED000C16030BC1846F4F719BA30BC70472DE980
:10BEE000F041856B174604460026026C82B1C7B14B
:10BEF000E068F4F70BFAE168206C091AE160226847
:10BF0000914202D2A168081AE060022F16D017E011
:10BF10002068A8B9A06801F0F9FB06460020A060DF
:10BF20000EE06068F4F7F2F9216C60680844606024
:10BF3000A168884204D32068606001E005B16D1EED
:10BF40006D1CA5633046BDE8F08110B5044690F83D
:10BF5000590058B101280CD002280FD0502080F38E
:10BF60001188BFF34F8FBFF36F8FFEE7206B00F098
:10BF7000E7FD2046BDE8104000F0E2BD10BD000026
:10BF800010484FF48041420706D0C01D0D4920F0F3
:10BF90000700411AC1F580410B4A00230144C2E960
:10BFA00000030839183A21F0070111604B600B605B
:10BFB0000B1AC0E9001393604FF0004053605061CA
:10BFC00070470000484400203C010020144E154CEE
:10BFD000A6F29C474FF08058DFF84C9012E000BF6B
:10BFE00000F07AFDF068C568281D00F011FDA0681A
:10BFF000401EA0606068401E606000F08DFD284615
:10C00000FFF7A3FF60680028EAD138680128F9D952
:10C01000C9F80080BFF34F8FBFF36F8FF2E70000C6
:10C0200008430020D400002004ED00E070B51D4658
:10C03000049C51B1C4F80020C4E90F01012120463D
:10C0400001F018F884F84C5070BD2460F4E700004B
:10C050002DE9F05F8846DDE90B9415468346910093
:10C060009A460A9EA522206BF4F762F96FF003014D
:10C07000206B01EB8501084420F00707780707D003
:10C08000502080F31188BFF34F8FBFF36F8FFEE70F
:10C090000025B8F1000F0FD05FF00000221818F84B
:10C0A000001082F8341018F8001011B1401C10284C
:10C0B000F4D384F8435001E084F83450382E00D390
:10C0C0003726E662C4E91365201D00F0DEFC04F1AA
:10C0D000180000F0DAFC2461C6F138006462A06147
:10C0E000656584F8585052465946384600F06AFA59
:10C0F0002060B9F1000F01D0C9F8004000F000B88D
:10C1000030BCBDE8C09F000030B5114900E01146C9
:10C110000A688242FBD34B685C18844203D14068B2
:10C1200018444860084643681C18944209D1084CDA
:10C13000183C2468A24209D052681A4442600A6836
:10C1400012680260814200D0086030BD0460F9E7E7
:10C150003C01002070B5002441600B4D006191420C
:10C1600006D8D11A8269914206D2011D286907E0DA
:10C170009A4203D2994201D3012403E0011DE868E9
:10C1800000F086FC204670BD1001002010B504466A
:10C1900000F0A2FCA06B28B15FF0000400F0BCFC32
:10C1A000204610BD0124F9E730B589B03C4D6EE062
:10C1B0000498002806DADDE90601059A90470498FC
:10C1C000002864DB069C606910B1201D00F020FC93
:10C1D00003A800F0D7F8024604980A2857D2DFE8EF
:10C1E00000F00505052D334A05052D3394F8280088
:10C1F00040F0010084F828000599A069059B0144DE
:10C200002046FFF7A7FF68B3216A2046884794F8C5
:10C21000280040073BD5002000900598A169002325
:10C2200042181946204601F07BFBD8B9502080F314
:10C230001188BFF34F8FBFF36F8FFEE714F8280FFD
:10C2400020F00100207022E094F8280040F0010066
:10C2500084F828000598A06128B18118134620466B
:10C26000FFF778FF13E0502080F31188BFF34F8F62
:10C27000BFF36F8FFEE794F82800810703D42046B0
:10C2800000F05EFC03E020F0010084F828000022AA
:10C2900004A9286801F042F8002889D109B030BD0E
:10C2A000100100202DE9FC410F46054600F0C4FDB9
:10C2B00001A800F067F80446019818B101F09EFA51
:10C2C000BDE8FC81254EAFB130690068D0B30027CE
:10C2D000291B3A46306800F0E1FC01F08FFA002893
:10C2E000EED11F494FF080500860BFF34F8FBFF36E
:10C2F0006F8FE5E7A542EBD801F080FAF06827469A
:10C30000C068C468201D00F083FB94F82800410732
:10C3100019D5A0692B4641193A462046FFF71AFF66
:10C32000A8B100200346014600902A46204601F0AD
:10C33000F7FA60B9502080F31188BFF34F8FBFF335
:10C340006F8FFEE707E020F0010084F82800216AE3
:10C3500020468847B4E70127BAE700001001002013
:10C3600004ED00E00648416B096829B1416BC968DA
:10C37000C9684968816270474FF0FF31FAE70000F1
:10C38000D400002070B5054601F056F9064E04466B
:10C39000B068844203D200F009F8012000E00020D8
:10C3A00028602046B46070BD10010020F8B5194D1A
:10C3B00020E0C068C4680668201D00F029FB216ADF
:10C3C0002046884794F82800400713D5A0693044D8
:10C3D000B04206D924616060211DE86800F058FB76
:10C3E00008E000200346014600903246204601F056
:10C3F00097FA38B1E86801680029DAD12969C5E9F6
:10C400000310F8BD502080F31188BFF34F8FBFF3A6
:10C410006F8FFEE710010020002101E0401C491C45
:10C420000278A52AFAD0C1F38F0070470848406807
:10C43000401C4FF0500080F3118804D0BFF34F8FA1
:10C44000BFF36F8FFEE7BFF34F8FBFF36F8FFEE732
:10C4500044010020074CE068016841B1C068002138
:10C46000D0F80000FFF71EFFFFF79EFEF3E7012163
:10C470000020F7E7100100202DE9F041044600F00C
:10C480002BFB94F9455004F1240609E0606A48B199
:10C49000304601F07BF908B100F050FC6D1E6DB222
:10C4A000002DF3DC4FF0FF3684F8456000F034FBDC
:10C4B00000F012FB94F9445004F1100709E02069E0
:10C4C00048B1384601F062F908B100F037FC6D1E42
:10C4D0006DB2002DF3DC84F84460BDE8F04100F05B
:10C4E0001BBBFDF7A5BB00002DE9F0410546002769
:10C4F00000F0A2FC324E306808B9FFF741FD7069C8
:10C5000005424ED1C5B3083568070ED005F00700C7
:10C51000C0F108000544680707D0502080F3118857
:10C52000BFF34F8FBFF36F8FFEE72DB37068854267
:10C5300037D82348183001460C6801E020460C46E5
:10C540006168A94202D221680029F7D131688C4282
:10C5500027D007682168016060680837411B1029EF
:10C560000FD96019420708D0502080F31188BFF31B
:10C570004F8FBFF36F8FFEE713E041606560FFF7F9
:10C58000C3FD61687068401A7060B268904200D262
:10C59000B060706901430020C4E90001F068401CEC
:10C5A000F06001F02BF9780707D0502080F3118854
:10C5B000BFF34F8FBFF36F8FFEE73846BDE8F081C2
:10C5C0002401002010B5031F4FF080741C601B1F56
:10C5D00021F001011960191F044B0B6014390A6026
:10C5E000091F6FF0020244380A6010BD2DC4000814
:10C5F0002DE9F0479A460023DFF8449189E00025B1
:10C600004FEA090707EBC50637F83540B678A04270
:10C6100026441FFA86FC7DD360457BD2041BA6B25C
:10C62000ACEB0004A4B2A14200D20C4609EBC50554
:10C63000D5F80480ED78A5B1012D15D0022D32D0AA
:10C64000032D7BD14EE0771938F817704FEA172C7D
:10C6500002F803C05B1C9BB2D7545B1C6D1C9BB2E1
:10C66000ADB2A542EFD350E0002519E07719BFB273
:10C670004FEA570C47F3000758F82CC07F1C02D034
:10C680004FEA1C4701E01FFA8CF74FEA172C02F81B
:10C6900003C05B1C9BB2D7545B1C6D1C9BB2ADB23C
:10C6A000A542E3D331E0002519E07719BFB24FEA84
:10C6B000570C47F3000758F82CC07F1C02D04FEAF4
:10C6C0001C4701E01FFA8CF74FEA172C02F803C051
:10C6D0005B1C9BB2D7545B1C6D1C9BB2ADB2A542D8
:10C6E000E3D312E098F8006000253EB1012E1BD084
:10C6F000022E1BD0032E1BD04FF6FF752E0AD654E8
:10C700005B1C9BB2D5545B1C9BB22044091B80B2BE
:10C7100089B201E00EE011E000297FF470AFAAF8C1
:10C7200000300120BDE8F0879225E7E79525E5E791
:10C730009825E3E76D1C3D2DFFF464AF0020F1E781
:10C740005801002006490020064A8860C8609063AE
:10C75000D0631064506488610861087070470000FD
:10C760001C0000106032001070B5174C657B403C17
:10C7700025706070080AA070E170412020710020CF
:10C780006071A271180AE071237200206072A072B9
:10C79000E07220730D212046FEF7D9FA6073000A7B
:10C7A000A07309480F210C46403800F01FF90748D4
:10C7B0000078002806D02146BDE870400248403885
:10C7C00000F0E2B870BD000040320010040000200C
:10C7D00070B5174C657B203C25706070080AA0700E
:10C7E000E1704120207100206071A271180AE0718F
:10C7F000237200206072A072E07220730D21204627
:10C80000FEF7A5FA6073000AA07309480F210C46D1
:10C81000203800F0EBF807480078002806D02146C1
:10C82000BDE870400248203800F0AEB870BD00008E
:10C83000403200100400002070B5174C657B603C4E
:10C8400025706070080AA070E170412020710020FE
:10C850006071A271190AE171237201216172A072E3
:10C86000E07220730D212046FEF771FA6073000A12
:10C87000A07309480F210C46603800F0B7F807484C
:10C880000078002806D02146BDE870400248603894
:10C8900000F07AB870BD00004032001004000020A3
:10C8A0002DE9F0412A4E0D460746002404EB840092
:10C8B00056F820103846F3F788FD40B1641C3E2C32
:10C8C000F4D33946BDE8F04122A0FCF7D5BA04EB19
:10C8D000840006EB8000017C0029284900D0096D06
:10C8E00042685418017A06292CD2DFE801F00A10B8
:10C8F000171E2503C1682B4621A22046FCF7CCFA5F
:10C9000020E00A2200212846F3F761FE12E00A2205
:10C9100000212846F3F793FE207013E00A2200213D
:10C920002846F3F78CFE20800CE0002211462846B2
:10C93000F3F785FE206005E028460021FCF720FB88
:10C9400084ED000ABDE8F0410E48F6F7B4BE0000E1
:10C95000FCDF000873796E635F4A73526F6F745F18
:10C960006669656C643A20756E6B6E6F776E206BCE
:10C970006579203D2025730A000000004032001038
:10C9800025730000302700102DE9F041A0B00F46BC
:10C9900080466E46802130460DA2FCF77DFA0446A3
:10C9A00000250AE018F80530C4F1800130190BA207
:10C9B000FCF772FA6D1C0444ADB2BD4201D27D2C6D
:10C9C000F0D3694607A0F4F77DFF20B0BDE8F08101
:10C9D00054585F4255463A20000000002530325836
:10C9E0002000000025730D0A0000000070B50C4601
:10C9F00005460122D1024FF09040F6F71DFE224677
:10CA00002946BDE870400148F8F71CBEA427001075
:10CA1000D0E9013201699A60D0E901235A604A687D
:10CA2000824201D182684A60002202610868401E89
:10CA3000086008687047000008B902480068006B89
:10CA4000FFF7EABCD4000020034B036003F15C0055
:10CA50000860802010607047282B0010044B036092
:10CA600003F15C0008604FF48070106070470000B4
:10CA7000842D001000F108014FF0FF32C0E90112CF
:10CA8000C1600161002101607047002101617047B0
:10CA900030B50B685A1C02D000F1080202E00269AE
:10CAA00004E02246546825689D42FAD953684B60D9
:10CAB00099608A60516008610168491C016030BD5D
:10CAC00042684A6093688B6093685960916008611E
:10CAD0000168491C01607047502080F31188BFF342
:10CAE0004F8FBFF36F8F0A494868401C4860012888
:10CAF0000CD10848006810F0FF0F07D0502080F3D9
:10CB00001188BFF34F8FBFF36F8FFEE770470000B0
:10CB10004401002004ED00E00849486828B1401EA7
:10CB2000486001D180F311887047502080F311884C
:10CB3000BFF34F8FBFF36F8FFEE70000440100206B
:10CB400070B500282AD0164DA0F108046068696904
:10CB5000084207D1502080F31188BFF34F8FBFF3F5
:10CB60006F8FFEE722683AB1502080F31188BFF33F
:10CB70004F8FBFF36F8FFEE78843606000F05CF972
:10CB800060686968084468602046FFF7BDFA286954
:10CB9000401C2861BDE8704000F030BE70BD000050
:10CBA000240100204FF0E02000210161816105494E
:10CBB0004FF47A720968B1FBF2F1491E4161072115
:10CBC00001617047D000002010B5F3F745FB114913
:10CBD00010280ED300F1E02090F8F0030A7890427C
:10CBE00007D2502080F31188BFF34F8FBFF36F8FB0
:10CBF000FEE709480068896800F4E060884207D9C8
:10CC0000502080F31188BFF34F8FBFF36F8FFEE783
:10CC100010BD0000440100200CED00E010B5084BF1
:10CC2000002200BF53F832401CB1521C082AF9D32D
:10CC300010BD43F8321003EBC201486010BD000084
:10CC40002C3E002010B504000AD000F013F894F830
:10CC5000460000280CD12046BDE81040FFF770BF09
:10CC6000502080F31188BFF34F8FBFF36F8FFEE723
:10CC700010BD0000084A002102EBC1035B6883423B
:10CC800006D1002042F8310002EBC1014860704734
:10CC9000491C0829F0D370472C3E002070B515467A
:10CCA0000E460446FFF718FF94F944100020491C73
:10CCB00001D184F8440094F94510491C01D184F84D
:10CCC0004500FFF729FFA06B28B92A46314604F139
:10CCD000240000F051F82046BDE87040FFF7CCBBBF
:10CCE00010B5020014D00F48006B38B1502080F30B
:10CCF0001188BFF34F8FBFF36F8FFEE700F09CF8F2
:10CD000000211046FFF716F800F078FD002807D143
:10CD100005494FF080500860BFF34F8FBFF36F8F0E
:10CD200010BD0000D400002004ED00E002490A6AB2
:10CD30000260C96841607047D400002001490120A9
:10CD4000C8617047D400002010B50C4650B10949A5
:10CD500009681831FFF79CFE2046BDE8104001210C
:10CD6000FEF7E8BF502080F31188BFF34F8FBFF369
:10CD70006F8FFEE7D400002070B514460D4668B1F1
:10CD80000A4909681831FFF79BFE0CB14FF0FF35D7
:10CD900021462846BDE87040FEF7CCBF502080F306
:10CDA0001188BFF34F8FBFF36F8FFEE7D4000020D1
:10CDB00030B587B00024039405AA04A903A80494FD
:10CDC000FFF742FEDDE903010094CDE901100023E5
:10CDD00015A11748059A00F0F5FB164D0028E862EA
:10CDE0001FD000F06DFD012809D0401C19D1502042
:10CDF00080F31188BFF34F8FBFF36F8FFEE7502092
:10CE000080F31188BFF34F8FBFF36F8F4FF0FF3068
:10CE1000A86201206861EC6007B0BDE8304000F016
:10CE200045B807B030BD000049444C450000000043
:10CE3000CDBF0008D40000200248016B491C0163EB
:10CE400070470000D4000020164810B5016B11B1E6
:10CE50000121C16110BD0021C1610169124A01E0D7
:10CE6000B9B1491E01EB810352F82330002BF7D0F2
:10CE700001EB810302EB830202F1080453685B6853
:10CE80005360A34201D15B685360DA6802600161BC
:10CE900010BD502080F31188BFF34F8FBFF36F8F09
:10CEA000FEE70000D40000206C3E00201CB537488F
:10CEB0000168374A914207D1502080F31188BFF3AF
:10CEC0004F8FBFF36F8FFEE700683149491E8842DC
:10CED00007D1502080F31188BFF34F8FBFF36F8FBE
:10CEE000FEE72C4908780190FF20087008788DF83B
:10CEF00000009DF800009DF8002000F0F000904236
:10CF000007D0502080F31188BFF34F8FBFF36F8F8E
:10CF1000FEE79DF80000204C00F050002070072034
:10CF2000A06005E09DF8002052008DF80020401E12
:10CF30009DF800201206F5D4A060032807D05020E9
:10CF400080F31188BFF34F8FBFF36F8FFEE74FF46D
:10CF50004070A060019808700C482030016841F4CE
:10CF600070010160016841F070410160FFF71AFE35
:10CF700000206060F3F738F90848016841F040414B
:10CF80000160F3F71DF900201CBD000000ED00E07A
:10CF900071C20F4100E400E04401002034EF00E0E2
:10CFA00010B5502080F31188BFF34F8FBFF36F8F00
:10CFB00000F048FB18B104494FF080500860002091
:10CFC00080F3118810BD000004ED00E0F8B51746AD
:10CFD0000E46050013D005FB06F05030FFF784FA2B
:10CFE00004000AD0002084F8460004F150023B46B9
:10CFF000314628460094FFF719F82046F8BD502026
:10D0000080F31188BFF34F8FBFF36F8FFEE738B502
:10D01000049D18B153B1CAB181B120E0502080F312
:10D020001188BFF34F8FBFF36F8FFEE7502080F35F
:10D030001188BFF34F8FBFF36F8FFEE7502080F34F
:10D040001188BFF34F8FBFF36F8FFEE739B15020C8
:10D0500080F31188BFF34F8FBFF36F8FFEE750242B
:10D060001C46012384F846302B460094FEF7DEFF71
:10D07000204638BD70B50D46040025D0FFF72CFDC5
:10D08000D4E90F20216802FB0011A1600021A163F7
:10D09000216861600A46D4E90F01401E00FB0121AE
:10D0A000E16021464FF0FF3001F8440F487004F171
:10D0B00010008DB1FFF7DEFC04F12400FFF7DAFC6D
:10D0C000FFF72AFD012070BD502080F31188BFF3C7
:10D0D0004F8FBFF36F8FFEE721690029F0D000F07A
:10D0E00055FB0028ECD004494FF080500860BFF396
:10D0F0004F8FBFF36F8FE3E704ED00E02DE9FF47AB
:10D1000082B01D468A464FF00008040003D0BAF1F1
:10D11000000F08D011E0502080F31188BFF34F8F2B
:10D12000BFF36F8FFEE7206C38B1502080F3118879
:10D13000BFF34F8FBFF36F8FFEE7022D0AD1E06B75
:10D14000012807D0502080F31188BFF34F8FBFF321
:10D150006F8FFEE700F062FA3F4F4FF000094FF08B
:10D16000805648B9049838B1502080F31188BFF335
:10D170004F8FBFF36F8FFEE7FFF7AEFCA06BE16B45
:10D18000884207D3022D05D00498D0B1B8F1000F22
:10D190001AD01EE02A4651462046FEF7A0FE616ADC
:10D1A00019B104F1240000F0F1FA20B13E60BFF3A0
:10D1B0004F8FBFF36F8FFFF7AFFC012006B0BDE8C4
:10D1C000F087FFF7A9FC22E06846FFF7AFFD4FF0BC
:10D1D0000108FFF7A1FCFFF72FFEFFF77DFC94F994
:10D1E0004400401C01D184F8449094F94500401C4F
:10D1F00001D184F84590FFF78FFC04A9684600F040
:10D2000077F930B12046FFF737F900F0F7FA002040
:10D21000D4E7FFF761FCA06BE16B884213D1FFF705
:10D220007BFC04F110000499FFF78EFD2046FFF708
:10D2300023F900F0E3FA00289ED13E60BFF34F8F40
:10D24000BFF36F8F98E7FFF767FC2046FFF714F9ED
:10D2500000F0D4FA90E7000004ED00E02DE9F0477B
:10D260001F4690468946040003D0B9F1000F08D04C
:10D2700011E0502080F31188BFF34F8FBFF36F8F01
:10D28000FEE7206C38B1502080F31188BFF34F8F38
:10D29000BFF36F8FFEE7022F0AD1E06B012807D0A2
:10D2A000502080F31188BFF34F8FBFF36F8FFEE7DD
:10D2B000FFF78AFC5020EFF3118680F31188BFF34B
:10D2C0004F8FBFF36F8FA06BE16B884206D3022FA5
:10D2D00004D0002086F31188BDE8F08794F945500A
:10D2E000A06B3A4649462046FEF7F9FD681C04D07B
:10D2F0006D1C84F845500120ECE7606A0028FAD0E4
:10D3000004F1240000F042FA0028F4D0B8F1000F34
:10D31000F1D00121C8F80010EDE700002DE9F74732
:10D32000002683B08A46040003D0BAF1000F08D06B
:10D3300011E0502080F31188BFF34F8FBFF36F8F40
:10D34000FEE7206C38B1502080F31188BFF34F8F77
:10D35000BFF36F8FFEE700F061F9DFF8F4804FF064
:10D3600000094FF0805748B9059838B1502080F334
:10D370001188BFF34F8FBFF36F8FFEE7FFF7ACFB52
:10D38000A56BC5B151462046FEF796FD6D1EA563FF
:10D39000206950B104F1100000F0F8F928B1C8F884
:10D3A0000070BFF34F8FBFF36F8FFFF7B5FB012006
:10D3B00006B0BDE8F087059808B11EB106E0FFF79A
:10D3C000ABFB27E06846FFF7B1FC0126FFF7A4FBA3
:10D3D000FFF732FDFFF780FB94F94400401C01D1B8
:10D3E00084F8449094F94500401C01D184F845909C
:10D3F000FFF792FB05A9684600F07AF8002820465E
:10D400000AD0FFF739F800F0F9F92046FEF7BEFE22
:10D410000028B3D00020CBE7FEF7B8FE90B104F1AE
:10D4200024000599FFF790FC2046FFF725F800F04F
:10D43000E5F90028A2D1C8F80070BFF34F8FBFF301
:10D440006F8F9BE72046FFF717F800F0D7F995E7B5
:10D4500004ED00E02DE9F04790468946040003D032
:10D46000B9F1000F08D011E0502080F31188BFF30C
:10D470004F8FBFF36F8FFEE7206C38B1502080F3E1
:10D480001188BFF34F8FBFF36F8FFEE7FFF79CFB51
:10D490005020EFF3118680F31188BFF34F8FBFF355
:10D4A0006F8FA76BF7B194F9445049462046FEF7B9
:10D4B00003FD7F1EA763681C04D06D1C84F84450D4
:10D4C000012010E020690028FAD004F1100000F0DB
:10D4D0005DF90028F4D0B8F1000FF1D00121C8F8AF
:10D4E0000010EDE7002086F31188BDE8F08700000A
:10D4F0002DE9F0410C46050011D0C4B1FFF7ECFA5C
:10D50000174BDA686E682068911B471C17D02F688C
:10D510001B6A9F4219D0964217D8012410E0502070
:10D5200080F31188BFF34F8FBFF36F8FFEE750205A
:10D5300080F31188BFF34F8FBFF36F8FFEE7002496
:10D54000FFF7EAFA2046BDE8F081884205D9401A83
:10D5500020602846FFF7EAFBF1E700202060DCE7C7
:10D56000D40000202DE9FF5F8346DDE90E87994650
:10D5700016468A469000FEF7B7FF05001CD05C20D7
:10D58000FEF7B2FF040014D00020256384F8590090
:10D59000CDE90240CDE900874B4632465146584618
:10D5A000FEF756FD2046FEF7F3FB012004B000F025
:10D5B00006B82846FFF7C4FA4FF0FF30F6E730BC54
:10D5C000BDE8C09FF0B585B0DDE90B640A9DA6B14A
:10D5D000DCB15C2700972663022684F85960002698
:10D5E00004AFCDE90246CDE90057FEF731FD2046F4
:10D5F000FEF7CEFB049805B0F0BD502080F31188F3
:10D60000BFF34F8FBFF36F8FFEE7502080F3118879
:10D61000BFF34F8FBFF36F8FFEE7000005484169EE
:10D6200019B1006B18B1002070470120704702202B
:10D6300070470000D40000200148C0687047000017
:10D64000D40000202DE9F0412E4C0027206B28B19A
:10D65000A069401CA0613846BDE8F081E668761CF0
:10D66000E66013D1606B006838B1502080F31188F8
:10D67000BFF34F8FBFF36F8FFEE7606BA16B6163EA
:10D68000A063206A401C2062FEF76CFEA06ADFF8EF
:10D690007880864209D3606B0068A0B1606BC06877
:10D6A000C5686868864211D2A0622068C06A00EB33
:10D6B000800158F82100012800D90127E0690028DD
:10D6C000C9D00127C7E74FF0FF30EDE7281DFFF76E
:10D6D0009FF9A86A18B105F11800FFF799F9E86AEF
:10D6E0002169884200D9206100EB800108EB8100AC
:10D6F000291DFFF7E5F9E86A2168C96A8842CAD39B
:10D700000127C8E7D40000206C3E002070B504005B
:10D710004FF0000133D01B4D2868844207D05020C1
:10D7200080F31188BFF34F8FBFF36F8FFEE7206D3B
:10D7300038B1401E2065E36CE26A9A421FD040B1C6
:10D740001DE0502080F31188BFF34F8FBFF36F8F20
:10D75000FEE7201DFFF75CF9E06CE062C0F13800E5
:10D76000A061E06A2969884200D92861064900EB76
:10D77000800001EB8000211DFFF7A2F9012108467E
:10D7800070BD0000D40000206C3E002070B5C06861
:10D79000C46854B104F118000646FFF739F9144D76
:10D7A000286B50B13146134815E0502080F31188A2
:10D7B000BFF34F8FBFF36F8FFEE7201DFFF728F9F0
:10D7C000E06A2969884200D928610B4900EB800092
:10D7D00001EB8000211DFFF773F9E06A2968C96A2F
:10D7E000884202D90120E86170BD002070BD0000B0
:10D7F000D4000020F44200206C3E00202DE9F047C8
:10D800002C4D00242746286B38B1FFF765F9286BAB
:10D81000401E2863286B40B146E0502080F31188F9
:10D82000BFF34F8FBFF36F8FFEE7A968224E012031
:10D83000D1B3A6F5916980463068E0B1F068C4685C
:10D8400004F11800FFF7E4F8201DFFF7E1F8E06AA3
:10D850002969884200D9286100EB800109EB810029
:10D86000211DFFF72DF9E06A2968C96A8842E3D3D0
:10D87000C5F81C80E0E70CB1FEF774FDAC694CB153
:10D880004FEA0806FFF7DEFE00B1EE61641EF9D133
:10D890000020A861E86938B1084901273807086005
:10D8A000BFF34F8FBFF36F8FFFF736F93846BDE8F0
:10D8B000F0870000D4000020F442002004ED00E0D6
:10D8C00010B586B0FEF7CCFA114C2068B8B1002034
:10D8D0000390049005AA04A903A8FFF7BFF8DDE9A7
:10D8E000032102208DE8070000230AA10B48059AB6
:10D8F000FFF768FE606010B106B0012010BD502037
:10D9000080F31188BFF34F8FBFF36F8FFEE70000E6
:10D9100010010020546D72205376630055C4000836
:10D920002DE9FF411E46134602000A9D4FF00000FC
:10D9300016D0144C2768002F0FD0CDE900130292A7
:10D94000062917DAFFF76AFE02284FF000030FD00E
:10D95000002269462068FFF7D1FB04B0BDE8F081E2
:10D96000502080F31188BFF34F8FBFF36F8FFEE716
:10D970002A46EEE70023324669463846FFF76EFC3A
:10D98000EBE700001001002014E600080000000092
:10D990000000000000000000000000000004000083
:10D9A000300000000000000000000000E4E5000876
:10D9B0000000000000000000000000000000000067
:10D9C000000400001800000000000000000000003B
:10D9D000F0E500080000000000000000000000006A
:10D9E0000000000000080000180000000000000017
:10D9F00000000000FCE5000800000000000000003E
:10DA000000000000000000000008000010000000FE
:10DA100000000000000000006CE5000800000000AD
:10DA200000000000000000000000000000040000F2
:10DA300018000000000000000000000008E60008D8
:10DA400000000000000000000000000000000000D6
:10DA500000020000200000000000000000000000A4
:10DA6000D4E5000800000000A018002050000000CD
:10DA70006003002040150000C8E500080000000019
:10DA80008824001050000000C8020010C0210000CF
:10DA9000B8E5000800000000F03A00205000000047
:10DAA000F01800200022000088E5000800000000B7
:10DAB0005025001050000000D8240010780000000D
:10DAC00078E5000800000000403B00205000000006
:10DAD000A0250010780000005CE5000800000000B0
:10DAE0001826001050000000903B00207800000035
:10DAF00098E5000800000000083C002050000000ED
:10DB00006826001078000000A8E50008000000006A
:10DB1000E026001050000000583C00207800000073
:10DB200000000000000000000102030406070809CD
:10DB3000A0860100400D0300801A060000350C008D
:10DB400040420F0080841E0000093D0000127A0050
:10DB50000024F40000366E010048E801006CDC028D
:10DB60000000000001020304D5F85B42AAF15B4209
:10DB70007FEA5B424EE25B4217D95B42ECD15B42EB
:10DB8000BAC95B4289C15B4233B35B42DDA45B42ED
:10DB9000A09A5B420000B4420000B6420000B842C6
:10DBA0000000BA420000BC420000BE420000C04279
:10DBB0000000C2420000C4420000C6420000C84249
:10DBC000A602EB431B0EDE43EBE3D1439B76C64339
:10DBD000A3B9BB4368A1B1431C23A843B6349F43F8
:10DBE000E7CC964309E38E43006F8743586980432F
:10DBF000189673433D1B6743FE555B430F3B5043F1
:10DC0000DFBF4543A0DA3B4320823243CCAD2943FA
:10DC1000A85521433A72194385FC114301EE0A438A
:10DC20008A400443E0DCFB42A9E4EF42638EE44215
:10DC3000B1D0D942D1A2CF426AFCC542D0D5BC42B4
:10DC4000C827B44278EBAB42781AA442CCAE9C42CF
:10DC5000D1A2954241F18E4225958842BA898242ED
:10DC600067957942BBA76E42AA426442ED5E5A4272
:10DC70008EF550420000484238783F42795837428A
:10DC8000239B2F424A3B2842EB3321429D801A427C
:10DC9000E01C1442D0040E426E34084224A8024212
:10DCA00024B9FA41E09CF0415AF5E641D3BCDD418C
:10DCB00091EDD441AA82CC413277C44174C6BC41B3
:10DCC000BA6BB5415463AE412AA9A7415839A14165
:10DCD00062109B41CE2A9541BC858F411B1E8A4113
:10DCE000A4F084412BF67F41257576414B596D4157
:10DCF0001B9E64417D3F5C41EF38544159864C4145
:10DD00000B244541560E3E418941374130BB3041DD
:10DD100032772A4182732441DAAC1E415C201941DA
:10DD2000FBCB1341DAAC0E41ECC00941BC05054107
:10DD3000A77900416E34F840C1CAEF40D0B3E74044
:10DD400085EBDF40986ED840C139D1408C4ACA403B
:10DD5000E09CC3401B2FBD40C5FEB6409A08B140B1
:10DD6000234AAB408FC2A540C66DA040234A9B40CA
:10DD7000D65696409790914094F68C4059868840AC
:10DD8000423E84407E1D8040D044784018957040CB
:10DD9000302A6940D2006240FC185B40226C54403B
:10DDA000E7FB4D4061C34740ECC04140E5F23B40DA
:10DDB000A857364091ED30405BB12B4005A326407B
:10DDC00048BF214081041D40B07218408E061440A7
:10DDD0001AC00F40B29D0B40B29D07401AC00340CD
:10DDE000A301004055C1F83FA5BDF13FF1F4EA3F62
:10DDF000AA60E43F1904DE3FF5DBD73FF7E4D13FEB
:10DE0000DA1BCC3FE483C63F00C0030800C8030808
:10DE100000D003080000000010E800080000000027
:10DE2000A4E9000800000000ACE9000800000000C0
:10DE3000A0EB00080000000018EA00080000000045
:10DE4000F8EC0008010000005CEC00080100000094
:10DE500060EB000801000000CCEB000801000000AE
:10DE6000F0EA000801000000B0EA0008010000002C
:10DE700070EB000801000000E8E900080100000064
:10DE800034EC00080100000084E9000801000000F3
:10DE900000EB00080100000080EB0008010000001A
:10DEA00050EB000801000000F8E900080100000044
:10DEB00008EA00080100000058ED00080100000019
:10DEC000BCEB00080100000010EB0008010000009E
:10DED0002CED00080100000070EA000801000000BD
:10DEE00068ED00080100000024EC000801000000BB
:10DEF0001CED00080100000094E90008010000008A
:10DF0000ACEB0008010000000CED0008010000006F
:10DF100014EC000801000000A0EA00080100000065
:10DF200090EB0008010000006CEC0008010000000C
:10DF30003CED00080100000088EC00080100000032
:10DF4000A8E800080100000044E800080100000003
:10DF5000D0EC00080100000080EA00080100000089
:10DF60002CE9000801000000B8E8000801000000EA
:10DF700054E8000801000000E4EC00080100000083
:10DF800090EA00080100000040E9000801000000DC
:10DF9000B8EC000801000000DCE800080100000007
:10DFA000C8E800080100000080E800080100000047
:10DFB00068E8000801000000A0EC00080100000073
:10DFC000F0E800080100000098E8000802000000E6
:10DFD0001CE90008020000000CE900080200000033
:10DFE00024E800080200000024EA00080200000003
:10DFF00030EA00080200000034E8000884ED000860
:10E0000000000000050000000D00000000000000FE
:10E0100090ED000810000000000000000400000067
:10E020000000000098ED0008400000000000000023
:10E0300004000000000000008CEE00080D0000004D
:10E04000010000000100000000000000F4ED0008E5
:10E050004400000000000000040000000000000078
:10E0600064EE00081400000003000000040000003B
:10E0700000000000A0EE00083000000003000000D7
:10E08000040000000000000000EE00082000000076
:10E09000000000000400000000000000DCEB0008AD
:10E0A000240000000500000009000000000000003E
:10E0B00088ED0008340000000200000002000000AB
:10E0C0000000000058EE00084800000000000000BA
:10E0D000040000000000000094EE00084C00000066
:10E0E0000000000004000000000000004CEE0008EA
:10E0F00038000000000000000400000000000000E4
:10E1000054E90008000000000400000004000000C2
:10E1100001000000B8E9000804000000040000004D
:10E12000040000000100000040EA000808000000B0
:10E13000040000000400000001000000C0EA000824
:10E140000C000000040000000400000001000000BA
:10E1500020EB000810000000040000000400000094
:10E1600001000000E4EB00081400000004000000BF
:10E17000040000000100000044EC0008180000004A
:10E180000400000004000000010000006CE9000829
:10E190001C0000000400000004000000010000005A
:10E1A000D0E9000820000000040000000400000086
:10E1B0000100000058EA00082400000004000000EC
:10E1C0000400000001000000D8EA00082800000058
:10E1D00004000000040000000100000038EB00080B
:10E1E0002C000000040000000400000001000000FA
:10E1F000FCEB0008300000000400000004000000F8
:10E200000100000050EC0008340000000400000091
:10E2100004000000010000007CEC00083800000051
:10E220000400000004000000010000004CED0008A4
:10E230003C00000004000000040000000100000099
:10E2400078ED000840000000040000000400000019
:10E250000100000000E90008440000000400000084
:10E26000040000000100000060E9000860000000F8
:10E27000040000000400000001000000C4E90008E0
:10E280006400000004000000040000000100000021
:10E290004CEA0008680000000400000004000000D0
:10E2A00001000000CCEA00086C000000040000003F
:10E2B00004000000010000002CEB000870000000CA
:10E2C000040000000400000001000000F0EB000862
:10E2D00074000000040000000400000001000000C1
:10E2E00078E9000848000000040000000400000075
:10E2F00001000000DCE900084C0000000400000000
:10E30000040000000100000064EA00085000000062
:10E31000040000000400000001000000E4EA00081E
:10E320005400000004000000040000000100000090
:10E3300044EB000858000000040000000400000046
:10E340000100000008EC00085C0000000400000070
:10E350000400000001000000B0EE0008780000009A
:10E3600004000000040000000100000008EE0008A6
:10E370007C00000004000000040000000100000018
:10E38000A0ED000880000000020000000200000074
:10E390000100000000EF00088400000004000000FD
:10E3A00004000000010000006CEE0008880000007E
:10E3B000040000000400000001000000E0EE00087E
:10E3C0008C000000040000000400000001000000B8
:10E3D00014EE00089000000004000000040000009B
:10E3E00001000000ACED00089400000002000000F5
:10E3F000020000000100000010EF0008980000007B
:10E400000400000004000000010000007CEE000891
:10E410009C00000004000000040000000100000057
:10E42000F0EE0008A000000004000000040000005E
:10E4300001000000D0EE0008A4000000040000006D
:10E44000040000000100000030EE0008A8000000F9
:10E4500004000000040000000100000020EE00089D
:10E46000AC000000040000000400000001000000F7
:10E47000D0ED0008B0000000020000000200000023
:10E4800001000000BCED0008B20000000200000026
:10E490000200000001000000C0EE0008B40000000F
:10E4A00004000000040000000100000040EE00082D
:10E4B000B80000000400000004000000010000009B
:10E4C000E4ED0008BC0000000200000002000000B3
:10E4D0000100000000404040404040404040414179
:10E4E0004141414040404040404040404040404029
:10E4F00040404040400502020202020202020202C3
:10E5000002020202022020202020202020202002BF
:10E51000020202020202909090909090101010104F
:10E5200010101010101010101010101010101010EB
:10E53000020202020202888888888888080808087F
:10E54000080808080808080808080808080808084B
:10E550000202020240000000D5E4000866696C7403
:10E560006572717565756531000000005265616402
:10E570005461736B3032000066696C74657271753A
:10E58000657565320000000066696C7465727175AE
:10E59000657565330000000066696C74657271759D
:10E5A000657565340000000066696C74657271758C
:10E5B0006575653500000000636F6E736F6C656D87
:10E5C00073677175657565007072696E74717565D4
:10E5D00075650000756172743438357278717565CF
:10E5E00075650000526561645461736B0000000042
:10E5F0004465616C5461736B00000000436F6D6D86
:10E600006F6E5461736B000046696C74657254617F
:10E61000736B0000486967686573745461736B00BD
:10E62000726F645F766F6C5F6F66667365743D25AD
:10E630002E33662C20726F645F6469616C6F673D76
:10E64000252E33662C206F696C5F706172615F6983
:10E650006E64753D252E33662C206F696C5F70618A
:10E6600072615F6361703D252E33662C206F696C8B
:10E670005F6361705F6F66667365743D252E3366F8
:10E680002C206F696C5F6469616C6F673D252E3368
:10E69000662C20726F645F636F6C74696D653D25D5
:10E6A000640A00007265735F706172615F696E6415
:10E6B000753D252E33662C207265735F7061726123
:10E6C0005F6361703D252E33662C207265735F6336
:10E6D00061705F6F66667365743D252E33662C200E
:10E6E0007265735F766F6C5F6F66667365743D25E8
:10E6F0002E33662C207265735F6361705F6469619D
:10E700006C6F673D252E33662C207265735F766FC4
:10E710006C5F6469616C6F673D252E33662C2072D7
:10E7200065735F6F696C5F6361705F636F6C746961
:10E730006D653D25642C207265735F6F696C5F7633
:10E740006F6C5F636F6C74696D653D25640A0000D2
:10E750006D61633D25732C20616464723D25752CC9
:10E7600020726F6C653D25642C20766572735F693D
:10E77000643D25752C206167653D25642C2061670B
:10E78000655F6D733D256C642C2069617053697AF7
:10E79000653D25642C206961704D64353D25732CE1
:10E7A000206961704C6F61645374617475733D25A9
:10E7B000752C20737562636F64653D25752C20751B
:10E7C000626F6F746261636B3D25642C20646562C7
:10E7D00075673D25642C20636F6E736F6C653D25F6
:10E7E000642C2062617564726174653D25642C201F
:10E7F0007570646174655F6F6B3D25642C20757066
:10E80000646174655F6572723D25640A00000000F2
:10E810006D61633D30303138303030303030303041
:10E82000000000006961706D64353D30303030307B
:10E830003030300075626F6F746261636B3D3430ED
:10E8400030000000726F645F636F6C74696D653DCA
:10E8500031300000726F645F6F696C5F636F6C745E
:10E86000696D653D313000007265735F6F696C5F83
:10E87000766F6C5F636F6C74696D653D313000005D
:10E880007265735F6F696C5F6361705F636F6C74F7
:10E89000696D653D3130000074656D705F636F6C4C
:10E8A00074696D653D313000726F645F6469616CDD
:10E8B0006F673D31300000006F696C5F6469616CA7
:10E8C0006F673D31300000007265735F766F6C5F7B
:10E8D0006469616C6F673D31300000007265735F81
:10E8E0006361705F6469616C6F673D313000000087
:10E8F00074656D705F6469616C6F673D31300000F5
:10E900006F696C5F63617031300000006961707322
:10E91000697A653D34303936300000006961704CE9
:10E920006F61645374617475733D30006F696C5F1F
:10E930006361705F6F66667365743D300000000050
:10E940007265735F6361705F6F66667365743D3097
:10E9500000000000726F645F766F6C300000000092
:10E960007265735F766F6C30000000006F696C5FDA
:10E9700063617030000000007265735F6361703026
:10E98000000000006F696C5F636170313D322E30B2
:10E99000310000007265735F766F6C343D322E3843
:10E9A00032310000726F6C653D310000636F6E7331
:10E9B0006F6C653D31000000726F645F766F6C3183
:10E9C000000000007265735F766F6C31000000001C
:10E9D0006F696C5F63617031000000007265735F86
:10E9E0006361703100000000726F645F766F6C3697
:10E9F0003D342E34303200006F696C5F63617035D6
:10EA00003D332E31320000006F696C5F63617036F8
:10EA10003D332E32320000006261756472617465AC
:10EA20003D3200007570646174655F6F6B3D32004C
:10EA30007570646174655F6572723D32000000003C
:10EA4000726F645F766F6C32000000007265735FF6
:10EA5000766F6C32000000006F696C5F636170322A
:10EA6000000000007265735F636170320000000097
:10EA70007265735F766F6C303D322E373133000034
:10EA80006F696C5F706172615F6361703D33330009
:10EA90007265735F706172615F6361703D333300F3
:10EAA0007265735F636170323D312E38363300001A
:10EAB000726F645F766F6C343D332E3836330000EE
:10EAC000726F645F766F6C33000000007265735F75
:10EAD000766F6C33000000006F696C5F63617033A8
:10EAE000000000007265735F636170330000000016
:10EAF000726F645F766F6C333D332E3530340000B7
:10EB00006F696C5F636170323D322E3134000000FA
:10EB10006F696C5F636170393D332E3834000000DB
:10EB2000726F645F766F6C34000000007265735F13
:10EB3000766F6C34000000006F696C5F6361703445
:10EB4000000000007265735F6361703400000000B4
:10EB50006F696C5F636170343D332E3035000000A7
:10EB6000726F645F766F6C313D322E393035000044
:10EB7000726F645F766F6C353D342E313235000034
:10EB80006F696C5F636170333D322E333500000076
:10EB90007265735F636170333D312E35343500002B
:10EBA000616464723D323535000000007265735F48
:10EBB000766F6C353D322E38353500006F696C5FED
:10EBC000636170383D332E3635000000726F645F2C
:10EBD000766F6C323D332E31363500006961706DD1
:10EBE00064350000726F645F766F6C350000000062
:10EBF0007265735F766F6C35000000006F696C5F43
:10EC000063617035000000007265735F6361703589
:10EC1000000000007265735F636170313D322E3316
:10EC2000353600007265735F766F6C323D322E3779
:10EC3000363600006F696C5F636170303D312E388D
:10EC400036000000726F645F766F6C360000000063
:10EC50006F696C5F6361703600000000726F645F03
:10EC6000766F6C303D322E36333700007265735F3D
:10EC7000636170343D392E38370000006F696C5F76
:10EC80006361703700000000726F645F766F6C5FC5
:10EC90006F66667365743D302E30303800000000BA
:10ECA00074656D705F766F6C5F6F66667365743DDB
:10ECB000302E3030380000007265735F766F6C5F05
:10ECC0006F66667365743D302E303038000000008A
:10ECD0006F696C5F706172615F696E64753D313838
:10ECE000000000007265735F706172615F696E643D
:10ECF000753D31380000000076657273696F6E3DB6
:10ED00003030303743313238000000007265735FB5
:10ED1000636170303D322E36373800007265735FA4
:10ED2000766F6C333D322E37383800006F696C5F78
:10ED300063617031303D332E393800007265735F86
:10ED4000636170353D332E39380000006F696C5FA8
:10ED500063617038000000006F696C5F6361703739
:10ED60003D332E33390000007265735F766F6C316E
:10ED70003D322E37333900006F696C5F6361703943
:10ED8000000000006D616300737562636F6465006D
:10ED9000726F6C6500000000636F6E736F6C6500CE
:10EDA000726F645F636F6C74696D6500726F645F2E
:10EDB0006F696C5F636F6C74696D65007265735F1A
:10EDC0006F696C5F766F6C5F636F6C74696D650003
:10EDD0007265735F6F696C5F6361705F636F6C74A2
:10EDE000696D650074656D705F636F6C74696D65E6
:10EDF00000000000626175647261746500000000CB
:10EE000069617073697A6500726F645F6469616CCF
:10EE10006F6700006F696C5F6469616C6F67000009
:10EE20007265735F766F6C5F6469616C6F67000019
:10EE30007265735F6361705F6469616C6F67000026
:10EE400074656D705F6469616C6F670075626F6F88
:10EE5000746261636B0000007570646174655F6F5C
:10EE60006B00000076657273696F6E006F696C5F8E
:10EE7000706172615F636170000000007265735FB2
:10EE8000706172615F6361700000000061646472B0
:10EE9000000000007570646174655F657272000047
:10EEA0006961704C6F616453746174757300000024
:10EEB000726F645F766F6C5F6F6666736574000077
:10EEC00074656D705F766F6C5F6F666673657400F6
:10EED0007265735F766F6C5F6F6666736574000052
:10EEE0006F696C5F6361705F6F6666736574000065
:10EEF0007265735F6361705F6F666673657400004F
:10EF00006F696C5F706172615F696E6475000000AB
:10EF10007265735F706172615F696E647500000095
:10EF200060EF0008000000206003000012150008D8
:10EF30000CF1000800000010C802000012150008C3
:10EF40000CF100086003002048B40000C88F0008DE
:10EF500044F20008C8020010E0340000C88F000826
:10EF600092000180056F12033C0EF00890410000F2
:10EF700004420001011418C13C016801E201890347
:10EF800072093D871300AA016183260211100D400A
:10EF900002015432001002400100580812100812F9
:10EFA0004D08121110128408100620400300402062
:10EFB000112E100702A80000200208122C081204CB
:10EFC000081006040000100618126018100700014F
:10EFD0000103540120120128114812040812AC50F8
:10EFE00012060812B05812080812B460120A081269
:10EFF000B868120C0812BC70120E0822C0781108F2
:10F0000012C47012120812C87812140812CC80129E
:10F01000160812D08812180812D490121A0812D8A2
:10F0200098121C0812DCA0121E0822E0A811081277
:10F03000E4B012220812E80812240812EC08122682
:10F040000812F00812280812F408122A0812F80808
:10F05000122C0812FC08122EB010060033001030DB
:10F06000B81204081232C01208081234C8120C0870
:10F070001236D01210081238D8121408123AE012C0
:10F080001808123CE8121C38150727020818110846
:10F09000152513200408121408120610120C081269
:10F0A0000A10122008120C08122808120E1012184A
:10F0B00008121018121C0812121812240812162016
:10F0C000123808121808124008121A0812440812BE
:10F0D0001C08124C08121E08125008216912300830
:10F0E0001222301234081224301D0D03132026285A
:10F0F000124808122C28125408122E08125C08120A
:10F1000030081258180A1D276E00000092000112E4
:10F110000104032910000100061104004800201416
:10F12000D145100A10400000A5A5000811081006DE
:10F13000D59E00084010124D10124208200549A229
:10F1400000087912C52012053F500E02010200711D
:10F15000A40008A8320010040C12AC0C52060C12C9
:10F16000B00C52080C12B40C520A0C12B80C520C0F
:10F170000C12BC0C520E0C12C00C52100C12C40C0F
:10F1800052120C12C80C52140C12CC0C52160C1247
:10F19000D00C52180C12D40C521A0C12D80C521C4F
:10F1A0000C12DC0C521E0C12E00C52200C12E40C5F
:10F1B00052220C12E80C52240C12EC0C52260C12A7
:10F1C000F00C52280C12F40C522A0C12F80C522C8F
:10F1D0000C12FC0C562E085406003300103014128A
:10F1E000040C56322012080C56342C120C0C5636D5
:10F1F0003812100C56384412140C563A5012180C8F
:10F20000563C5C121C545306023C50050000200E74
:10F210000C12180C52100C121C0C52120C12240C52
:10F2200052200C12300C52220C12340C52240C12AC
:10F230003C0C52260C12480C52300C12580C036035
:04F240008000010049
:040000050800018D61
:00000001FF
